:020000040800F2
:1000000000500020E50100082D020008000000005B
:100010002D0200082D0200082D020008000000003B
:100020000000000000000000000000002D02000899
:100030002D020008000000002D0200082D0200081B
:100040002D0200082D0200082D0200082D020008D4
:100050002D0200082D0200082D0200082D020008C4
:100060002D0200082D0200082D0200082D020008B4
:100070002D0200082D0200082D0200082D020008A4
:100080002D0200082D0200082D0200082D02000894
:10009000391B00082D0200082D0200082D0200085F
:1000A0002D0200082D0200082D0200082D02000874
:1000B0002D0200082D0200082D0200082D02000864
:1000C0002D0200082D0200082D0200082D02000854
:1000D0002D020008AD230008692400080924000847
:1000E0002D0200082D0200082D0200082D02000834
:1000F0002D0200082D0200082D0200082D02000824
:100100002D0200082D0200082D0200082D02000813
:100110002D0200082D0200082D0200082D02000803
:100120002D0200082D0200082D0200082D020008F3
:100130002D02000800000000000000000000000088
:1001400000000000000000000000000000000000AF
:10015000000000000000000000000000000000009F
:10016000000000000000000000000000000000008F
:10017000000000000000000000000000000000007F
:10018000000000000000000000000000000000006F
:10019000000000000000000000000000000000005F
:1001A000000000000000000000000000000000004F
:1001B000000000000000000000000000000000003F
:1001C000000000000000000000000000000000002F
:1001D000000000000000000000000000000000001F
:1001E0005FF8E0F1684620F007018D4601B50A4A44
:1001F0000A4B0B4903E052F8040B43F8040B8B4203
:10020000F9D3084B0849002201E043F8042B8B4244
:10021000FBD300F00DF8FEE7683E00080000002068
:100220005000002050000020E8160020FEE70000EB
:10023000F0B5002087B001F08FF9002001F004FB39
:1002400005AD012001F08AFA284602F0C9FA02231E
:100250008DF81630CA4812338DF817300C33C94C5C
:1002600003612946ADF8143002F061FA4FF40053EF
:10027000236120462946ADF8143002F058FA402395
:10028000236120462946ADF8143002F050FABE4EE4
:100290000024331930599B88294603610834ADF88E
:1002A000143002F044FA282CF3D1B54E8027B54C17
:1002B000776130462946ADF8147002F038FA4FF4F1
:1002C0000043636148F2000220462946ADF814203D
:1002D00002F02DFA2023636120462946ADF8143040
:1002E000019302F024FABC46202340224FF400512F
:1002F00073610120616162610193CDF800C001F07A
:10030000C5FA202131614FF40052491822610120C1
:10031000216101F0BBFADDF800C0994F1CF1FF3CF0
:10032000984D019BE1D1994C10224FF400434FF4BA
:1003300080564FF400517A6163616E6161614918C2
:1003400061610120CDF800C002910392019301F098
:100350009DFA039A019B02993A614FF4005223617E
:1003600001202E612261216101F090FA482306AC40
:100370008DF81730202324F8043D3846214602F03A
:10038000D6F94FF400512846ADF81410214602F07A
:10039000CEF9402228462146ADF8142002F0C7F9D4
:1003A000DDF800C0784D6746EB199B88E859214677
:1003B0000837ADF8143002F0BAF9282FF4D18023B1
:1003C0002146704E6E48ADF8143002F0B0F948F294
:1003D0000001ADF814103046214602F0A8F92022A1
:1003E00021463046ADF8142002F0A1F9642001F056
:1003F000E9F9B36813F0040F14BF0025012501F0DB
:10040000BBFBC4B21CB9B36813F0040F0DD14DB1DE
:100410004FF40000012102F0E5FC4FF40000002140
:1004200002F0E0FC002001F0AFFB002000F01CFB1C
:10043000002000F00FF964B9524B9B6813F0040FD1
:1004400007D0534B1B78422B03D1524B1B78002B08
:1004500044D1202000F0B6FA002C00F08B80102050
:1004600000F0B0FA86E001F0DFF96422B0FBF6F3A9
:10047000B3FBF2F102FB1133B0FBF7F207FB120200
:1004800041F288315B088A42B0FBF6F106FB1101AC
:1004900088BFC3F132030446994294BF0021012171
:1004A000012001F07BF90A23B4FBF3F203FB1244B1
:1004B0000CB900F037FE002000F020FD01F0B4F987
:1004C00044F61F629042CED900F0CEF80028CAD17F
:1004D00025B12C498B6813F0040FC4D002F0E4F965
:1004E0000120002101F05AF92B4BDB78082B2AD18F
:1004F0006FF00700012102F067FC6FF4000001219A
:1005000002F070FC4FF0FF30002102F05DFC4FF074
:10051000FF30002102F066FC55B101214FF40000CC
:1005200002F060FC4FF40000002102F05BFC03E0ED
:100530001A4B1D6004331D60194B1B6883F3088838
:10054000154B1B68984740F2F31401F063F9012042
:10055000014601F023F901F067F9A042FBD901F04F
:1005600059F90120002101F019F901F05DF9A042CB
:10057000FBD9EAE701F04EF9322642F2107772E732
:1005800000080140000C0140303C00080010014010
:10059000D23F0008D33F000804400008405C004000
:1005A00000400008134B1A78032A0CD8124900F0B7
:1005B0007F00D1F800C04FEACC1C4CEA0010086064
:1005C00013D1042212E0072A88BF4FF0FF300FD862
:1005D0000A4900F07F00D1F800C04FEACC1C4CEA79
:1005E0000010086001D1082200E001321A700020DA
:1005F000704700BF14050020500000205C00002060
:1006000070B5134B16461A7888B08DF800205A78CA
:100610000D468DF801209A7804468DF80220DA788C
:100620001B798DF803208DF8043000F0CDFDF72301
:100630008DF805006946204609228DF806508DF890
:1006400007608DF8083000F09BFA08B070BD00BF5D
:10065000E03C000810B9034B187001E04FF0FF3088
:10066000704700BF15050020014B1878704700BF88
:1006700015050020F7B51E460D461746044600F046
:1006800099FD01F0C7F8012E06D0022E18BF4FF0D9
:10069000FF3040F0748189E01DB1012DBC4B0BD1BE
:1006A00005E0BB4B1D70BB4B1D60BB4B91E01B7845
:1006B000072B00F2638197E01B78082B40F0E48061
:1006C000B44BB64D1F68B44B1E68B54B1A782A70F0
:1006D0005A786A709A78AA70DA781B79EA702B7166
:1006E00000F072FD4FEA566C6871780E0223E871D3
:1006F000C7F386416044AB712972C7F3C623411822
:10070000C7F30612C9186B728918C6F386432B7398
:10071000C918C6F3C623C9186B73C6F30613AB73A7
:10072000CB1803F0FF010023AA7285F80BC01A460C
:100730000F351846019422E010F807E04FF0000C46
:1007400001334FEADE14DBB244EA42024FEA4E0EB6
:10075000062BD2B25FFA8EFE09D9C3F107039A4085
:10076000D2B25118002305F8012BC9B21A460CF178
:10077000010C5FFA8CFCBCF1080FE1D10130B042F2
:10078000DAD1019C1BB1511805F8012BC9B24942BD
:100790002A4601F07F0102F8011B8049F72301324C
:1007A0006B70521A204600F0EBF9E7E015B1012D0D
:1007B0005CD111E0764B1D70764B1D60764B1D6051
:1007C000784B1D70784B1D70784B1D60784B1D6009
:1007D000784B1D602846D2E06D4B1878072807D863
:1007E000704B1A78BA181A703846FFF7DBFEC5E06E
:1007F000082832D16B4B1A78BA181A706B4B1B68E9
:10080000B3F5806F80F0BA80634A644E1468694A19
:100810004FF0000C1168664A254612680132C7F392
:1008200080147F00072A44EA4101FFB205D9F15440
:100830000133AB4228BF092000220CF1010CBCF1AE
:10084000070FEBD1DFF86CC1CCF8001058490A60F3
:10085000564A13604E4B187090E0092804BF524B63
:100860001F7000F08B800C221A7087E04A4B1F68C3
:100870004E4B1B68BB4203D220460E21012213E0DF
:10088000434B1B780C2B03D120460E2132460BE044
:10089000454B1A78434B1B785B4203F07F039A4227
:1008A00005D020460E210322FFF7AAFE66E0424B48
:1008B00001221A70374B1D6845EA070313F0030F36
:1008C0004FD13E4B9D424FD900F0D2FE00F1006067
:1008D0000138854235D801F0DBFF00262DE000937A
:1008E00000F0F0FE00F0C4FE3549009B884294BF42
:1008F0004FF480604FF40060B3FBF0F200FB123065
:1009000028B9184602F028F80428009B0AD1234889
:1009100082195178825D184642EA012101F0FEFFFA
:10092000042807D0142001F0C7FF00F0E1FE6FF0AB
:1009300003021BE000F0DCFE02367319BE42CED388
:100940001EE0B5F1005F0FD300F09AFE00F10050F9
:100950000138854208D8284610493A4603F05DF927
:100960000EE06FF0080201E06FF007025242D2B2CF
:1009700020460E21FFF744FE00F0D4FB0020FEBD10
:10098000084B20461A780F21524202F07F02F1E70D
:1009900014050020500000205C00002064000020AE
:1009A000E03C0008540000206000002010050020FA
:1009B0000C0500205800002015050020FF3F00080E
:1009C000FFFF030010B5114B88B01A7804468DF86C
:1009D00000205A788DF801209A788DF80220DA7874
:1009E0001B798DF803208DF8043000F0EDFB012316
:1009F0008DF805008DF806302046F633694608224A
:100A00008DF8073000F0BCF808B010BDE03C0008DD
:100A100008B52020FFF7D6FF1020FFF7D3FF024BC9
:100A20000020187008BD00BF1505002008B50A4A4F
:100A3000137803F00803DBB23BB1084B1B78834209
:100A400003D100231370064A1370064B1B6803B1D1
:100A50009847002008BD00BF3C0500202805002065
:100A60001D0500202C05002038B504464FF0FF304E
:100A7000002C32D1194A10231370194A20461370E2
:100A8000184B1C60184B1C60184B1C60184B1C60EA
:100A9000184B1C60184B1C6001F0E2F9C50F204692
:100AA00000F0B0FB154A0028B8BF45F0020500234E
:100AB0001370134A1370134A1370134B1B78422B95
:100AC00005D1124B1B7813F0800F08BF1370104A2A
:100AD000002313800F4A6842136038BD00000020D5
:100AE0000100002020050020180500203805002006
:100AF0002C050020300500202405002028050020BA
:100B00003C05002029050020D03F0008D13F000807
:100B10002A0500203405002010F0F00F70B50446BF
:100B20000D4604D101280CBF124B134B1C78134BFC
:100B300004F00F061B682BB166F307152046294603
:100B40009847A8B904F0F004102C05D0202C18BF49
:100B50004FF0FF300CD105E066F30715284601F091
:100B6000F3F905E066F307153046294600F004FC6A
:100B700070BD00BF0100002000000020180500200B
:100B8000F0B585B0174603900D46002606230722D0
:100B90004FF0040C40E0B91B022914D003291FD0E8
:100BA0000129A95D18BF6CF3030406F1010618BF03
:100BB00061F30F241AD1052060F3030461F30F24BD
:100BC0006FF3174409E0A95D63F30304013661F391
:100BD0000F24A95D013661F317446FF31F640DE024
:100BE000A95D62F3030461F30F240136A95D0136A8
:100BF00061F31744A95D013661F31F640398214630
:100C000001920293CDF800C0FFF786FF0028019AF9
:100C1000029BDDF800C002DBBE42BCD3002005B061
:100C2000F0BD000010B5F023A0B08DF80030002317
:100C30008DF801308DF802307E338DF80330322389
:100C40008DF804300E4B0DF16B0C1B788DF80530D0
:100C50000F238DF806306B46DA1D03E002F8014BD6
:100C6000624503D011F8014B002CF7D1F72102F8AF
:100C7000011BD21A6946FFF783FF20B010BD00BFE9
:100C80002905002000B5F02389B08DF8003000233D
:100C90008DF801308DF802307E338DF80330322329
:100CA0008DF80430084B8DF806101B788DF807205E
:100CB0008DF805306946F72309228DF80830FFF7D3
:100CC0005FFF09B000BD00BF29050020F0B5494E07
:100CD0008BB0337804460D461746FFF7CBFC00284F
:100CE00080F2858031780D2964D001D829B174E073
:100CF0000E297CD00F2970D162E01DB1012D3E4B31
:100D000005D102E03C4B1D7071E01F706FE01B7855
:100D1000052B28D00AD8022B18D002D8012B45D198
:100D200011E0032B15D0042B40D115E0082B32D055
:100D300004D8062B21D0072B38D129E0092B2DD040
:100D40007F2B33D12FE020462C4929E020462C4927
:100D500026E020462B4923E000F084FC6D46024645
:100D6000294968460FE0684600F092FC00286D466D
:100D7000BCBF2046254908DA12E000F079FC24497E
:100D800002466D46684601F0C3FC2046694607E00E
:100D900000F076FCF3E720461E4901E01E4920469C
:100DA000FFF740FF23E0FFF733FE20E020460E214F
:100DB0000D220FE0022D1AD120460E21102209E04B
:100DC000164B15B1012D154B01D15D600FE05A682E
:100DD0006AB92046FFF756FF09E00E210A46204671
:100DE000FFF750FF0D4A00231370024A13700020D2
:100DF0000BB0F0BD1D0500201C050020783C00084C
:100E00007F3C00088F3C0008993C00089E3C00088D
:100E1000A03C0008A33C0008B53C00083C050020AD
:100E2000F72910B50A465CD82F4B1C7804F008034C
:100E3000DBB21BB12D49097881424FD1A0F11101DC
:100E4000C9B206294AD9294908700BBB264B1B7821
:100E500003F00703042B03D82549C95C914223D131
:100E600004F00704052C03D12249097891421BD1D3
:100E7000013303F007021C4B052A197862F30201C3
:100E800084BFCAB242F00802197088BF1A7028E005
:100E900012F0800F0ED0F72A06D104F01004E4B24D
:100EA00014B10221FFF712FF0F4B00201870124BF4
:100EB000187017E004F01004E4B25CB90A4B19781A
:100EC00041F0100119700C4B21461A70FFF7FEFE1D
:100ED000204607E00121FFF7F9FE02E04FF0FF3066
:100EE00000E0002010BD00BF3C05002028050020C8
:100EF000E03C0008290500201D050020F0B5012177
:100F000087B000250646029101952B4600E0039B21
:100F10005A1CD2B203920C2B2ED8DFE813F00D002E
:100F200015001B0021002700CA00CA00CA00CA0021
:100F3000CA00CA00CA00CA0005A801F01FF8059C33
:100F4000C4F30314103425E0002005A900F020FAB2
:100F500020241FE0012005A900F01AFA212419E03D
:100F6000022005A900F014FA222413E0032005A9A9
:100F700000F00EFA23240DE001992B1E18BF012367
:100F800009298CBF002303F00103002B40F0C3802C
:100F900002938EE010F10A0F05D12046FFF746FDBF
:100FA0000022029285E00028C0F283800199013579
:100FB0004B1C0599DBB26FF30711019301F00F038E
:100FC00003F1080202F00F02062AEDB2059102D8E1
:100FD000204686B96DE09A1E0D2A6AD8DFE802F035
:100FE00007070D444848696969696969690D002EF8
:100FF0005FD005992046B0475BE09DF81510F729B2
:10100000F5D8F0291CD1454A1368CBB904F0F00299
:10101000102A02D0302A13D109E0414A138001225C
:1010200004F00F0312FA03F33C4A138008E03C4A31
:101030001380012204F00F0312FA03F3374A53809E
:101040002046FFF7EDFE9DF8143003F00F030F2B41
:101050002FD09DF816102046FFF7E2FE9DF81710DE
:101060002046FFF7DDFE24E09DF81520F72ABED8C4
:10107000043BDBB2EBB19DF8157020463946009376
:10108000FFF7CEFE009B012B0ED09DF81670204678
:101090003946FFF7C5FE009B022B05D09DF817705F
:1010A00020463946FFF7BCFEF72F02D11B4B00212B
:1010B00019601A4B1A683AB319490A88B2F57A7F4F
:1010C00022D9198861B1002251FA02F313F0010309
:1010D00003D10132102AF7D11A461032D0B20DE0F6
:1010E000588858B10B4650FA03F212F0010203D1AE
:1010F0000133102BF7D113463033D8B2FFF796FCEB
:10110000064B00221A6003E0029A002A7FF4FFAE29
:10111000002007B0F0BD00250395CAE73405002084
:101120002A05002010B500F055FF044600F092F8A3
:10113000044B4FF6FF711A8820438A4201D00132D6
:101140001A8010BD2A05002008B5034B1B680BB19F
:10115000984700E0184608BD20050020F0B5134E62
:1011600085B034680746ECB1C1F307638DF80E30E3
:101170000F4BC1F30742C1F30720002401F00F0118
:101180008DF80D208DF80C005A5C254608E003AB65
:10119000595D3846019233689847019A04430135F6
:1011A0009542F4DB204605B0F0BD00BF20050020CD
:1011B000683C0008012817BF024B4FF0FF30187041
:1011C0000020704701000020014B1878704700BFD5
:1011D00029050020012810B5044688BF4FF0FF30D4
:1011E0000BD800F06FFA054BFF221A55044B002272
:1011F00023F8142000F07CFA002010BD44050020E4
:101200006405002010B504464FF0FF30ECB90F4BD9
:10121000FF221C601C715C719C71DC711C81DC60A4
:101220001C745C749C74DC749C82094B20461A709C
:10123000FFF7D0FF0120FFF7CDFF204600F012FF9F
:101240000028B4BF4FF0FF30002010BD480500203B
:101250006005002008B500F035FA124B4FF6FF711B
:101260001A888A4201D001321A800F4B4FF6FF7163
:101270001A898A4201D001321A810A4B4FF6FF7156
:101280005A888A4201D001325A80074B4FF6FF71CB
:101290009A8A8A4201D001329A8200F029FA00200B
:1012A00008BD00BF6405002048050020F7B50128EF
:1012B000C1F3072601F00F03C1F307420446F7B25A
:1012C000C1F3076144D846E026488DF8046030F841
:1012D00014C08DF80520BCF57A7F8DF8061003D96F
:1012E0002046FFF777FF22E0DFF87CC09CF800C0C3
:1012F0004CFA04FC1CF0010F19D0072B17DD0E2B44
:10130000CCBF00230123012D94BF002303F0010370
:101310006BB1164B1B5DBB4206D1013D8DF804201D
:101320008DF80510EDB202E0002320F81430F72FFD
:1013300098BF0E4B204698BF1E5501A92A4601F0C2
:1013400027F8023002289CBF094B53F8200001D92E
:101350004FF0FF30FEBD0748C55C2846002DB3D1D5
:10136000F8E700BF64050020600500204405002068
:10137000E83C0008683C000838B505460C4628469D
:101380002146FFF793FF10F1020FF8D038BD00009F
:101390000128F8B504460E4688BF4FF0FF3000F232
:1013A000D280ABE0C0B210F0800F55D0F72808D93A
:1013B000336843F00F03336000237070B370F37031
:1013C000C2E0C0F30213FB5C28716B71002B3BD1B0
:1013D0005E4900F00F028A5CF0286A7103D1012295
:1013E0006870EA7131E0F72821D1EA791AB1012A4F
:1013F0002A7810D108E02B78052161F303032B70C4
:101400006870AA70EA700CE0062161F303022A708A
:10141000A870EB7005E01346072262F303032B70FC
:10142000E8702B6833600023EB7101330DE062B983
:101430002B78052161F303032B706870AA70EA70A2
:101440002B683360012300E000236A79AA7100222F
:101450002A81002B57D077E02B79F02B17D1EB792D
:101460000133DBB2012BEB7102D0022B04D101E07E
:10147000687048E0A87046E02B78042262F303030A
:10148000E8702B702B6833600023EB715CE0AB7964
:1014900023B96A792B81013AAA7101E0013BAB7152
:1014A0006B79012B03D1013BA870EB7004E0AB79A1
:1014B0000BB1A87000E0E870AB7923BB2B7903F087
:1014C000F002F02A02D01A092B780BE06B791BB1DD
:1014D000012B2B7805D102E02B78052202E00222B5
:1014E00000E0032262F303032B700C236343184ACA
:1014F000D11808794870D358336025E0144B0C2577
:1015000005FB0435134F204600F050FE0028BFF6BF
:1015100049AF00200C235C430D490B199A796AB13D
:101520001A89B2F57A7F09D900220A511A715A71C3
:101530009A71DA711A816FF0090004E000280CBF7B
:101540004FF0FF300020F8BD0120E3E7583C0008D1
:1015500048050020D83C000837B505464FF0FF305D
:10156000002D6FD101AC01217D2001F011FC20463E
:1015700001F036F9482321468DF8073032484EF203
:10158000FF73ADF8043001F0D2F84FF0FF3321467D
:101590002E48ADF8043001F0CAF821462C4801F07D
:1015A000C6F821462B4801F0C2F801F067FB082875
:1015B00008BF2C4633D001F00BFB4FF4803001F014
:1015C00027FB01F033FC0128044628D1102001F04C
:1015D00053F9022001F046F9284601F057FB28464E
:1015E00001F068FB4FF4806001F05AFB4FF40040BB
:1015F00001F070FB4FF480304FF4801101F024FBB8
:10160000204601F02BFB392001F0FAFB0028FAD02C
:10161000022001F029FB01F031FB0828FBD1002159
:101620000D4801F023FC4FF4407001F015FC04203C
:1016300001F028FC094A0A4B012C14BF4FF0FF307F
:1016400000201A603EBD00BF0008014000100140AC
:1016500000140140000C01400000000800FF1F00C2
:10166000042004E0014B1868704700BF002004E02C
:10167000024B188880B28002704700BFE0F7FF1F5E
:10168000024B188880B28002704700BFE2F7FF1F4C
:1016900000230B4A59108A18127813F0010F08BF63
:1016A000120902F00F02092A94BF302137218A184B
:1016B000C2540133182BECD100230376184670472F
:1016C000E8F7FF1F084B1B681BB9EFF31082074BAD
:1016D0001A604FF0010080F31088034B00201A6855
:1016E00001321A60704700BF6C05002068050020B9
:1016F000064A4FF0FF3013683BB1013B13601BB942
:10170000034B1B6883F31088002070476C05002092
:10171000680500200F2988BF4FF0FF3018D80D4B07
:1017200042B2DB685209DB43C3F30223C3F1040373
:101730009940094B0901C318C9B283F8001300F09E
:101740001F00012313FA00F0034B43F8220000208E
:10175000704700BF00ED00E000E100E037B501ADEB
:101760000446284601F03CF810238DF80730032387
:1017700014F0010F8DF8063006D0042306482946E0
:10178000ADF8043000F0D3FF34F001040CBF204664
:101790006FF001003EBD00BF0014014010F0010FCA
:1017A00007D011F0010F064B0CBF4FF4802204222A
:1017B0001A6130F0010018BF6FF00100704700BFE0
:1017C0000014014030B5012185B00446102001F01D
:1017D000EDFA4FF0FF33ADF8083048235C430C4D71
:1017E000013CADF804402846002401A9ADF80A40A8
:1017F000ADF8064001F054F901210A46284601F0EF
:10180000CCF92846012101F0BBF9204605B030BDD6
:10181000001000400348012108B5818401F0D4F98B
:10182000002008BD00100040064810B50121848C3E
:1018300001F0BEF9A4B200280CBF20464FF0FF30E3
:1018400010BD00BF001000401FB504464FF0FF3030
:10185000C4B94FF40060012101F09AFA4FF0FF3350
:10186000ADF808300848472301A9ADF80430ADF8B9
:101870000A40ADF8064001F013F90348012101F0D8
:101880007FF9204604B010BD002C0140044B9A8C17
:1018900092B2998C891A89B28142FAD90020704794
:1018A000002C0140014B04221A6070477005002093
:1018B00070477047022070470220704721B9012805
:1018C0008CBF0220002000E00220704708B5054BC5
:1018D0001B689B7A2BB1012000F0C8FA024B05224D
:1018E0001A6008BDD41600207005002070B5C6B07F
:1018F00051490C22044641A802F08FF93CA84F49F7
:10190000122202F08AF94E4B1B68DB78032B00F29F
:101910008F80DFE803F00E0602604A4901220023AF
:101920002AE040A903310DF1020202234FF0000C1E
:101930000CE009238DF8023004238DF8033069E0B0
:10194000023302F8020C02F801CC9BB211F8010F2D
:101950000232051E18BF0125C72B8CBF002505F0DC
:101960000105002DECD155E0A0F12002D2B25F2A92
:101970008CBF0022012201331F2BCCBF002002F0BC
:1019800001001FFA83FC20B111F8010F0028EBD1F0
:101990000122BCF1000F0CBF002202F001023CA9A1
:1019A00002B1294902236A464FF0000C06E0D054E8
:1019B000581C80B2023302F800C09BB211F8010B30
:1019C000051E18BF0125C72B8CBF002505F001059A
:1019D000002DECD11EE032AD2846FFF759FE00285D
:1019E00026DB013D0DF102020223002005E0023357
:1019F00002F8021C02F8010C9BB215F8011F02321A
:101A00000E1E18BF0126C72B8CBF002606F001064C
:101A1000002EECD103218DF80110204644A98DF849
:101A20000030CDF810D1ADF8143101F049FC00E0E0
:101A3000002046B070BD00BF5C3D0008A33C00081C
:101A4000D4160020DF3F0008E03F000807B5054935
:101A500002466B4603C983E803001046694601F05D
:101A60002FFC0EBD683D000807B5054902466B46D0
:101A700003C983E803001046694601F021FC0EBD4E
:101A8000703D000838B5294B00241B6880259C72E6
:101A90005D72DC72204601F0A7FF20464FF4007112
:101AA00001F0ACFF1021204601F0C0FF402120468C
:101AB00002F044F82946204602F030F8204601F0B2
:101AC000F5FF1B4B20461B6893F82C1002F070F8B2
:101AD000204601F0D9FF0120214601F08FFF0220AE
:101AE000214601F08BFF0120C02102F017F80120F0
:101AF000402102F04FF80120202101F097FF022041
:101B00004FF4807102F01AF84021022002F050F8E0
:101B1000022001F0B9FF204601F02AFE204600F025
:101B2000A5F9044B01221A6038BD00BFD41600206D
:101B3000CC160020700500200D4B10B51C68A4B217
:101B400014F4806F06D04FF6FF321A60094B1B6801
:101B50005B68984714F4007F1EBF054B4FF6FF5299
:101B60001A6014F4004F01D001F05CFE10BD00BFFC
:101B7000445C0040CC16002008B5002001F04DFF69
:101B8000003818BF012008BD73B5044601A800F055
:101B900027FE022C88BF4FF0FF3077D8FFF792FD69
:101BA0003B4B00221A60FFF7A3FD022C13D0394AE9
:101BB000394B1A60394B05221A7001225A70384A83
:101BC000384B1A60384A394B1A60394A394B1A6017
:101BD000394A3A4B5A60304D002000F047F92B68E3
:101BE000022600221E729A729CB9FFF7C5FF80B1CF
:101BF0000120202101F01AFF304601F045FF2B683B
:101C000080225A7201229A72284B1B685B6898479F
:101C10002DE01F4A032313604FF48052ADF80420D7
:101C200001A9102226488DF807208DF8063000F013
:101C30007EFD244B22494FF4805213F1FF334A6159
:101C4000FBD1134A022111601D4A0A2010F1FF3016
:101C50005361FBD10E4B18600433186001F034F867
:101C600001214FF4000001F0A1F8022C06D0164B20
:101C700000221A6002F50442043B1A60134B002450
:101C80001C6014200821FFF745FD20467CBD00BFE5
:101C9000405C004074050020D4160020D8160020B7
:101CA0002C3D0008CC160020F43C0008D016002083
:101CB000E51F000804000020F91F00082000002094
:101CC00000080140400D0300445C00407005002006
:101CD000F0B585B0FFF7F6FC264B1B78002B45D0FE
:101CE000022001F085FFC0F38F05002D3ED0224B6E
:101CF00029B21A8892B2C2F50072914236DA1F4EAA
:101D00001F4C204A40F2FF1C36F8081C36F8047CB1
:101D1000039241EA0747C7F3031010303946019395
:101D2000CDF808C0FFF71AFA039A019BDDF808C046
:101D300080B9218889B242F821702188013189B2A5
:101D40002180218889B2614588BF208019880131AE
:101D500089B21980013DADB229B208360029D3DC21
:101D6000044B00221A70022001F08EFEFFF7C0FC27
:101D700005B0F0BD981500209005002008620040D5
:101D80009C150020980D002010B5FFF79BFC2D4BF3
:101D90001B78002B52D12C4B1A8892B2002A4DD0BE
:101DA0002A4A1278002A49D01A8892B2102A98BF7B
:101DB0001C88244B94BFA4B21024A4B20120A1001B
:101DC000187089B201F0E6FE1F4B21491A8840F2D3
:101DD000FF10121B92B21A80013C1E4BA4B2E318F2
:101DE0004FEAC30C1C4A1D4BB3F800E01FFA8EFEED
:101DF00031F82EE042F808ECB3F800E01FFA8EFE4E
:101E000051F82EE04FEA1E4E42F804ECB3F800E021
:101E10000EF1010E1FFA8EFEA3F800E0B3F800E009
:101E20001FFA8EFE864584BF4FF0000EA3F800E037
:101E300008326245D8D1012001F014FEFFF758FCAA
:101E400010BD00BF940D00209E150020A21500209B
:101E500094050020320C000888610040A015002085
:101E6000002814BF4FF0FF3000207047104A0023B5
:101E7000138011880F4A89B2118011880E4A89B2E5
:101E800011800E4A13700E4A138011880D4A89B2D0
:101E9000118011880C4A89B211800C490C4A10B18A
:101EA0000120087001E00B700123137000207047BF
:101EB000900500209C150020920500209815002018
:101EC0009E150020A4150020A0150020A2150020BA
:101ED000940D002038B5184D04462B784FF0FF3094
:101EE0004BB3164B1B889BB2B3F5FF7F09D9FFF7A5
:101EF0004BFF2B78002B14BF6FF001004FF0FF3029
:101F000019E0FFF7DFFB0E4B0E491A8892B241F839
:101F10002240013292B21A801A8892B2B2F5007F42
:101F200001D300221A80054B1A88013292B21A801E
:101F3000FFF7DEFB002038BDA21500209E15002013
:101F4000A41500209405002070B506460A4C42F204
:101F50000F7504E02388AB420CD801332380304650
:101F6000FFF7B8FF10F1020FF4D0002802DB024B9C
:101F700000221A8070BD00BF9A150020124B10B5C8
:101F80001B8804469BB24FF0FF30E3B1FFF79AFB8A
:101F90000E4B0F4A198889B252F8212022601A8804
:101FA000013292B21A801A8892B2B2F5007F01D340
:101FB00000221A80044C2388013B9BB22380FFF748
:101FC00097FB208880B210BD90050020920500206C
:101FD000980D002008B5FFF77BFEFFF7D5FE002027
:101FE00008BD000008B5034B00221A70FFF7CCFEB5
:101FF00008BD00BF940D002008B5034B01221A70E4
:10200000FFF766FE08BD00BF9815002030B5012817
:10201000044685B00D4688BF4FF0FF301AD84FF008
:10202000000304A9ADF80430ADF80630ADF808306F
:10203000ADF80C3041F8105D4FF00C0314BF0648AA
:1020400006486946ADF80A3000F0A6FC044B0020B3
:1020500043F8245005B030BD00380140004800402E
:10206000BC16002073B504464FF0FF30002C40F042
:10207000868001AD0121424800F0BAFB284600F0FD
:10208000AFFB022329468DF806301C264FF400735F
:102090003C48ADF804308DF8076000F048FB4FF481
:1020A000806329463848ADF804308DF8076000F0A9
:1020B0003EFB482329468DF8073032484FF48063B1
:1020C000ADF8043000F033FB4FF4006329462E488E
:1020D000ADF8043000F02BFB4FF48040012100F0FC
:1020E00057FE4FF4C020012100F060FE47F6122198
:1020F0002046FFF78BFF47F612210120FFF786FFEE
:1021000004212520FFF706FB0122204840F225513B
:1021100000F0ABFC04212720FFF7FCFA1C4840F23A
:102120002551012200F0A1FC1A481B4904700378D4
:10213000DFF868E00B700B78194A8EF800301470E5
:1021400092F800C0174B83F800C01D78DFF858C024
:102150008CF8005044704078487049780B488EF8ED
:1021600001105470527801215A705B788CF801305C
:1021700000F06EFC0648012100F06AFC20467CBDA0
:102180001000140000080140001001400038014018
:1021900000480040AC150020B4160020B015002007
:1021A000B8160020C4160020A8150020012838B554
:1021B000044688BF4FF0FF301DD80F4B6FF0010071
:1021C0001B5DC3B1FFF77EFA0C4B0D491A5D02EBA4
:1021D00084128D5C1A5D0132D2B21A551A5D3F2A03
:1021E00001D900221A55044B1A5D013AD2B21A5590
:1021F000FFF77EFA284638BDAC150020B015002048
:1022000034160020012838B504460D4688BF4FF02B
:10221000FF301FD8104B1B5D3F2B88BF6FF00100B4
:1022200018D8FFF74FFA0D4B0D491A5D02EB8412D7
:102230008D541A5D0132D2B21A551A5D3F2A01D966
:1022400000221A55044B1A5D0132D2B21A55FFF71B
:102250004FFA002038BD00BFAC150020B416002096
:1022600034160020012838B5044688BF4FF0FF30EF
:102270001DD80F4B6FF001001B5DC3B1FFF722FAB1
:102280000C4B0D491A5D02EB84128D5C1A5D013214
:10229000D2B21A551A5D3F2A01D900221A55044BB1
:1022A0001A5D013AD2B21A55FFF722FA284638BD14
:1022B000B8160020A8150020B4150020F0B501289C
:1022C000044687B00D46174688BF4FF0FF3052D8FE
:1022D0002A4E335DD3183F2BC8BF6FF001004ADC94
:1022E000FFF7F0F90022264B2648274901973CE0EA
:1022F00013F804C015F8017BDFF890E00CEB841CA8
:102300000EF80C7013F804C00CF1010C5FFA8CFC91
:1023100003F804C013F804C0BCF13F0F84BF4FF0B2
:10232000000C03F804C016F804C00CF1010C5FFAAD
:102330008CFC06F804C016F804C0BCF1010F12D1E1
:10234000012C15BFB1F80CC0B0F80CC01FFA8CFC02
:102350001FFA8CFC15BF4CF0800C4CF0800CA1F8DF
:102360000CC0A0F80CC0013292B2019FBA42BFD398
:10237000FFF7BEF9002007B0F0BD00BFB81600207F
:10238000C41600200048004000380140B415002069
:1023900070B505460C461646284621463246FFF7DC
:1023A0008DFF10F1020FF7D070BD0000144B10B577
:1023B0001A8812F0200F09D09C882020E4B2214610
:1023C000FEF7C2FE10B92146FFF71CFF0C4C238814
:1023D00013F0800F13D00B4B1B7853B10020FFF785
:1023E00041FF0028A4BF80B2A08008DAFF23A380A9
:1023F00005E0A38923F080031B041B0CA38110BDFF
:1024000000380140B8160020154B10B51A8812F09C
:10241000200F0AD09C882120E4B22146FEF794FECA
:1024200018B901302146FFF7EDFE0D4C238813F05B
:10243000800F13D00B4B5B7853B10120FFF712FFD5
:102440000028A4BF80B2A08008DAFF23A38005E0A3
:10245000A38923F080031B041B0CA38110BD00BFC4
:1024600000480040B81600200E4B10B51A8812F034
:10247000200F0AD09C882220E4B22146FEF764FE99
:1024800018B902302146FFF7BDFE064A138813F043
:10249000800F05D0938923F080031B041B0C9381CC
:1024A00010BD00BF00440040002A30B5C8BF4FF047
:1024B000000C044602DC12E00CF1010C11F80C00D7
:1024C0000028F9D19445B4BFCCEB0202024613F0C8
:1024D000020F0CBF4FF0200C4FF0300C01E04FF01A
:1024E000200C13F001000CD108E02CB1236883F814
:1024F00000C02368013323600130013A002AF4DC74
:1025000008E0002006E024B125682B702368013321
:102510002360013011F8013B002BF4D108E02CB10D
:10252000236883F800C02368013323600130013A37
:10253000002AF4DC30BD7FB594461C46089A099BFE
:102540000D4649B94FF0300C8DF8051001A98DF8F2
:1025500004C0FFF7A9FF46E0BCF10A0F14BF002139
:102560000121002C0CBF002401F001042CB1002D2E
:1025700002DA6D42012400E000240A9E0DF1100EE3
:1025800000210EF8011D3A3E0BE0B5FBFCF10CFBFF
:1025900011510929C8BF891930310EF8011DB5FB49
:1025A000FCF57146002DF0D1D4B192B113F0020FB9
:1025B0000FD058B1D0F800C04FF02D0E8CF800E0CD
:1025C000D0F800C00CF1010CC0F800C0013A0124A1
:1025D00006E04FF02D0C0EF1FF310EF801CC002477
:1025E000FFF762FF001904B070BD0000F0B589B0BC
:1025F00005460E46059200247DE0252B72D116F883
:10260000013F002B7BD0252B6CD02D2B02D1013626
:10261000012303E0002301E043F00203374616F8EC
:10262000012B302AF8D0002202E00A2000FB02C26F
:1026300039783E46A1F1300C5FFA8CF00137092859
:10264000F3D9732909D10599081D059009682F4808
:10265000002908BF0146284641E064290ED10599AA
:102660000193612300920293081D096805900A22D4
:1026700028460123FFF75FFF24183BE0782906D1A5
:1026800005990193081D05900092612307E05829E0
:102690000AD105990193081D0590009241230293E8
:1026A0002846096810220BE075290BD10599019382
:1026B000612300920293081D096805900A222846AA
:1026C0000023D7E7632915D10599081D09680590EE
:1026D0008DF81C1000218DF81D10284607A9FFF762
:1026E000E3FEC9E7327825B12B681A702B680133F5
:1026F0002B60013401363378002B7FF47EAF15B1A7
:102700002B6800221A70204609B0F0BDE03D000899
:102710000EB40FB505AA52F8041B019001A803924C
:10272000FFF764FF04B05DF804EB03B07047CB78AB
:10273000F7B513F0100F03F00F020F881CBF8B7852
:102740001A4317F0FF0F22D0D0F800C000230197E2
:10275000012414FA03F5019E05EA0604AC4211D1E6
:102760009E000F2717FA06F512FA06F62CEA050C5A
:10277000CD784CEA060C282D08BF446102D0482DC4
:1027800008BF04610133082BE2D1C0F800C00F88F4
:10279000FF2F24D9D0F804C000230192012203F1B5
:1027A000080512FA05F505EA0704AC4212D19E00AD
:1027B0000E3212FA06F5019A2CEA050C12FA06F608
:1027C000CD784CEA060C282D08BF446102D0482D74
:1027D00008BF04610133082BE0D1C0F804C0FEBD7E
:1027E0004FF0FF33038002238370DB18C370704700
:1027F0000028B4BF1A4B1A4B00F4401CB4BFDB696D
:102800005B68BCF5401F10B582B20AD1DFF850C03A
:1028100023F07063DCF8044024F07064CCF80440CA
:1028200012E010F4801F02BF4FEA505C4FEA0C1C0C
:1028300002FA0CFC04D0C0F3034C032404FA0CFC91
:1028400023EA0C0343F0706319B1410D09018A407A
:1028500013430028B5BF024A014AD361536010BD3B
:1028600000000140034B1A6802F038021043186060
:10287000704700BF00200240044B1A6822F010028B
:102880001A601A6810431860704700BF00200240A9
:10289000034B044A5A6002F188325A60704700BF05
:1028A0000020024023016745024B1A6942F0800272
:1028B0001A61704700200240014BD860704700BF8A
:1028C00000200240094BDA6812F0010F0AD1DA68E1
:1028D00012F0040F08D1DB6813F0100F0CBF0420B6
:1028E000032002E0012000E00220704700200240A7
:1028F00010B50446FFF7E6FF00E0013C012814BFD5
:1029000000230123002C0CBF002303F00103002B44
:10291000F3D1002C08BF052010BD000070B504469F
:102920004FF400500E46FFF7E3FF042810D1094D85
:102930004FF400502B6943F001032B612680FFF711
:10294000D7FF05281FBF2A6941F6FE7313402B618C
:1029500070BD00BF0020024038B505464FF430205E
:10296000FFF7C6FF042814D10A4C4FF43020236926
:1029700043F0020323616561236943F0400323614F
:10298000FFF7B6FF05281FBF226941F6FD7313400C
:10299000236138BD00200240038ACA8823F44053D3
:1029A0001B041B0C134330B503820D468389098930
:1029B000AA8823F4B05341EA0202698923F00C0388
:1029C0000A431B041B0C92B242EA03038381838AED
:1029D000AA8923F440731B041B0C134387B00446DD
:1029E000838201A800F080F9184BA2899C4212B2A0
:1029F0000CBF049B039B002A2A6803DA1921594360
:102A0000520002E01921594392006423B1FBF2F114
:102A1000B1FBF3F21201100903FB1011A08900B2FF
:102A2000002806DAC9003231B1FBF3F303F00703E3
:102A300005E009013231B1FBF3F303F00F0343EA80
:102A4000020292B2228107B030BD00BF00380140BF
:102A500021B183899BB243F4005304E0838923F4BA
:102A600000531B041B0C83817047C1F342134FF0CA
:102A7000010C01F01F0163450CFA01F101D10C308A
:102A800004E0022B01D1103000E014301AB10368C9
:102A900043EA010102E0036823EA01010160704793
:102AA0002D4ADFF8B8C00388904214BF00220122EB
:102AB000604508BF42F0010210B59BB2CAB9284C6C
:102AC000B0F1804F14BF4FF0000C4FF0010CA0424A
:102AD00014BF64464CF001045CB9224CDFF888C096
:102AE000A04214BF00240124604508BF44F0010443
:102AF0002CB1B1F802C023F0700343EA0C031B4C65
:102B0000DFF86CC0041B18BF012460450CBF002413
:102B100004F0010434B123F44073B1F806C09BB251
:102B200043EA0C0303808B8883850B8803856AB98D
:102B3000104B114A984214BF00230123904208BF52
:102B400043F0010313B90D4B984201D10B7A038670
:102B50000123838210BD00BF002C014000340140DE
:102B60000004004000080040000C0040001000403D
:102B70000014004000400140004401400048014072
:102B800021B103889BB243F0010304E0038823F0E2
:102B900001031B041B0C038070471AB183899BB28D
:102BA000194303E083899BB223EA010181817047C5
:102BB000038A828911420CBF0020012019420CBFF8
:102BC000002000F001007047C94389B201827047BC
:102BD0000D4B1A6842F001021A6059680B4A01EA6B
:102BE00002025A601A6822F0847222F480321A605B
:102BF0001A6822F480221A605A6822F4FE025A608F
:102C00004FF41F029A607047001002400000FFF866
:102C10000C4BB0F5803F1A6822F480321A601A68B3
:102C200022F480221A6003D0B0F5802F08D103E08F
:102C30001A6842F4803202E01A6842F4A0221A6054
:102C4000704700BF00100240034B5A6822F47C1208
:102C5000104308435860704700100240014B186051
:102C6000704700BF60004242034B5A6822F00302E3
:102C700010435860704700BF00100240024B586874
:102C800000F00C00704700BF00100240034B5A6870
:102C900022F0F00210435860704700BF001002405D
:102CA000034B5A6822F4E06210435860704700BF3B
:102CB00000100240034B5A6822F4605242EAC000FE
:102CC0005860704700100240014B1860704700BF09
:102CD000D8004242034B5A6822F4404210435860E5
:102CE000704700BF00100240224B5A6802F00C02ED
:102CF000042A02D0082A15D101E01F4B13E05A68BC
:102D00005968C2F38342023211F4803F08BF1B4B63
:102D100005D05B6813F4003F14BF194B164B5A43A0
:102D2000026001E0174B0360124B17495A68D0F854
:102D300000C0C2F303128A5C2CFA02F24260D3F89C
:102D400004C0CCF3022C11F80CC022FA0CFCC0F821
:102D500008C0D3F804C0CCF3C22C11F80C10CA4040
:102D6000C2605B680949C3F38133CB5CB2FBF3F209
:102D70000261704700100240001BB70000093D00CF
:102D8000808D5B0000127A00400000203C00002093
:102D900019B1054B9A69104303E0034B9A6922EA83
:102DA00000009861704700BF0010024019B1054B48
:102DB000DA69104303E0034BDA6922EA0000D861C4
:102DC000704700BF0010024019B1054BDA6810438C
:102DD00003E0034BDA6822EA0000D860704700BFC6
:102DE0000010024019B1054B1A69104303E0034B70
:102DF0001A6922EA00001861704700BF0010024003
:102E00004309012B04BF084B1B6805D0022B0BBFE5
:102E1000054B054B1B6A5B6A00F01F0033FA00F09C
:102E200000F00100704700BF0010024007B500230A
:102E300001933120FFF7E4FF019B01330193019BD4
:102E4000B3F5A06F01D00028F3D03120FFF7D8FFF1
:102E5000003818BF01200EBD40F0BE60024B40F4A8
:102E60002020D860704700BF00ED00E021F06041F5
:102E700021F07F01024B41EA00009860704700BFDB
:102E800000ED00E004280BBF054B054B1A681A68DB
:102E90000CBF42F0040222F004021A60704700BF27
:102EA00010E000E010B5064C18B9236801221A8220
:102EB00005E0044B1B681B68984720680A3010BD6A
:102EC000D4160020D016002010B5064C18B923687F
:102ED00001221A8205E0044B1B689B689847206812
:102EE0000C3010BDD4160020D016002008B5274B9A
:102EF00018B91B6802221A8247E0254800221B6885
:102F000002801A7812F07F0215D15B7A027813F0F2
:102F1000200F14BF42F0020222F0020213F0400F11
:102F20001B4B027015BF1A781A7842F0010222F08A
:102F300001021A7022E0012A27D0022A24D15A79EC
:102F400002F00F0312F0800F4FEA830308D003F161
:102F5000804303F5B8431B6803F03003102B08E0EF
:102F600003F1804303F5B8431B6803F44053B3F502
:102F7000805F02BF037843F001030370054B1B68B9
:102F80001B699847024800E0002008BDD4160020C5
:102F9000DC160020D0160020F7B5274B1C68238ACA
:102FA000267AD3F1010238BF0022042E14BF002676
:102FB00002F00106AEB12149214A0B78012B0CD158
:102FC000204B04271868204B80B2C3185B000020F8
:102FD00018603023138008702AE01023138007271D
:102FE00026E0A58AAB428CBF022704279D4228BF5A
:102FF0001D462846A369984703463046019300F0D2
:10300000ADFD019B2A460146184600F0C7FC294643
:10301000304600F0BFFD238A30225B1B2382638A87
:10302000ED18074B65821A80084B4FF440521A8006
:10303000014B1B681F72FEBDD4160020C81600206D
:10304000E0160020505C004002300020DE16002018
:1030500010B50A4B0A491B684978DA7891420AD3BD
:10306000997841B99C8834B99A72064B1B685B68A1
:103070009847204600E0022010BD00BFD416002073
:10308000D8160020D016002038B50E4A0E4C126813
:1030900023685879D9789369984723689A7A7AB1DE
:1030A00070B91A7962B99D7855B9084B1B68DB680D
:1030B0009847236828465A79DA72DA781A7300E05A
:1030C000022038BDCC160020D4160020D0160020D7
:1030D00010B53F4B1B68187810F07F0002BF5A7A7A
:1030E00022F020025A7272D002286FD15A88002A28
:1030F0006DD11A79002A6AD15A79DFF8D8C022F046
:10310000800012F0800F4FEA800415BF04F1804464
:1031100004F1804404F5B84404F5B84414BF2168B0
:1031200021689CF800C014BF01F0300101F4405147
:10313000604534BF4FF0000C4FF0010C002914BF64
:1031400061464CF00101002940D19B7A002B3DD013
:1031500012F0800F4FEA800411D004F1804404F58E
:10316000B844236803F03003102B29D1C4B22046A1
:1031700000F0C0FC2046302100F058FC20E004F1B3
:10318000804404F5B844236803F44053B3F5805FEA
:1031900016D130B9104B1B6893F82C1000F008FDC5
:1031A00002E0C0B200F092FC22684BF68F7302EA94
:1031B000030383F4405343F4004343F0800323604C
:1031C000064B1B685B699847002000E0022010BD99
:1031D000D4160020D8160020CC160020D0160020CF
:1031E00008B52B4BDFF8ACC018689CF800C04179DB
:1031F00021F0800211F0800F4FEA820315BF03F126
:10320000804303F1804303F5B84303F5B84315BF8A
:103210001B681B6803F0300303F44053624535D24A
:10322000B0F802C0BCF1000C18BF4FF0010C002B2D
:1032300014BF63464CF0010343BB837A33B311F0F0
:10324000800F4FEA82030BD003F1804303F5B843AC
:10325000196848F6BF7201EA020282F010020AE021
:1032600003F1804303F5B84319684BF68F7201EA06
:10327000020282F4805242F4004242F080021A605C
:10328000054B1B689B699847002000E0022008BDA1
:10329000D4160020D8160020D016002008B5064B02
:1032A0001B685A7A42F020025A72044B1B68DB6991
:1032B0009847002008BD00BFD4160020D01600207B
:1032C000054B1A68538A18B98988CB1A138201E012
:1032D0000868C018704700BFD416002070B580245D
:1032E000A2B0064608496846224600F096FC3046E1
:1032F0000DEB04016D46CDF880D0ADF88440FFF7AA
:10330000DFFF22B070BD00BFE83D000808B50C4BE0
:1033100000201B6893F82C1000F04AFC094B1B6836
:10332000187A082806D1084B4FF480521A80074BB0
:1033300010221A80092814BF0020012008BD00BFF8
:10334000CC160020D4160020DE160020E016002047
:10335000F8B5384B1C68237A022B14BF00260126CF
:10336000042B08BF46F00106002E5BD1032B14BFCF
:1033700000220122052B08BF42F00102002A4BD097
:10338000A369228A191E18BF0121002A0CBF00213F
:1033900001F00101A1B1A58A954228BF1546284632
:1033A0009847238A07465B1B2382638A3046EB18C3
:1033B000638200F0E1FB2A460146384600F004FB38
:1033C000238A53B11C4B4FF4405200201A8001460F
:1033D00000F0E0FB194B30221A80238AA28A9A421D
:1033E00003D8144B03221B6803E0124A1BB1136875
:1033F00005221A720CE0126806211172104A116837
:10340000104A89B28A18520013600C4B30221A807D
:10341000084B1B681B7A06E0072B03D10A4B1B687D
:10342000DB6898470823034A12681372FFF76EFFA0
:10343000F8BD00BFD4160020DE160020E0160020E4
:10344000505C004002300020CC160020BB4BF7B58A
:103450001A68BB4EBB4B92B2D31835685B001F682D
:103460002B7A092B1AD0BFB207F1005707F5405746
:103470007F003C4614F8013B2B707B780A376B7059
:10348000B4F8030000F0C4FB6880B4F807003568A6
:1034900000F0BEFBA88033687F88DF80A84C012243
:1034A00023681A72DA885D78002A61D11A7812F0DE
:1034B0007F022ED1092D02D1FFF7CAFD3BE0052D79
:1034C0000DD193F90320002A4DDB9A78002A4AD1C6
:1034D0009A88002A47D19B7A002B35D043E0032DF0
:1034E0000BD1DA78012A27D19A882ABB5B7A13F0AC
:1034F000200F21D0FFF7D2FE1DE0012D1CD1DA787C
:10350000012A19D19A88BAB95B7A13F0200F13D027
:103510000AE0012A04D10B2D0ED1FFF7B5FD0AE018
:10352000022A09D1012D02D1FFF7D2FD03E0032DBC
:1035300002D1FFF755FE38B1834B28461B685B6903
:10354000984703280DD070B97C4B30211A687F4B07
:1035500092B2D3185B0000221A607D4B19800623BB
:1035600002E0092300E00823754A12681372E1E0C3
:10357000062D18D11A7812F07F0F40F095809B78B5
:10358000012B03D1704B1B68DB6984E0022B03D154
:103590006D4B1B681B6A7EE0032B40F085806A4BF5
:1035A0001B685B6A77E0002D48D1598800297BD1E0
:1035B0005A6822F47F42B2F5003F75D11A7812F0B2
:1035C0007F0203D19B88002B63D06DE0012A09D1D3
:1035D0005D4A5879126893699847002864D1236836
:1035E0009B7A28E0022A5FD15B795A4803F00F02E8
:1035F00013F0800F03F070014FEA820315BF03F14F
:10360000804303F1804303F5B84303F5B84314BF87
:103610001B681B68007814BF03F0300303F44053A9
:1036200082422CBF00220122002914BF002202F096
:103630000102002A38D0002B2BD135E0082D06D10D
:103640001B7813F07F0F08BF434B25D02CE00A2DC9
:1036500016D11A7802F07F02012A25D19A7A1AB37C
:10366000598809BB5A6822F47F42B2F5803F1BD1CA
:10367000354A5879126893699847384B60B113E01E
:10368000552D11D15B887BB9802A08BF344B0BD1F3
:1036900002E0344B00E03BB122680021518293618B
:1036A0000020984700200AE0274B22681B685078CA
:1036B0001B699847032804BF214B1B6806D0204B89
:1036C0004FF6FF711B681A8A8A4201D1092203E072
:1036D000022800D012B908221A722BE093F90010C8
:1036E000002921DAD98801910198824284BF019A88
:1036F0001A8211D88A420FD21349096891F82C1006
:103700008A4201D2002105E092FBF1F001FB102278
:1037100012B90121144A11700B4A126892F82C2038
:103720009A82FFF739FC05E003221A720F4B4FF41F
:1037300040521A80FFF7EAFDFEBD00BF505C00401A
:10374000D416002004300020CC16002002300020C7
:10375000E0160020D8160020A52E0008C92E00086B
:10376000DD320008ED2E0008C8160020DE1600200D
:1037700030B50F4B93F800C0002312E0DAB291008D
:1037800001F1804101F5B8410D6842F4004242F078
:10379000800440F60F7205EA020244EA02020A605F
:1037A00001336345EAD3034B40F08000186030BD1D
:1037B000D81600204C5C004010B5164C23681A7ACD
:1037C000022A14BF00210121042A08BF41F001018F
:1037D00021B1FFF7E1FB23681B7A14E0062A11D11F
:1037E0005A78052A0AD11A7812F07F0F06D1D878B4
:1037F000FFF7BEFF084B1B681B6A9847074B1B6807
:103800009B6898470823034A12681372FFF77EFDEE
:1038100010BD00BFD4160020D0160020CC1600200A
:1038200070470000F7B50022ADF80620544F554E02
:103830009DE013F00F0571D13A6813F0100F92B2AA
:1038400032803188504A01F03001118032884C4C6E
:1038500002F44052328039684BF6BF7201EA02022C
:1038600082F4005282F0200242F4004242F08002D0
:10387000444D3A6008D1226848F60F7302EA030308
:103880002360FFF799FF1EE03B689BB2ADF806305E
:10389000BDF8063013F4006F08D0226840F68F732D
:1038A00002EA03032360FFF7D1FD0CE0BDF8063008
:1038B0001BB2002B5BDA226840F68F7302EA030327
:1038C0002360FFF745FD22684BF6BF7302EA03034E
:1038D0002A8802F4805292B20AB183F48053294AB2
:1038E000128802F4005292B20AB183F40053264ABD
:1038F000128802F0100292B20AB183F01003224A39
:10390000128802F0200292B20AB183F020031F4A0B
:1039100043EA02021A4B92B21A602FE0AC0004F1A3
:10392000804404F5B84423689BB2ADF80630BDF876
:1039300006301BB2002B0ADA226840F68F7302EAC7
:103940000303134A23606B1E52F823309847BDF8D7
:10395000063013F0800F0AD0226848F60F7302EA8F
:1039600003030C4A013D236052F8253098470A4A68
:1039700013689BB213F4004F7FF45BAFFEBD00BF32
:10398000005C0040DE160020E01600208080FFFF73
:103990002000002004000020445C004001F10051A0
:1039A000013201F540514900520808E010F801CCFD
:1039B00010F8023C013A43EA0C2321F8043C02309F
:1039C0000431002AF2D1704701F10051013201F5B2
:1039D00040514900520804E051F8043B013A20F8F4
:1039E000023B002AF8D170474FF6F873024A00EA0A
:1039F00003031360704700BF505C0040800000F17B
:103A0000804000F5B840036823F4EC4323F07003D2
:103A100043EA010189B201607047800000F18040F3
:103A200000F5B840006800F4C0607047800000F105
:103A3000804000F5B840026848F6BF7302EA03030D
:103A400001F0100292B20AB183F0100301F02001DC
:103A500089B209B183F0200343F4004343F08003AB
:103A600003607047800000F1804000F5B8400268B4
:103A700048F6BF7302EA030383F0300343F40043C4
:103A800043F0800303607047800000F1804000F540
:103A9000B84002684BF68F7302EA030383F4405385
:103AA00043F4004343F0800303607047800000F15B
:103AB000804000F5B840026840F60F6302EA030355
:103AC00043F4004343F0800303607047800000F13B
:103AD000804000F5B840036813F4804F09D00268B5
:103AE00040F60F7302EA030343F4404343F08003BC
:103AF00003607047800000F1804000F5B840036823
:103B000013F0400F09D0026840F60F7302EA030376
:103B100043F4004343F0C00303607047064B490879
:103B20001B6849009BB203EBC00000F1005000F598
:103B30004050400001607047505C0040054B490810
:103B40001B6849009BB203EBC000034BC3185B002A
:103B500019607047505C004004300020054B1B6822
:103B60009BB203EBC00303F1005303F540535B002A
:103B700018887047505C0040044B1B689BB203EBF5
:103B8000C000034BC3185B0018887047505C0040AE
:103B900004300020044B1B689BB203EBC000034BB6
:103BA000C3185B0019607047505C00400230002071
:103BB0000D4B1A680D4B92B2D31803EBC0004000B6
:103BC0003E2909D94B0911F01F0F01D1013B9BB2CE
:103BD0009B0243F4004305E04B0811F0010F18BFAE
:103BE00001339B0203607047505C004006300020A8
:103BF000054B1B689BB203EBC000044BC3185B0072
:103C000018688005800D7047505C00400630002029
:103C1000C3B2000A40EA03207047002305E011F810
:103C200003C0013A00F803C00133002AF7D17047FE
:103C3000000801401000000000100140008000005A
:103C4000000C0140001000000010014000200000A6
:103C500000100140004000000101020100000000CE
:103C60000000000000000000000002030301020346
:103C700003030303020203014D494F533332004D46
:103C80004248505F434F52455F53544D33320053C7
:103C9000544D3332463130780025303878003F00BB
:103CA0002564004D494F53333220426F6F746C6F5F
:103CB0006164657200286329203230313220542E2D
:103CC000204B6C6F73650020253032580020202077
:103CD00000253038582000000202020201010200D3
:103CE000F000007E32000000FEFFFFFFFFFFFFFF3D
:103CF0000000000021380008CD1800082138000815
:103D0000213800082138000821380008213800082F
:103D100021380008A5180008120100020000004028
:103D2000C016FE0310100102030100000000000095
:103D3000851A0008B1180008B3180008B518000863
:103D4000B9180008BD180008691A00084D1A0008C3
:103D5000ED18000800000000400000006D69646973
:103D6000626F782E6F726700783D00086500000072
:103D7000183D0008120000000902650002010080E1
:103D800032090400000001010002092401000109B8
:103D900000010109040100020103000207240100DF
:103DA000014100062402010100062402020200096A
:103DB000240301030102010009240302040101019B
:103DC000000905020240000000000525010101096B
:103DD00005810240000000000525010103000000EC
:103DE000286E756C6C290000D10FED54CFC5FBB85F
:103DF0009752389138910E7D0FED389301910E91C5
:103E000000C11F020E91F7041040006E106EE76AA9
:103E100000000000000000000000000000000000A2
:103E2000000000000000040000000000000000008E
:103E3000000000002F55461F00D84840376AF76A37
:103E400000300000C7062E734A2C137BE97F320036
:103E50002A280D9BFE0B21EF422A2F73B5B8DA7684
:103E6000E679BF0FEB793E0B1010000021380008F7
:103E700021380008213800082138000821380008BE
:103E800021380008213800082138000821380008AE
:103E9000213800082138000821380008213800089E
:103EA0002138000802040608000000000102030493
:103EB0000102030406070809FFFFFFFFFFFFFFFFE2
:103EC000FFFFFFFFFFFFFFFFFFFFFFFFFFFFFFFF02
:103ED000FFFFFFFFFFFFFFFFFFFFFFFFFFFFFFFFF2
:103EE000FFFFFFFFFFFFFFFFFFFFFFFFFFFFFFFFE2
:103EF000FFFFFFFFFFFFFFFFFFFFFFFFFFFFFFFFD2
:103F0000FFFFFFFFFFFFFFFFFFFFFFFFFFFFFFFFC1
:103F1000FFFFFFFFFFFFFFFFFFFFFFFFFFFFFFFFB1
:103F2000FFFFFFFFFFFFFFFFFFFFFFFFFFFFFFFFA1
:103F3000FFFFFFFFFFFFFFFFFFFFFFFFFFFFFFFF91
:103F4000FFFFFFFFFFFFFFFFFFFFFFFFFFFFFFFF81
:103F5000FFFFFFFFFFFFFFFFFFFFFFFFFFFFFFFF71
:103F6000FFFFFFFFFFFFFFFFFFFFFFFFFFFFFFFF61
:103F7000FFFFFFFFFFFFFFFFFFFFFFFFFFFFFFFF51
:103F8000FFFFFFFFFFFFFFFFFFFFFFFFFFFFFFFF41
:103F9000FFFFFFFFFFFFFFFFFFFFFFFFFFFFFFFF31
:103FA000FFFFFFFFFFFFFFFFFFFFFFFFFFFFFFFF21
:103FB000FFFFFFFFFFFFFFFFFFFFFFFFFFFFFFFF11
:103FC000FFFFFFFFFFFFFFFFFFFFFFFFFFFFFFFF01
:103FD000FFFFFFFFFFFFFFFFFFFFFFFFFFFFFFFFF1
:103FE000FFFFFFFFFFFFFFFFFFFFFFFFFFFFFFFFE1
:103FF000FFFFFFFFFFFFFFFFFFFFFFFFFFFFFFFFD1
:10400000000001205D580008A7580008CD4D0008A9
:10401000A7580008A7580008A7580008000000008B
:10402000000000000000000000000000155500081E
:10403000A75800080000000089550008C555000871
:10404000A7580008A7580008A7580008A758000854
:10405000A7580008A7580008A7580008A758000844
:10406000A7580008A7580008A7580008A758000834
:10407000057D0008A75800081D7D0008917E0008F6
:10408000A7580008A7580008A7580008A758000814
:1040900061870008A7580008A7580008A75800081B
:1040A000A7580008A7580008A7580008A7580008F4
:1040B0007D830008A1830008A7580008A7580008BE
:1040C000A7580008B99000087D920008A75800087A
:1040D000A7580008BD8F00087990000819900008C3
:1040E000A7580008A7580008A7580008A7580008B4
:1040F000A7580008A7580008A7580008A7580008A4
:10410000A7580008A7580008C5830008A75800084A
:10411000A7580008A7580008A7580008A758000883
:10412000A7580008A7580008A7580008A758000873
:10413000A758000800000000000000000000000078
:10414000000000000000000000000000000000006F
:10415000000000000000000000000000000000005F
:10416000000000000000000000000000000000004F
:10417000000000000000000000000000000000003F
:10418000000000000000000000000000000000002F
:10419000000000000000000000000000000000001F
:1041A000000000000000000000000000000000000F
:1041B00000000000000000000000000000000000FF
:1041C00000000000000000000000000000000000EF
:1041D00000000000000000000000000000000000DF
:0441E0005FF8E0F1B3
:1041E400F7B500F0B5FF019001A8012101F0C6F870
:1041F4003F4B40491F78404B00221E880846134617
:104204003E4D21E0072B23D830F902EBBEF1000F1D
:1042140019DA3B4C04F803C015F902C0394C0CFB05
:1042240006FC24F813C00133BEF1FF3F02BFDFF8E0
:10423400D8C00EF1010E4FF6FE74DBB204BF4CF889
:1042440022E020F8024C01325FFA82FCBC45D9D34B
:104254002E4A1278D2F1010238BF0022072B98BFF0
:1042640042F00102002A3FD0214A24481678224A0B
:104274001588002234E0072B36D831F802EB0FFA08
:104284008EF7002F2BDD1E4F1E4C07F803C010F8CD
:1042940002C00EF1FF3E4FFA8CF76F431FFA8EFEF9
:1042A40024F8137001331EF0070F08BF184F21F8CC
:1042B40002EC08BF17F802E0DBB204BFCEEB0C0C33
:1042C40000F802C010F902C0BCF1000FDFBF4FF0CC
:1042D400000C4FF0000E00F802C021F802EC01328D
:1042E4005FFA82FCB445C6D30A4A13707CE700BF68
:1042F40074560020484B002002000020F43A0020AD
:10430400CC4C0020343B0020CC4B0020D44C00206B
:10431400B4390020C84B0020F8B5134F05460E46AB
:1043240007EB4517114801F01DFF3146384608F0E8
:1043340073FB0446384608F0EBFB002C04DA2146F4
:104344000B4801F00FFF0CE00A4B002243F8252034
:10435400BB68094A094842F825302946324601F02B
:1043640001FF2046F8BD00BF4843002080CE00086E
:1043740090CE0008CC4B0020F4390020B7CE0008C2
:10438400F7B5144B054653F822600C46760A01969D
:10439400009208F02DFB019B0746B3FBF0F61F2E9D
:1043A400009A88BF4FF0FF3012D80B4B06EB421235
:1043B40053F8220008F022FB019B294607FB16361E
:1043C400801902F0A7FC0028ACBF20466FF0010062
:1043D400FEBD00BFCC4B002070110020F7B54A4B46
:1043E40003F5806200280CBF1E461646474B1B7817
:1043F40033B91A46F2500433B3F5806FFAD182E030
:1044040004F018F80120014603F088FD404A1378AF
:104414001A46002B6ED000243E4D3F4F3FE03F4AEA
:104424004FF4007102EB44202A5DFFF7A9FF002836
:1044340006DA2B5D002227F81320394B23F81420C9
:104444002B5D384951F8232002F5007241F82320EE
:10445400354951F823108A4202D3002227F8132049
:1044640003F0F2FF2D2804F1010417D9284D0A2284
:104474002B78B0FBF2F102FB110200932B48234688
:1044840001F070FE2C70224B294A93F800E0234C73
:10449400012302EB4E0E47F6FF7C27E0E4B21C4AF0
:1044A4001378A342BBD8EEE70F7811F8015C01F54D
:1044B400007105EB072530F9027F2DB207FB0522B9
:1044C4007045F1D1D2136245C8BF47F6FF7203DCD1
:1044D40018498A42B8BF0A46120442EA124246F810
:1044E400042B023340F20122934208D01048E11811
:1044F4000022E5E7F2500433B3F5806FFAD10120CE
:10450400002103F00BFDFEBD703100207039002046
:10451400C84B0020CC4C0020484B002070010020E8
:10452400343B0020CC4B0020F4390020EBCE0008B3
:10453400323B00200080FFFFF0B5684B9DB07F2226
:1045440016AC1A801AAD06466549204608F0C1FB30
:1045540032462846634905F00DF82946204608F0FE
:104564009EFB0120014603F0D9FC5F4B00251D7022
:104574005E4B01221A7021465D4801F0F3FD5D484F
:10458400214608F049FAA84203DA5B4801F0EAFD43
:104594009DE006AEB31C594F2C46049330463F2190
:1045A40008F004FB002836D000211022049800F003
:1045B400A7FCDFF84CC1002145F80C000A22701D4D
:1045C40000F09EFC4F4A00211055F01D0A2200F015
:1045D40097FCDFF834C1C3B20CF8043013B1434A7A
:1045E4000021117006F10C011E223846039308F0D5
:1045F4007FFB039B434A0093135DDFF804C10193DF
:104604003A4655F80C304148214601F0ABFD364B93
:104614001A7801321A7001341E370435402CBDD18A
:10462400344808F075FA00244BE0344B1E2101FB9A
:1046340004312046FFF770FE054618B1344801F0F6
:1046440091FD38E008F0D4F9324B334A400203EBD1
:10465400C413059004932E4602EB4417DFF8BCC044
:104664005CF824309D4226D2384608F019FA002816
:1046740021DB284608F068FA0028034605DB0DF123
:104684006F00012108F070FA03463846039308F0DE
:104694003FFA039B002B0EDB049B3A69314643F837
:1046A400042F1F480493013601F05CFDDDF814C0AB
:1046B400202E6544D2D11B4B002223F81420013450
:1046C400E4B2DFF824C09CF80030A342ADD8012046
:1046D400002103F023FC1DB0F0BD00BF0200002048
:1046E4000800002029CF000874560020D44C002074
:1046F4002CCF00089439002041CF0008483B00200B
:1047040078560020C8420020084300205BCF0008F0
:10471400A8CF00086C11002048430020F439002081
:10472400C1CF0008484B002010B5002420460134B6
:104734000421E4B203F07AFC082CF7D103F079FCED
:10474400C0B27F2812D0BF2808BF204619D0DF2866
:104754000ED0EF280ED0F7280ED0FB280ED0FD285F
:104764000ED0FE2814BF012002200AE0092008E030
:10477400072006E0062004E0052002E0042000E013
:10478400032010BDF7B500F0E3FC02AC114F124E4C
:10479400124D44F8040D2046642100F0EFFD104A48
:1047A4001378002BF7D0FFF7BFFF3B780146834215
:1047B400F1D0387030700B4801F0D4FC00230A4863
:1047C4002B7001F0CFFC3078FFF7B6FE01232B707D
:1047D400E1E700BF0400002005000020703900203C
:1047E400443B002075D00008D1CF0008F0B5224921
:1047F40089B0224801F0B6FC21481F4908F00CF9A1
:104804000028A4BF01AE1F4F03DA1F4801F0AAFC21
:1048140030E03046192108F0C9F940B31B4930464D
:1048240008F07AFA1A490546002008F075FA044699
:1048340029462246174801F095FC1749284608F0F6
:104844003DFA014620B920460A2200F059FB38708F
:104854001249284608F032FA01460028D9D12046E8
:104864000A2200F04DFB0E4B01381870D1E70448C2
:1048740008F04EF909B0F0BD00D00008E9CF0008F7
:1048840074390020443B00200BD00008BADB000838
:1048940003D2000827D0000843D000084AD00008FB
:1048A40000000020F8B5DFF8FCC0C1F303249CF835
:1048B40000C0C1F307420CF1FF3C080E6445D3B2BB
:1048C4006ED101F00F0CACF10804E4B2012C4AD80B
:1048D400C1F3072101F0F001902900D148B9324A0F
:1048E40000211578314ADFF8C8C0177831480A46E4
:1048F40035E02D4A304915782E4C0022DFF8BCC033
:104904002F4F2E460BE051F8045FAB4201BF4FF02E
:10491400FF3524F812503D5C0CF802500132D5B238
:10492400B542F0D33CE0274EB45CB4B95CF8224005
:10493400A34212D127B9244CA65C0EB1445E14B92B
:104944000026465209E01D4C4652A456F60801368C
:1049540094FBF6F61D4C0136A65401320231D4B252
:10496400AC42E0D31CE0BCF10C0F11D1184C194639
:104974002270184D184801F0F5FB00232B701748DE
:1049840001F0F0FB2078FFF7D7FD01232B7007E03F
:10499400134B144A01EA0303934204BF124B1880D9
:1049A400F8BD00BF0000002074560020D44C002045
:1049B40078560020484B002074560020F43A00201A
:1049C40000CE0008C842002008430020B43900206B
:1049D400050000207039002056D00008D1CF00080F
:1049E4000F00FF000B0007000200002008B54FF481
:1049F4000071024A024803F02DFA08BDE1430008A1
:104A0400703100201FB54FF0FF3003F067FA2D4BD3
:104A140001221A702C4801F0A5FB2C4801F0A2FBDE
:104A24002B4801F09FFB002007F0C0FF002802DAAA
:104A3400284801F097FB0024002002F023F9002805
:104A440006DC0134B4F57A7FF6D1234801F08AFB01
:104A5400FFF7CCFE214B1B7833B1214801F082FBD8
:104A6400FFF762FE1F4B18701E4B00241878FFF7E7
:104A740063FD1D4801F076FB1C4B01221A700020D7
:104A8400FFF7B4FF1A4801F06DFB642003F0AAFCA1
:104A940003230093174923464FF480721648019468
:104AA4000294039400F05CFA0223009313494FF438
:104AB40080722346124801940294039400F050FA41
:104AC4001FBD00BF7857002089D00008AAD0000875
:104AD400D3D00008EAD0000805D10008443B0020E8
:104AE40027D10008050000203AD1000870390020C1
:104AF40050D1000861D10008E54100086CD10008DC
:104B0400894700087047704713B500F021FB02ACD9
:104B140044F8040D0121204600F030FC00F018FB9D
:104B2400019A431F9A4238BF019001F02BFD0248BD
:104B340001F066FBEEE700BFA948000813B500F0DA
:104B440007FB02AC44F8040D0121204600F016FCDA
:104B540000F0FEFA019A431F9A4238BF01900348BD
:104B640003F0B3FC01F095FDEEE700BF0B4B00082A
:104B740030B5002085B002F00DFA002003F074FC7B
:104B8400002003F0A1F9002002F044FF002001F00E
:104B940059FF002003F096FC002001F050FF002094
:104BA40003F004FE002000F0A9FF002001F038FD0E
:104BB400002001F03BFD002000F0BCFE012000F0CD
:104BC40079FE002006F07AFB002000F073FE00203E
:104BD40003F0AEF808F02CF8FFF714FF00F052FFD2
:104BE4004FF4FA644FF47A7003F060FC14F1FF346C
:104BF400F8D1032523460D494FF480720C480095E3
:104C040001940294039400F0ABF90A494FF48072C2
:104C140023460948009501940294039400F0A0F9F6
:104C240000F06AFA204605B030BD00BF81D100080B
:104C3400414B00087CD100080D4B0008704708B5B3
:104C4400FFF760FF08BD000070B50024642642F23F
:104C540010750134B4FBF6F306FB13430BB901F0F2
:104C640091FC084801F0CCFAB4FBF5F305FB1343BF
:104C7400002BEED103F066F9C143012003F04EF995
:104C8400E7E700BFA948000810B5036888B0079398
:104C94004368374C069383680593C3680493036998
:104CA40003934369029383690193C3692046009384
:104CB40001F058FA2F4801F055FA204601F052FA53
:104CC40007992D4801F04EFA06992C4801F04AFA4A
:104CD40005992B4801F046FA04992A4801F042FA52
:104CE4000399294801F03EFA0299284801F03AFA5A
:104CF4000199274801F036FA0099264801F032FA62
:104D0400254B2648196801F02DFA254B25481968CA
:104D140001F028FA244B2548196801F023FA244BA2
:104D24002448196801F01EFA234B2448196801F03D
:104D340019FA6FF07F4000F0D8FE002000F0D9FE91
:104D4400002000F0B7FD00F05BFE0020014600F0FB
:104D5400B7FD1B4800F088FE0121002000F0B0FDE3
:104D64000199184800F0AEFEFFF76EFF08B010BDC1
:104D7400DDD10008F1D1000805D2000810D20008E6
:104D84001BD2000826D2000831D200083DD2000808
:104D940048D2000853D2000838ED00E05FD2000882
:104DA40028ED00E06CD200082CED00E079D2000878
:104DB40030ED00E086D200083CED00E093D200081C
:104DC400A0D20008B1D200081EF0040F0CBFEFF30C
:104DD4000880EFF30980FFF757BF7047F0B587B03D
:104DE4000492464A0F4612680846039210F8012BB3
:104DF400039C014604EB020C9CF8015015F00805D5
:104E0400F4D12D2A03D111F8012B012503E02B2A1B
:104E140008BF11F8012BD3F1010038BF0020102B7B
:104E240014BF044640F00104BCB1302A10D191F8FB
:104E340000C0BCF1780F14BF00240124BCF1580F4A
:104E440008BF44F001041CB14A781023023104E085
:104E540018B1302A14BF0A230823002D0CBF6FF0A9
:104E640000404FF00040B0FBF3FC03FB1C000024A7
:104E7400059001952046039EB5186D7815F0040F32
:104E840001D0303A08E015F0030F22D015F0010FDD
:104E94000CBF57253725521B9A421ADA604594BF36
:104EA4000025012555EAD4740ED1059D604514BF33
:104EB40000240124AA42D4BF002404F001041CB934
:104EC40003FB0020013401E04FF0FF3411F8012B03
:104ED400D1E7B4F1FF3F019D06D1002D0CBF6FF067
:104EE40000404FF0004001E005B14042049E1EB175
:104EF40004B14F1E049B1F6007B0F0BD7800002072
:104F040008B58C4686461346002071466246FFF774
:104F140065FF08BD0D4B10B51A68044650600C4A75
:104F24001268904206D20B4A10681968043100F0E6
:104F3400AAFA0AE0084A10681968043100F0A3FAD2
:104F4400064B1A68944238BF1C6010BD904D002077
:104F5400A84D0020AC4D0020F04C0020180000208B
:104F6400F0B587B0039048200491144605930C9E35
:104F74000E9F00F0E7FB0546002800F09B801FB958
:104F8400A00000F0DFFB07462F631FB9284600F09E
:104F9400A3FB8FE0A2003846A52107F078FE2B6B17
:104FA40004991022671E05F1340003EB870707F00C
:104FB4009FFE002385F843302C1D042E34BF334656
:104FC4000423EB626B642046019300F04CFA05F174
:104FD400180000F048FA019B27F00707C3F1050306
:104FE400AB612D616D6238460399059A00F080FA31
:104FF4000D9B286003B11D6000F0AAFA304A1368C3
:10500400013313602F4B1F68002F28D11D601368D4
:10501400012B2CD12C4A133303FB072001370292B6
:10502400019300F015FA052F029A019BF4D1274B46
:10503400274F1846019300F00BFA384600F008FA9F
:10504400244800F005FA244800F002FA234800F04E
:10505400FFF9019B224A1360224B1F6007E0224A9A
:10506400126822B91A68D26AB24298BF1D601F4AF8
:10507400EB6A11688B4288BF13601D4A11680131C5
:1050840011601C4A11688B4288BF13600E4A1420B9
:1050940000FB0320214600F0E9F900F067FA124B07
:1050A4001B6853B1074B1B68DB6AB34205D200F09F
:1050B4003FFA02E04FF0FF3000E0012007B0F0BDFE
:1050C400D04D0020904D0020244D0020B84D0020EC
:1050D400104D0020944D0020FC4C0020DC4C00209E
:1050E400F04C0020AC4D0020F44C0020D44D0020A6
:1050F400B44D0020B04D002030B5002485B00C48DC
:105104000C494FF480722346009401940294039452
:10511400FFF726FF0128054607D100F011FA064BD8
:105124001D60064B1C6000F067FA05B030BD00BF7F
:1051340019530008BED20008F44C0020A84D0020EA
:10514400024B1A6801321A60704700BF884D002074
:1051540010B500F0FDF9034B1C6800F007FA204677
:1051640010BD00BFA84D00202F4BF7B51B68002BC6
:105174004ED12E4B1A6801321A601B68ABB92C4B06
:105184002C4A19681068186011602B4A11680131A3
:1051940011601A681168294A11B94FF0FF3303E00E
:1051A4001B68DB68DB685B681360204F234B3A683D
:1051B4001B689A4232D31E4D214C224E2B681B6829
:1051C40013B94FF0FF3206E02B68DB68DB683968FF
:1051D4005A68914202D2194B1A601FE01A1D1046F8
:1051E4000192009300F069F9009B9A6A22B103F1DD
:1051F400180000F062F9009BD86A2368019998426C
:1052040088BF2060142303FB006000F02FF9D5E76A
:105214000D4B1A6801321A60FFF710FD0A4B1B6828
:105224000BB9FFF70BFDFEBD884D0020A84D0020F3
:10523400F04C0020AC4D00208C4D002018000020C4
:10524400B04D0020244D0020D84C0020F7B500F0CC
:105254007FF9284B1A68013A1A601D68002D43D162
:10526400254B1C68002C40D0244F254E1DE0FB68C4
:10527400DC6804F1180000F020F9211D08460191B2
:1052840000F01BF9E06A3368019998421D4B88BF0E
:105294003060142202FB003000F0E8F81A4A136868
:1052A400E26ADB6A9A4228BF01253B68002BDED103
:1052B400164C23682BB908E0FFF756FF2368013B1F
:1052C40023602368002BF7D107E0012D05D0104A95
:1052D4001268012A18BF1C4607D10D4B00221A6020
:1052E40000F026F9012400E0002400F03FF92046F4
:1052F400FEBD00BF884D0020D04D0020944D0020FD
:10530400B04D0020244D0020904D0020D84C0020AA
:10531400CC4D0020F8B5154C154F164E1AE0FFF78A
:105324000FFF3D68FFF792FFA5B100F011F9FB688C
:10533400DD68281D00F0C1F83368013B3360236841
:10534400013B236000F012F9286B00F0C5F92846F0
:1053540000F0C2F92368002BE1D1074A1368012B3E
:1053640001D900F0E5F8FFF76AFCF3E7F84C0020F8
:10537400FC4C0020D04D0020244D002038B50C46B4
:105384000546FFF7DDFE124A2B681168E4189942BE
:1053940002D29C4208D201E09C4207D313689C428B
:1053A40094BF0023012302E0002300E001232C60CA
:1053B4003BB1084B1868043000F07FF82046FFF733
:1053C400A9FDFFF743FF08B900F0B2F838BD00BFEC
:1053D400A84D0020904D0020184B10B51B6833B128
:1053E4000122174B28E018680138186002E0154BB9
:1053F40015491422D3F800C0134802FB0CFC51F8E1
:105404000C40002CEFD00F4B4FF0140C19680CFB20
:1054140001FC00EB0C035A680CF1080C5268604460
:1054240082425A6004BF52685A60074B142202FB3E
:1054340001314B68DA68054B1A6010BD884D0020B5
:10544400CC4D0020B04D0020244D0020904D002074
:1054540000F108034FF0FF3282604360C3600361D0
:1054640000230360704700230361704743685A6850
:105474008B604A605A6891605960036841600133E7
:105484000861036070470A68B2F1FF3F0CBF03690B
:1054940000F1080301D106E05B68D3F804C0DCF82E
:1054A40000C09445F8D95A68086191604A6059600F
:1054B4008B600368013303607047436882689A60B5
:1054C4008268536003695968814208BF5A600022A8
:1054D40002611A68013A1A60186870470348006844
:1054E400006880F3088862B600DF00BF08ED00E0C2
:1054F400031F4FF0807C40F804CC181F43F8041CB1
:10550400002140F8041C40F8182CA3F13C0070471B
:10551400064B19680868B0E8F00F80F309884FF06B
:10552400000080F311884EF00D0E7047904D00205E
:10553400024B4FF080521A60704700BF04ED00E048
:10554400EFF311804FF0BF0181F311887047002001
:1055540008B5FFF7F5FF024B1A6801321A6008BD5F
:105564001C00002080F311887047000008B5044B2C
:1055740018680138186008B9FFF7F4FF08BD00BFC8
:105584001C000020EFF309800C4B1A6820E9F00F8F
:1055940010602DE908404FF0BF0080F31188FFF739
:1055A4001BFF4FF0000080F31188BDE80840196824
:1055B4000868B0E8F00F80F309887047904D002028
:1055C40008B5064B4FF080521A60FFF7B9FFFFF79A
:1055D400CBFD0020FFF7C6FF08BD00BF04ED00E0CF
:1055E400034A044B1A600722043B1A60704700BF49
:1055F4003F19010014E000E0094B10B51A680024BB
:1056040042F47F021A601A6842F07F421A60FFF780
:10561400E7FF044B1C60FFF761FF204610BD00BF8D
:1056240020ED00E01C000020F0B50C2404FB00FC7D
:1056340009180B4B04FB01F533F80C605F1926F4D1
:1056440000465E53788033F80C0089B24004400C65
:1056540004FB0034618042EA010123F80C10F0BD20
:10566400885700200C2110B548430A4B1A18B2F889
:1056740006C0948801FB0C3CACF80440B2F804C0AA
:10568400D28801FB0C31CA801A5A22F400421A5201
:1056940010BD00BF88570020F8B50C2505FB00F6A7
:1056A4000C4C0746A05B05FB00F3E35E002B0FDA0E
:1056B400FFF7D8FFA35B6B43E35A5B045B0C05FB6A
:1056C40003435F80A35B5D43635B23F40043A35305
:1056D400F8BD00BF8857002070B5064600282ED0BC
:1056E400174C0C25361BFFF72BFDB6FBF5F6B6B2AF
:1056F4003046FFF7D1FF05FB06F3E21850886843F4
:10570400215E00290BDAE15A6FEA41416FEA514107
:105714002152E35A528805FB034462800DE0A188BC
:1057240005FB014591800021EE80A680D180E25ADC
:105734006FEA42426FEA5242E252FFF787FD70BDC0
:1057440088570020F7B5064600287FD0FFF7F8FCFD
:10575400082E07D9A6F109010C23B1FBF3F102319C
:1057640089B200E001213A4847F6FF738488002596
:1057740022464FF00C0E18E030F80C506D04C4EBC8
:105784005545ADB28D4234BF4FF0000C4FF0010CC3
:105794009D422CBF4FF0000C0CF0010CBCF1000F2B
:1057A40018BF224618BF2B4634460EFB04FC00EB00
:1057B4000C06B688002EDFD147F6FF70834218BF6F
:1057C4001D4618BF14460C226243214B9A5A5204B8
:1057D400560C82B18D4203D12046FFF743FF2EE0E1
:1057E4006D1AADB2204629464FF400422C19FFF73A
:1057F4001BFFA4B223E06218B2F5557F06DB2246F4
:10580400144800F0AFFCFFF721FD1FE01CB9012292
:105814001A809A8001340C2202FB04F30C4E6518A2
:10582400F118C888AFB202FB006002FB05658780EF
:105834002846019307F020FA019B6C80F752FFF78A
:1058440005FD034B0C2606FB043604363046FEBD2C
:1058540088570020E8D30008684620F007018D46E9
:1058640001B50A4A0A4B0B4903E052F8040B43F80A
:10587400040B8B42F9D3084B0849002201E043F89A
:10588400042B8B42FBD3FFF773F9FEE720EA0008F1
:10589400000000207001002070010020C07F002063
:1058A4007047FEE7024B93F90000C00F704700BF3A
:1058B400887F0020014B187000207047E44D0020C1
:1058C40008B50B4B18800B4B19800B4B9A8812B1FF
:1058D400D2B29B7901E0082306224243DFF81CC0C0
:1058E4004B43ACF80020064A138005F0A9FF08BD1D
:1058F400927F0020987F0020D84D00209A7F0020BE
:10590400847F002008B5034B1880034B198005F0F1
:105914002BFF08BD9A7F0020847F0020044A0023C7
:10592400C15C99540133042BFAD10020704700BFA5
:10593400947F002007B5002839D11E4B1E4A9C468F
:1059440007CAACE80300ACF800201C4A1278422ACB
:105954000ED11B4A12781A701A4A12785A701A4ACF
:1059640012789A70194A12789A80194A1278DA8051
:10597400184B00229A80184B02A81B6840F8043D7B
:10598400FFF7CCFF4CF2503002F090FD002005F000
:1059940095FC00280DDB05F059FE00200146FFF7B9
:1059A4008FFF00200146FFF7ADFF002001E04FF01C
:1059B400FF300EBD887F002080D40008C03F00085F
:1059C400C13F0008C23F0008C33F0008C43F0008AD
:1059D400C53F0008D84D00200CD400088278074B3E
:1059E400043282181A6002789A804278DA80C27887
:1059F40000201A8101229A72704700BFD84D0020FE
:105A040008B505F023FE08BD1FB5144B844693F971
:105A14000030002B17DA124B4FF0FF309A88D2B1C6
:105A24000DF1040E93E807008EE80700DA8819895F
:105A3400D2084A430CFB020CCDF804C09EE80700D0
:105A440005F02CFF01E005F043FB002803DB054BC8
:105A54001A8801321A8005B000BD00BF887F00207B
:105A6400D84D0020927F002038B50546002402E07E
:105A7400FFF7CAFF044315F8010B0028F8D12046AC
:105A840038BD000038B50C4B00241C70214620465C
:105A9400FFF716FF05460948FFF7E6FF012140EA34
:105AA40005052046FFF70CFF05430548FFF7DCFF1B
:105AB40045EA000038BD00BFE44D002089D000084D
:105AC400AAD000080FB410B592B014AA52F8041B5F
:105AD40001AC2046119203F05CFD2046FFF7C4FFA1
:105AE40012B0BDE8104004B0704708B505F0D0FE10
:105AF40008BD08B505F0CFFE08BD000038B5044662
:105B04004FF0FF30002C39D11D4A102313701D4A69
:105B1400204613701C4B1C601C4B1C601C4B1C60EF
:105B24001C4B1C601C4B1C601C4B1C6002F0A0FF37
:105B3400C50F204600F0CEFD0028B8BF45F0020591
:105B4400002000F071FF164A0028B8BF45F0040594
:105B540000231370134A1370134A1370134B1B78EA
:105B6400422B05D1124B1B7813F0800F08BF137022
:105B7400104A00231380104A6842136038BD00BFE6
:105B84002100002022000020F04D0020E84D0020DC
:105B9400104E0020144E0020084E0020F44D00202A
:105BA400F84D0020004E0020FA4D0020D03F0008A0
:105BB400D13F0008FC4D00200C4E002010F0F00FE7
:105BC40070B505460C4604D101280CBF164B174B83
:105BD4001D78174B05F00F061B682BB166F30714ED
:105BE400284621469847E8B905F0F005202D0CD049
:105BF400302D11D0102D18BF4FF0FF3012D166F3A5
:105C04000714204602F0A6FF0CE066F307143046A2
:105C1400214600F019FE05E066F3071430462146DC
:105C240000F007FF70BD00BF22000020210000200B
:105C3400E84D0020F0B585B0174603900D460026C8
:105C4400062307224FF0040C40E0B91B022914D0AC
:105C540003291FD00129A95D18BF6CF3030406F1C1
:105C6400010618BF61F30F241AD1052060F3030461
:105C740061F30F246FF3174409E0A95D63F3030490
:105C8400013661F30F24A95D013661F317446FF304
:105C94001F640DE0A95D62F3030461F30F24013670
:105CA400A95D013661F31744A95D013661F31F64F0
:105CB4000398214601920293CDF800C0FFF77EFFBE
:105CC4000028019A029BDDF800C002DBBE42BCD36F
:105CD400002005B0F0BD000010B5F023A0B08DF891
:105CE400003000238DF801308DF802307E338DF8BA
:105CF400033032238DF804300E4B0DF16B0C1B78FE
:105D04008DF805300F238DF806306B46DA1D03E05D
:105D140002F8014B624503D011F8014B002CF7D176
:105D2400F72102F8011BD21A6946FFF783FF20B05E
:105D340010BD00BFFA4D002000B5F02389B08DF8E6
:105D4400003000238DF801308DF802307E338DF859
:105D5400033032238DF80430084B8DF806101B787D
:105D64008DF807208DF805306946F72309228DF850
:105D74000830FFF75FFF09B000BD00BFFA4D0020F7
:105D8400F7B517460025042262F303056FF00F02EE
:105D940062F30F256FF317456FF31F650B46294612
:105DA40004460193FFF70AFF7E2262F30F25322295
:105DB40062F317450C4A06461278204662F31F65C3
:105DC4002946FFF7FBFE0D22019B62F30F2563F3C7
:105DD400174567F31F6540EA060629462046FFF784
:105DE400EDFE46EA0000FEBDFA4D0020F0B585B098
:105DF40003900B461646002A35D000250F462E4642
:105E04004FF0040C2DE0595D6CF3030431B101F043
:105E14007F0161F30F24797819B909E061F30F2444
:105E240006E001F07F0161F31744B97819B907E07E
:105E34006FF3174404E001F07F0161F31F6401E094
:105E44006FF31F640398214600920193CDF808C0B4
:105E5400FFF7B4FEDDF808C0019B009A0643033542
:105E640003379542CFD3304605B0F0BD08B50021C5
:105E7400052363F303016FF0080363F30F216FF34A
:105E840017416FF31F61FFF799FE08BDF8B505468A
:105E940006F026FF0A4E0746402130782A78FFF79D
:105EA4006FFF012F044605D93078691C7A1EFFF76D
:105EB4009DFF0443024B1878FFF7D8FF2043F8BD39
:105EC4002200002030B50B465E498BB009780446A9
:105ED4000D295ED001D839B1A6E00E2900F0AE80BC
:105EE4000F2940F0A18093E01BB1012B564B02D146
:105EF40056E0554AA1E01B78052B25D00AD8022B81
:105F040017D002D8012B40D111E0032B13D0042B5E
:105F14003BD112E0082B2FD004D8062B1ED0072B20
:105F240033D11EE0092B29D07F2B2ED12AE04749FB
:105F340025E0474923E0474921E000F0CDFF6D46C5
:105F440002464549684612E0684600F0DBFF002837
:105F54006D46BCBF204641490BDA10E000F0C2FF99
:105F640001E000F0C7FF3E4902466D46684603F073
:105F740001FB2046694602E03A4900E03A49FFF74E
:105F8400ABFE5BE000F06CFF58E020460E210D22D2
:105F940047E01BB1012B354D18D103E0334BFF22F1
:105FA4001A704BE02B78FF2B08BF2A7046D013B130
:105FB400012B43D101E02E4B00E02E4B1B68002B3C
:105FC4003CD02D4908781146984737E02A78B2B971
:105FD4000F21FFF7B1FE2B78002B2FD1244B1B6828
:105FE400002B2BD1254B012C1D78254818BF1C7084
:105FF400FFF74CFF012D1CBF204B1D701EE0012A32
:1060040002D11C4B1B68CBB920460E21102208E09C
:106014001C4A13B1012B1B4A01D153600EE0526894
:1060240062B9FFF789FE09E00E210A462046FFF710
:1060340083FE144A00231370024A137000200BB02D
:1060440030BD00BFEC4D0020F94D0020ACD4000859
:10605400B3D40008C3D40008B9D20008CDD40008D2
:1060640029CF000889D00008AAD000082000002009
:10607400084E0020F44D0020F84D0020220000209E
:10608400CFD40008004E0020F72910B50A465CD88A
:106094002F4B1C7804F00803DBB21BB12D4909789F
:1060A40081424FD1A0F11101C9B206294AD9294927
:1060B40008700BBB264B1B7803F00703042B03D893
:1060C4002549C95C914223D104F00704052C03D16E
:1060D4002249097891421BD1013303F007021C4B7A
:1060E400052A197862F3020184BFCAB242F0080299
:1060F400197088BF1A7028E012F0800F0ED0F72AAA
:1061040006D104F01004E4B214B10221FFF7DAFE60
:106114000F4B00201870124B187017E004F0100495
:10612400E4B25CB90A4B197841F0100119700C4BB8
:1061340021461A70FFF7C6FE204607E00121FFF74B
:10614400C1FE02E04FF0FF3000E0002010BD00BFB0
:10615400004E0020F84D0020BCD50008FA4D002068
:10616400EC4D00200FB430B5A3B0269D284606F0B0
:10617400B7FD642888BF0E4813D801AC27AA294666
:106184002046219203F005FA204606F0A9FD2018C6
:1061940004E0237803F07F0304F8013B8442F8D140
:1061A40001A8FFF773FE23B0BDE8304004B0704788
:1061B4001DD5000810B50D4A0446137803F00803F2
:1061C400DBB23BB10A4B1B78834203D1002313702B
:1061D400084A1370084B1B680BB1204698472146A8
:1061E4000648FFF7BFFF002010BD00BF004E00208F
:1061F400F84D0020EC4D0020144E002070D500080E
:10620400F0B5002289B00121054604910192039260
:10621400134600E0059B5A1CD2B205920C2B58D8A9
:10622400DFE803F0070F151B21272D33393F454BBA
:10623400510007A802F0A8FC079CC4F3031410340F
:1062440058E0002007A900F00BFB202452E00120B5
:1062540007A900F005FB21244CE0022007A900F067
:10626400FFFA222446E0032007A900F0F9FA2324C8
:1062740040E0002007A900F0DFFB30243AE00120D1
:1062840007A900F0D9FB312434E0022007A900F06B
:10629400D3FB32242EE0032007A900F0CDFB3324E6
:1062A40028E0042007A900F0C7FB342422E00520DD
:1062B40007A900F0C1FB35241CE0062007A900F063
:1062C400BBFB362416E0072007A900F0B5FB3724F2
:1062D40010E0019A0399131E18BF012309298CBFEA
:1062E400002303F00103002B00F03F810022019200
:1062F400059208E110F10A0F04D12046FFF75AFF76
:10630400002332E10028C0F2FE800199039A4B1C5D
:10631400DBB207990193531CDBB26FF307110393AC
:1063240001F00F0303F1080202F00F02062A07919D
:1063340004D82046002D40F0E580E4E09A1E0D2AA2
:1063440000F2E180DFE812F07A007A000E007600B5
:106354007D007D00DF00DF00DF00DF00DF00DF0005
:10636400DF000E009DF81D10F72967D8F0291CD115
:10637400804A1368CBB904F0F002102A02D0302A04
:1063840013D109E07C4A1380012204F00F0312FAAE
:1063940003F3784A138008E0774A1380012204F05B
:1063A4000F0312FA03F3734A53802046FFF76CFE7F
:1063B4009DF81C3003F00F030F2B09D09DF81E101D
:1063C4002046FFF761FE9DF81F102046FFF75CFE94
:1063D4006A490B7803F00803DBB2002B40F093808A
:1063E400674A1668DEB19DF81D102046B0479DF837
:1063F4001C30C6B203F00F030F2B10D0604A9DF877
:106404001E101368204698475D4A07469DF81F10E2
:10641400136820469847074347EA0606F6B22B1E40
:1064240018BF0123002E14BF002603F00106002E1E
:1064340069D065E09DF81D20F72A02D9002D5FD1AF
:1064440061E0043BDBB20293002B00F090809DF8E6
:106454001D6020463146FFF717FE48490B7803F0CC
:106464000803DBB23BB9464A17682FB120463146D0
:10647400B847C7B200E00027029B012B2CD09DF83F
:106484001E6020463146FFF7FFFD3C490B7803F0C0
:106494000803DBB243B93A4A13682BB120463146AC
:1064A400984740EA0707FFB2029B022B14D09DF8DD
:1064B4001F6020463146FFF7E7FD30490B7803F0B3
:1064C4000803DBB243B92E4A13682BB12046314688
:1064D400984740EA0707FFB2F72E02D1254B002167
:1064E4001960264A137803F00803DBB25BB92B1E4C
:1064F40018BF0123002F14BF002703F0010717B1B1
:1065040007992046A8471B4B1A683AB31A4A1288BF
:10651400B2F57A7F22D9198861B1002251FA02F3C7
:1065240013F0010303D10132102AF7D11A461032B5
:10653400D0B20DE0588858B10B4650FA03F212F06D
:10654400010203D10133102BF7D113463033D8B2F3
:10655400FFF730FE074B00221A6003E0049B002B78
:106564007FF458AE002009B0F0BD0493CBE7029F3E
:10657400B7E700BF0C4E0020FC4D0020004E002069
:10658400104E002010B502F02BFB044600F0CAF8B0
:1065940040EA040400F04BFA054B4FF6FF711A88E9
:1065A40044EA00008A4201D001321A8010BD00BFC3
:1065B400FC4D002008B5034B1B680BB1984700E065
:1065C400184608BDF04D0020F0B5134E85B0346870
:1065D4000746ECB1C1F307638DF80E300F4BC1F3DE
:1065E4000742C1F30720002401F00F018DF80D20AC
:1065F4008DF80C005A5C254608E003AB595D38461B
:10660400019233689847019A044301359542F4DBBB
:10661400204605B0F0BD00BFF04D00209CD400081A
:10662400002814BF4FF0FF300020704738B9054BE5
:10663400054A186010231370044A137001E04FF0E8
:10664400FF307047184E0020230000202400002053
:1066540010F0F00F08B504D101280CBF064B074B0E
:1066640018780309022B18BF4FF0FF3003D100F054
:106674000F0002F093FC08BD24000020230000203A
:1066840007B502AB03F8011D19460122FFF7E0FF2D
:106694000EBD002300E013465A1C042BD2B2FAD9D3
:1066A40000207047012810B5044688BF4FF0FF3022
:1066B4000BD800F0FFFC054BFF221A55044B0022B7
:1066C40023F8142000F00CFD002010BD1C4E002007
:1066D4003C4E002010B504464FF0FF30ECB90F4B90
:1066E400FF221C601C715C719C71DC711C81DC607C
:1066F4001C745C749C74DC749C82094B20461A7074
:10670400FFF7D0FF0120FFF7CDFF204602F0B0FADB
:106714000028B4BF4FF0FF30002010BD204E0020F1
:10672400384E002008B500F0C5FC124B4FF6FF713F
:106734001A888A4201D001321A800F4B4FF6FF713A
:106744001A898A4201D001321A810A4B4FF6FF712D
:106754005A888A4201D001325A80074B4FF6FF71A2
:106764009A8A8A4201D001329A8200F0B9FC002050
:1067740008BD00BF3C4E0020204E0020F7B5012884
:10678400C1F3072601F00F03C1F307420446F7B231
:10679400C1F3076144D846E026488DF8046030F818
:1067A40014C08DF80520BCF57A7F8DF8061003D946
:1067B4002046FFF777FF22E0DFF87CC09CF800C09A
:1067C4004CFA04FC1CF0010F19D0072B17DD0E2B1B
:1067D400CCBF00230123012D94BF002303F0010348
:1067E4006BB1164B1B5DBB4206D1013D8DF80420F5
:1067F4008DF80510EDB202E0002320F81430F72FD5
:1068040098BF0E4B204698BF1E5501A92A4602F098
:10681400C5FB023002289CBF094B53F8200001D964
:106824004FF0FF30FEBD0748C55C2846002DB3D1AC
:10683400F8E700BF3C4E0020384E00201C4E0020DC
:10684400C4D500089CD4000838B505460C46284633
:106854002146FFF793FF10F1020FF8D038BD000076
:106864000128F8B504460E4688BF4FF0FF3000F209
:10687400D280ABE0C0B210F0800F55D0F72808D911
:10688400336843F00F03336000237070B370F37008
:10689400C2E0C0F30213FB5C28716B71002B3BD187
:1068A4005E4900F00F028A5CF0286A7103D101226C
:1068B4006870EA7131E0F72821D1EA791AB1012A26
:1068C4002A7810D108E02B78052161F303032B709B
:1068D4006870AA70EA700CE0062161F303022A7062
:1068E400A870EB7005E01346072262F303032B70D4
:1068F400E8702B6833600023EB7101330DE062B95B
:106904002B78052161F303032B706870AA70EA7079
:106914002B683360012300E000236A79AA71002206
:106924002A81002B57D077E02B79F02B17D1EB7904
:106934000133DBB2012BEB7102D0022B04D101E055
:10694400687048E0A87046E02B78042262F30303E1
:10695400E8702B702B6833600023EB715CE0AB793B
:1069640023B96A792B81013AAA7101E0013BAB7129
:106974006B79012B03D1013BA870EB7004E0AB7978
:106984000BB1A87000E0E870AB7923BB2B7903F05E
:10699400F002F02A02D01A092B780BE06B791BB1B4
:1069A400012B2B7805D102E02B78052202E002228C
:1069B40000E0032262F303032B700C236343184AA1
:1069C400D11808794870D358336025E0144B0C254E
:1069D40005FB0435134F204602F0EEF90028BFF6FC
:1069E40049AF00200C235C430D490B199A796AB115
:1069F4001A89B2F57A7F09D900220A511A715A719B
:106A04009A71DA711A816FF0090004E000280CBF52
:106A14004FF0FF300020F8BD0120E3E78CD40008DC
:106A2400204E0020B4D500084FF0FF3070470020FE
:106A340070474FF0FF3070474FF0FF3070474FF012
:106A4400FF3070474FF0FF30704710B504464FF0E9
:106A5400FF304CB92146204600F078FB2046032144
:106A6400072200F02FFF204610BD10F0800FF8B56C
:106A740004460D46164609D077200021FF22FFF771
:106A8400F4FF0128074675DC04F07F040020024669
:106A9400014600F071FC0020214600F0B5FC290EEF
:106AA400002000F0B1FCC5F30741002000F0ACFC6D
:106AB400C5F30721002000F0A7FCE9B2002000F094
:106AC400A3FC0020314600F09FFC4D2C11D1FF2186
:106AD400002000F099FCFF21002000F095FC00202C
:106AE400FF2100F091FC0746FF2814BF0025012573
:106AF4000DE000250020FF2100F086FCFF2807465A
:106B040004D10135082DF5D1012500E00025482CDC
:106B140014BF002301237A2C14BF1C4643F0010444
:106B2400C4B1BDB9FF21002000F06EFCFF210606B0
:106B3400002000F069FCFF210746002000F064FCFF
:106B4400FF210446002000F05FFC46EA07470743A4
:106B540047EA04270020FF2100F056FC55B100202D
:106B64000146012200F008FC0020FF2100F04CFC4B
:106B74004FF0FF373846F8BD002070B501460122BA
:106B840000F0FAFB00200321072200F09BFE002402
:106B94000020FF21013400F037FC0A2CF8D100203A
:106BA4000146024600F0E8FB4FF47A7001F07EFCE7
:106BB400402000219522FFF758FF0028044654DBAB
:106BC4002F4C00254820872225704FF4D571FFF7FC
:106BD4004CFFB0F5D57F19D1E9204FF08041FF2259
:106BE400FFF743FF044620B10135B5F5804FF3D1DB
:106BF40039E0FF227A202146FFF737FF204B10F0BF
:106C0400804F0CBF04220C221A7029E0E920FF22D5
:106C14002946FFF72AFF012801DC022300E00123B3
:106C2400174E237000253378022B03D1E92000216D
:106C3400FF2202E041200021F922FFF716FF00287D
:106C4400044604DB03D00135B5F5804FEBD1502069
:106C5400F9224FF40071FFF708FFB5F5804F02D019
:106C6400074B1B780BB96FF0010400200122014689
:106C740000F082FB0020FF2100F0C6FB204670BD1F
:106C8400404E002038B5044678B10321012200208B
:106C940000F018FE00200146024600F06DFB4D2076
:106CA4000021AF22FFF7E1FE25E00321072200F0D7
:106CB40009FE20462146012200F05EFB0A24013C25
:106CC4000020FF21E4B200F09FFB002CF7D1214605
:106CD4002246204600F050FB402095222146FFF733
:106CE400C4FE0028054607DB21460122204600F0A9
:106CF40043FBFFF741FF054600200122014600F057
:106D04003BFB0020FF2100F07FFBD5F1010038BFE1
:106D1400002038BD73B5244B04461B780E4613F08F
:106D2400080F08BF440203210122002000F0CAFD1D
:106D34005120FF222146FFF798FE0028054603D084
:106D4400B8BF6FF0FF0523E004460020FF2100F0E8
:106D54005BFBC0B2FF2806D10134B4F5803FF4D107
:106D64006FF4807514E0002432464FF4007321461A
:106D74002046009400F026FFFF21204600F044FB4B
:106D8400FF21204600F040FB2046FF2100F03CFBA1
:106D940000200122014600F0EFFA0020FF2100F05C
:106DA40033FB28467CBD00BF404E002037B52A4B3C
:106DB40004461B780D4613F0080F08BF4402032154
:106DC4000122002000F07EFD58202146FF22FFF71B
:106DD4004CFE0028044603D0B8BF6FF0FF042FE038
:106DE400FE2100F011FB22464FF400732046294691
:106DF400009400F0E7FEFF21204600F005FBFF2190
:106E0400204600F001FB2046FF2100F0FDFA00F0CF
:106E14000F00052818BF6FF4807411D12546002097
:106E2400FF2100F0F1FA10F0FF0F05D10135B5F59F
:106E3400001FF4D1094C03E00020FF2100F0E4FA24
:106E440000200122014600F097FA0020FF2100F003
:106E5400DBFA20463EBD00BF404E0020FEFEFFFF91
:106E640008B5FEF775FB6FF07F40FEF73EFE00208D
:106E7400FEF73FFE0020FEF71DFDFEF7C1FD0020DA
:106E84000146FEF71DFD1148FEF7EEFD00F012F974
:106E940000214FF0FF3001F041F86FF007000121AD
:106EA40002F0B6FF6FF40000012102F0BFFF4FF0C3
:106EB400FF30002102F0ACFF4FF0FF30002102F060
:106EC400B5FF034A034BDA60FEE700BFD0D50008E4
:106ED4000100FA0500ED00E0014B1868704700BF9F
:106EE400002004E0024B188880B28002704700BF83
:106EF400E0F7FF1F024B188880B28002704700BF82
:106F0400E2F7FF1F00230B4A59108A18127813F076
:106F1400010F08BF120902F00F02092A94BF3021A1
:106F240037218A18C2540133182BECD1002303767D
:106F340018467047E8F7FF1F07B56B4683E8030060
:106F440001214FF0C05002F055FF012003F00EF86C
:106F540003F004F84FF4407002F0CEFE012002F07A
:106F6400D3FE02F0EDFF02F0E3FF0120014602F040
:106F74009DFF02F0DDFF064802F0CAFF02F0D8FFD1
:106F8400009802F0B7FF02F0D3FF00200EBD00BF4F
:106F9400356E010030B5054685B04FF0FF30002D49
:106FA40077D103AC01217D2002F016FF204602F0C8
:106FB40051FB482321468DF80F3037484EF2FF73BA
:106FC400ADF80C3002F0EDFA4FF0FF3321463348B0
:106FD400ADF80C3002F0E5FA2146314802F0E1FA4E
:106FE4002146304802F0DDFA02F050FE082808BFBE
:106FF4002C4633D002F0F4FD4FF4803002F010FE42
:1070040002F03EFF0128044628D1102002F06EFB56
:10701400022002F061FB284602F040FE284602F0FE
:1070240051FE4FF4806002F043FE4FF4004002F042
:1070340059FE4FF480304FF4801102F00DFE2046CB
:1070440002F014FE392002F005FF0028FAD00220D5
:1070540002F012FE02F01AFE0828FBD100211248A9
:1070640002F094FF4FF4407002F086FF042002F017
:1070740099FF0E4A0E4B1A6000230193029301AB51
:1070840093E80300FFF758FF012C14BF4FF0FF30C3
:10709400002005B030BD00BF0008014000100140D1
:1070A40000140140000C01400040000800FF1F00D4
:1070B400042004E0084B1B681BB9EFF31082074B54
:1070C4001A604FF0010080F31088034B00201A6807
:1070D40001321A60704700BF484E0020444E002021
:1070E400064A4FF0FF3013683BB1013B13601BB9F4
:1070F400034B1B6883F3108800207047484E002020
:10710400444E00200F2988BF4FF0FF3018D80D4B94
:1071140042B2DB685209DB43C3F30223C3F1040325
:107124009940094B0901C318C9B283F8001300F050
:107134001F00012313FA00F0034B43F82200002040
:10714400704700BF00ED00E000E100E073B50446C5
:107154000D4601A802F07EFA072D00F20381DFE854
:1071640005F00A0806040C131A2100251BE000256B
:1071740012E0002509E0002500E0012503238DF835
:1071840006301026153313E0012503238DF806304D
:10719400142619330CE0012502238DF8063010263D
:1071A400163305E0012502238DF8063014261A3320
:1071B400012C5DD006D3022C18BF6FF0010540F0FE
:1071C400D380A2E001AC55B3DDB268482023214648
:1071D400ADF804308DF8075002F0E3F980236348DA
:1071E4002146ADF8043002F0DCF910235F48214653
:1071F400ADF804308DF8075002F0D3F948F20003DB
:107204005B482146ADF804308DF8076002F0C9F9F7
:1072140040238DF80750ADF8043054484EE08DF803
:107224000730524820232146ADF8043002F0B9F962
:1072340080234E482146ADF8043002F0B2F9102301
:107244004A482146ADF804308DF8076002F0A9F9E8
:1072540048F2000346482146ADF8043002F0A1F993
:1072640048238DF807304023ADF804303F4875E0DB
:1072740001AC45B3DDB23F484FF400532146ADF8AD
:1072840004308DF8075002F08CF948F200033948B5
:107294002146ADF8043002F084F94FF480533548A8
:1072A4002146ADF804308DF8075002F07AF94FF416
:1072B400804330488DF80750ADF80430214602F081
:1072C40070F9002550E08DF807302A484FF4005338
:1072D4002146ADF8043002F064F948F20003254871
:1072E4002146ADF8043002F05CF94FF48053214894
:1072F4002146ADF804308DF8076002F052F94823B6
:107304008DF807304FF4804325E05DBB02AC402389
:1073140024F8043D174821468DF8076002F041F92E
:10732400202314482146ADF8043002F03AF94FF412
:1073340000530F482146ADF8043002F032F94FF4FF
:1073440080430B482146ADF8043002F02AF9482363
:107354008DF8073080230748ADF80430214602F049
:1073640020F901E06FF0020528467CBD00080140C9
:1073740000100140000C0140012817D005D3022859
:1073840018BF6FF0010137D11AE011B1012931D1D1
:1073940006E012B11022194B1AE01021174B26E017
:1073A4004FF4004112B34FF400421BE011BB1AB179
:1073B4004FF48052124B0BE04FF48051104B16E007
:1073C40011B1012916D108E022B10E4B4FF400523D
:1073D4001A6111E04FF4005108E04FF480412AB1E2
:1073E4004FF48042074B00211A6105E0054B5961B7
:1073F400114601E06FF002010846704700080140A1
:10740400000C0140001001400128F7B500F03C8257
:1074140038BFDFF8A034C0F03882022818BF6FF0FC
:10742400010040F04582DFF890341B78032B00F212
:107434003D82DFE813F0040096001801A801DFF88C
:107444007C3411F0800F0CBF4FF4001220221A611B
:10745400402211F0400F0CBF4FF4001020209E6812
:107464001A611A611A615A6118619D681A6115F0EE
:10747400800518BF022511F0200F0CBF4FF4001037
:1074840020201A611A615A6118619C681A6114F00B
:10749400800418BF042411F0100F0CBF4FF4001027
:1074A40020201A611A615A611861D3F808C01A6160
:1074B4001CF0800C18BF4FF0080C11F0080F0CBF23
:1074C4004FF4001020201A611A615A6118619868FB
:1074D400C6F3C01610F0800018BF102011F0040F7E
:1074E40001900CBF4FF4001020201A611A611A6138
:1074F4005A6118619F681A6117F0800718BF202726
:1075040011F0020F0CBF4FF4001020201A611A6111
:107514005A61186198681A6110F0800018BF10460B
:1075240011F0010F0CBF4FF4001120211A611A61F0
:107534005A611961996821F07F0141EA06062E43D8
:10754400019946EA040444EA0C0C4CEA010C4CEAA6
:10755400070747EA00001A61C0B21A611A615A614A
:10756400A6E1D64B402211F0800F0CBF4FF400105F
:10757400202011F0400F1A6118615A610CBF4FF4BA
:10758400001020209E681A6118615A619D681A6172
:1075940015F0800518BF022511F0200F0CBF4FF421
:1075A4000010202018615A619C681A6114F080044C
:1075B40018BF042411F0100F0CBF4FF4001020204A
:1075C40018615A61D3F808C01A611CF0800C18BF06
:1075D4004FF0080C11F0080F0CBF4FF400102020DE
:1075E40018615A619868C6F3C01610F0800018BF7D
:1075F400102011F0040F01900CBF4FF40010202054
:107604001A6118615A619F681A6117F0800718BFE0
:10761400202711F0020F0CBF4FF400102020186136
:107624005A6198681A6110F0800018BF104611F072
:10763400010F0CBF4FF40011202119615A619B689E
:10764400019A23F07F0343EA060646EA050545EA64
:10765400040444EA0C0C4CEA020C4CEA070747EA1F
:107664000000C0B224E1954B11F0800F0CBF4FF421
:10767400001220221A61402211F0400F0CBF4FF477
:10768400001020209E685A615A615A611A6118617B
:107694009D685A6115F0800518BF022511F0200F6E
:1076A4000CBF4FF4001020205A615A611A6118610E
:1076B4009C685A6114F0800418BF042411F0100F60
:1076C4000CBF4FF4001020205A615A611A611861EE
:1076D400D3F808C05A611CF0800C18BF4FF0080C96
:1076E40011F0080F0CBF4FF4001020205A615A61AA
:1076F4001A6118619868C6F3C01610F0800018BFAC
:10770400102011F0040F01900CBF4FF40010202042
:107714005A615A615A611A6118619F685A6117F077
:10772400800718BF202711F0020F0CBF4FF4001080
:1077340020205A615A611A61186198685A6110F0E0
:10774400800018BF104611F0010F0CBF4FF4001158
:1077540020215A615A611A611961996821F07F01E7
:1077640041EA06062E43019946EA040444EA0C0C55
:107774004CEA010C4CEA070747EA00005A61C0B220
:107784005A615A617EE04D4B11F0800F0CBF4FF4EB
:10779400001220221A61402211F0400F5A610CBFDE
:1077A4004FF4001020209E681A6118615A619D6888
:1077B4001A6115F0800518BF022511F0200F0CBFC7
:1077C4004FF40010202018615A619C681A6114F06B
:1077D400800418BF042411F0100F0CBF4FF40010E4
:1077E400202018615A61D3F808C01A611CF0800C7B
:1077F40018BF4FF0080C11F0080F0CBF4FF4001025
:10780400202018615A619868C6F3C01610F08000F1
:1078140018BF102011F0040F01900CBF4FF400109A
:1078240020201A6118615A619F681A6117F0800755
:1078340018BF202711F0020F0CBF4FF400102020B6
:1078440018615A6198681A6110F0800018BF1046D8
:1078540011F0010F0CBF4FF40011202119615A617E
:10786400996821F07F0141EA06062E4346EA0404A2
:10787400019944EA0C0C4CEA010C4CEA070747EA6C
:107884000000C0B21A6113E00D4B99811A8802F40A
:10789400827222B11A8912F0800FFBD103E01A8997
:1078A40012F0010FFBD0988980B201E06FF0020062
:1078B400FEBD00BF00300140594E0020000C0140C5
:1078C4000038004030B5002387B0ADF804304FF4E1
:1078D4008273ADF806300023ADF808304FF400731E
:1078E400ADF80E300023ADF812300723ADF8143094
:1078F400072900F28380DFE801F009121923040D3F
:10790400141E0023ADF80630ADF80E300023ADF898
:107914000A3019E00023ADF80630ADF80E3000232C
:107924000FE00023ADF80630ADF80E300223ADF8B9
:107934000A30002308E00023ADF80630ADF80E301D
:107944000223ADF80A300123072AADF80C3052D8CF
:1079540001281ED005D3022818BF6FF001004FD1B3
:1079640035E0284C02F00702D200204601A9258800
:10797400ADF8102001F0C6FEBDF80630ADB2B3F587
:10798400827F36D12088454015F0030038D000208E
:1079940019E01D4B1D88ADB21AB102F00702013A7D
:1079A400D200194C01A92046ADF8102001F0AAFE1E
:1079B400BDF80630B3F5827F1BD12088454015F011
:1079C40003001DD00120FF21FFF71EFD11E0BDF8CB
:1079D400063083B10D4B197003290FD8DFE801F08D
:1079E400020206060A4B40225A6102E0084B40227A
:1079F4001A61002004E06FF0020001E06FF0030060
:107A040007B030BD0030014000380040594E00201E
:107A1400000C0140F0B504468FB04FF0FF30002C4D
:107A240040F0BB8003AD5E4F284602F015F80122FA
:107A340021463C602046FFF79FFC01210A46204670
:107A4400FFF79AFC03212046FFF780FB01214FF446
:107A5400805002F0C1F90120014602F0AFF951480B
:107A6400214602F006F8504B802603934D484FF40C
:107A7400805329460C930193049405940694079427
:107A8400089609940A940B940D9401F0BAFF4748A0
:107A9400214601F0EEFF4FF0100C44482946CDF882
:107AA40014C0CDF800C004940694089601F0A9FF10
:107AB40001213F4801F0B0FE012203213C4801F0BE
:107AC400C5FE05210C20FFF71DFB032106222046DD
:107AD400FFF7F8FE0120214602467C60FFF74CFCCC
:107AE400012002460146FFF747FC03210120FFF76E
:107AF4002DFB01214FF4804002F07CF90120014666
:107B040002F05CF92B48214601F0B3FF019B2A4A9D
:107B1400284829460C9303920494059406940794E8
:107B2400089609940A940B940D9401F06AFF234873
:107B3400214601F09EFFDDF800C020482946CDF81B
:107B440014C004940694089601F05BFF01211C48BC
:107B540001F062FE01220321194801F077FE05219C
:107B64000E20FFF7CFFA032106220120FFF7AAFE19
:107B7400012202202146BC60FFF7FEFB01210A46D8
:107B84000220FFF7F9FB03210220FFF7DFFA0220AE
:107B940003210622FFF796FE20460FB0F0BD00BF7A
:107BA4004C4E00201C0002400C30014030000240CA
:107BB40000300140440002400C38004058000240AC
:107BC40000380040F7B501281E460C461546089BB0
:107BD40036D030D3022818BF6FF001007CD1C2B177
:107BE400A1B1002707E0E15D02200093FFF70CFC40
:107BF400E855009B0137B742F5D315E00220FF2179
:107C04000093FFF701FC2855009B0134B442F5D3DF
:107C14000AE039B908E0615D02200093FFF7F4FB44
:107C2400009B0135B542F6D32C4A18469360002BCD
:107C340052D0984743E02A4A2A49DFF8ACC003E00F
:107C44002A4A2B49DFF8ACC05768CDF804C0002F8E
:107C540040D1DFF888C04CF82030DDF804C0BCF80F
:107C64000C00106820F0010CC2F800C01DB1D560F2
:107C74004CF0800C08E0DFF880C0FF258CF8005041
:107C8400C2F80CC020F0810C566008684CF0010C5E
:107C940020F001050D601CB1CC6045F0800005E0CA
:107CA400164CFF252570CC6020F081004E6040F01A
:107CB400010033B14CF0020CC2F800C0086000208F
:107CC4000AE02CF0020CC2F800C0086050680028DA
:107CD400FCD101E06FF00200FEBD00BF4C4E00205D
:107CE4001C000240300002400030014044000240C9
:107CF40058000240003800405A4E0020584E0020E0
:107D040008B5F02001F0C8FE024B1B6803B1984788
:107D140008BD00BF4C4E002008B54FF4704001F080
:107D2400BBFE024B5B6803B1984708BD4C4E002074
:107D3400F0B5044691B04FF0FF30002C7ED10FAE69
:107D4400304601F087FC0125182331464FF4805753
:107D54003B488DF83F308DF83E50ADF83C7001F053
:107D640020FC4FF4005331463548ADF83C3001F067
:107D740018FC48F2000331463148ADF83C3001F0BC
:107D840010FC402331462F48ADF83C300BAE01F0D7
:107D940008FC29464FF4804002F02CF8304601F0EC
:107DA40032FD4FF40073ADF832304AF644433146A5
:107DB4000D9325484FF40073ADF82C30ADF82E40E8
:107DC400ADF83040ADF8384001F0C9FC1E482946F2
:107DD40001F02FFD2946284601F0F0FF684601F026
:107DE4003BFE2146194801F044FE4FF4702001F097
:107DF40053FE174B154800931023029370330593D9
:107E04008033069303F5407307936946A3F57873AB
:107E14000893049409970A9401F0F3FD0B48062192
:107E24002A4601F030FE084802212A4601F00EFDE0
:107E34000F200521FFF766F96E46204611B0F0BD0C
:107E4400000C01400010014000380040580002407E
:107E54000C380040F8B50B4E05460C463046002160
:107E6400174601F006FE4FF4702001F015FE064B94
:107E740064001F603046F5600121746001F0F9FD73
:107E84000020F8BD580002405C4E002008B50C4BA1
:107E94001A6812F4802F06D04FF480225A60094BDE
:107EA40000201B689847064B1A6812F4003F06D05E
:107EB4004FF400325A60034B01201B68984708BDF9
:107EC400000002405C4E002010B9034B188001E012
:107ED4004FF0FF30704700BF604E002037B501AD52
:107EE4000446284601F0B6FB10238DF8073003231F
:107EF40014F0010F8DF8063006D0042306482946F5
:107F0400ADF8043001F04DFB34F001040CBF204601
:107F14006FF001003EBD00BF0014014010F0010FDE
:107F240007D011F0010F064B0CBF4FF4802204223E
:107F34001A6130F0010018BF6FF00100704700BFF4
:107F440000140140024BD868C0F38000704700BFA2
:107F5400001401400B2837B504460D4688BF4FF086
:107F6400FF303AD81D4B41B9012212FA04F41A88A1
:107F7400084622EA04041C802FE00122A24019884A
:107F840001A80A431A8001F065FB03238DF806302B
:107F9400134B013D03EBC4039B88ADF80430052D5E
:107FA40019D8DFE805F0030507090B0D002308E0E5
:107FB400042306E0282304E0482302E0102300E021
:107FC40014238DF80730064B01A953F8340001F04F
:107FD400E8FA002001E06FF001003EBD604E002091
:107FE400E4D500080B2888BF4FF0FF3018D80D4B9C
:107FF4001B88034113F0010F08BF6FF001000FD07D
:10800400094BC20031B153F830109B189B880020F3
:108014000B6105E053F830009B189B8843610846C8
:10802400704700BF604E0020E4D500084FF0FF30D9
:1080340070474FF0FF3070474FF0FF3070474FF0FC
:10804400FF3070474FF0FF30704700000128F7B54C
:10805400064688BF4FF0FF3054D801AD284601F0E2
:10806400F9FA294C29482A4A4FF480734FF40077CF
:108074004FF480214361676111614FF40002226172
:10808400A2F58002226110228DF8072029460222DF
:108094008DF80620ADF8043001F083FA2046294615
:1080A400ADF8047001F07DFA16B114238DF8073091
:1080B40002AC4FF4807324F8043D1348214601F0C8
:1080C40070FA802310482146ADF8043001F069FAB3
:1080D40040230D482146ADF8043001F062FA042330
:1080E4000B482146ADF8043001F05BFA48238DF8C3
:1080F400073005484FF480532146ADF8043001F0B1
:1081040050FA0020FEBD00BF0010014000080140ED
:10811400000C01402D4910F0800F0CBF4FF080730C
:108124004FF480730B614FF48072294B10F0400FB1
:108134000CBF4FF0807C944610F0200F5A611A61F6
:10814400C1F810C00CBF4FF0807C944610F0100FA3
:108154005A611A61C1F810C00CBF4FF0807C94467C
:1081640010F0080F5A611A61C1F810C00CBF4FF02B
:10817400807C944610F0040F5A611A61C1F810C053
:108184000CBF4FF0807C944610F0020F5A611A61C4
:10819400C1F810C00CBF4FF0807C944610F0010F62
:1081A4000CBF4FF0807010465A611A61C1F810C0BC
:1081B4005A611A6108615A611A614FF400730B61C4
:1081C40000200B610B614B61704700BF0010014040
:1081D400000801402C4910F0800F0CBF4FF480239D
:1081E40004230B618022294B10F0400F0CBF4FF485
:1081F400802C4FF0040C10F0200F5A611A61C1F862
:1082040010C00CBF4FF4802C4FF0040C10F0100F72
:108214005A611A61C1F810C00CBF4FF4802C4FF0A2
:10822400040C10F0080F5A611A61C1F810C00CBF99
:108234004FF4802C4FF0040C10F0040F5A611A61B3
:10824400C1F810C00CBF4FF4802C4FF0040C10F098
:10825400020F5A611A61C1F810C00CBF4FF4802C90
:108264004FF0040C10F0010F0CBF4FF480200420D9
:108274005A611A61C1F810C05A611A6108615A61E1
:1082840000201A61704700BF000C0140001001403B
:10829400044B00280CBF4FF080704FF480701861BD
:1082A4000020704700100140044B00280CBF4FF41D
:1082B4008020042018610020704700BF000C01409A
:1082C40028B1012818BF4FF0FF3010D107E0084B48
:1082D40000290CBF4FF400018021196107E0044B11
:1082E40000290CBF4FF48001402119610020704720
:1082F40000100140024B9868C0F30030704700BF83
:108304000010014000207047F7B5194B194E4FF08B
:10831400807204271A610C46376101210546FFF774
:10832400CFFF0028B8BF4FF0FF301FDB13E001215F
:108334002846FFF7C5FF0A21042311F1FF313361F9
:10834400FAD10191FFF7D6FF019907462846FFF7B6
:10835400B7FF17B1013C002CE9D1064B4FF4802242
:10836400002C1A6114BF00206FF00100FEBD00BF95
:1083740000100140000C014008B54FF0804001217D
:1083840001F01EFC38B14FF08040012101F024FCC3
:10839400014B1B68984708BD644E002008B5064889
:1083A400012101F00DFC30B10348012101F014FC5E
:1083B400024B5B68984708BD00040040644E0020EF
:1083C40008B50648012101F0FBFB30B10348012147
:1083D40001F002FC024B9B68984708BD000C00406A
:1083E400644E002030B5012185B00446102001F010
:1083F40001FD4FF0FF33ADF8083048235C430C4DCA
:10840400013CADF804402846002401A9ADF80A4017
:10841400ADF8064001F04CFB01210A46284601F064
:10842400C4FB2846012101F0B3FB204605B030BD52
:10843400001000400348012108B5818401F0CCFB01
:10844400002008BD00100040064810B50121848CAE
:1084540001F0B6FBA4B200280CBF20464FF0FF3059
:1084640010BD00BF001000401FB504464FF0FF30A0
:10847400C4B94FF40060012101F0AEFC4FF0FF33AA
:10848400ADF808300848472301A9ADF80430ADF829
:108494000A40ADF8064001F00BFB0348012101F04E
:1084A40077FB204604B010BD002C0140044B9A8C8D
:1084B40092B2998C891A89B28142FAD90020704704
:1084C400002C01404FF0FF3070474FF0FF307047F1
:1084D400014B04221A607047704E002070477047A9
:1084E400022070470220704721B901288CBF022066
:1084F400002000E00220704708B5054B1B689B7AFA
:108504002BB1012000F0BAFA024B05221A6008BD13
:10851400A47F0020704E002070B5C4B04F490C22D7
:1085240004463DA804F0A8FB42A84D49072204F0E4
:10853400A3FB4C4B1B68DB78032B00F28C80DFE839
:1085440003F00E06025F48490122002329E00DF1E1
:10855400F3010DF1060202234FF0000C0BE001AA17
:10856400092393700423D37069E0023302F8020CE8
:1085740002F801CC9BB211F8010F0232051E18BF9C
:108584000125C72B8CBF002505F00105002DECD17A
:1085940055E0A0F12002D2B25F2A8CBF0022012252
:1085A40001331F2BCCBF002002F001001FFA83FC13
:1085B40020B111F8010F0028EBD10122BCF1000F0A
:1085C4000CBF002202F0010242A902B12749022392
:1085D40001AA4FF0000C06E0D054581C80B20233BC
:1085E40002F800C09BB211F8010B051E18BF01254B
:1085F400C72B8CBF002505F00105002DECD11EE032
:1086040033AD2846FEF77EFC002824DB013D0DF146
:1086140006020223002005E0023302F8021C02F8DD
:10862400010C9BB215F8011F02320E1E18BF012661
:10863400C72B8CBF002606F00106002EECD101AA40
:10864400032151701370204640A94092ADF80431C3
:1086540001F0C6FE00E0002044B070BDACD60008B6
:10866400ACD40008A47F0020DF3F0008E03F0008EE
:1086740007B5054902466B4603C983E80300104663
:10868400694601F0ADFE0EBDB8D6000807B5054930
:1086940002466B4603C983E803001046694601F0AD
:1086A4009FFE0EBDC0D6000838B5294B00241B68B8
:1086B40080259C725D72DC72204602F025FA204609
:1086C4004FF4007102F02AFA1021204602F03EFA1B
:1086D4004021204602F0C2FA2946204602F0AEFAB2
:1086E400204602F073FA1B4B20461B6893F82C10AB
:1086F40002F0EEFA204602F057FA0120214602F079
:108704000DFA0220214602F009FA0120C02102F0EC
:1087140095FA0120402102F0CDFA0120202102F037
:1087240015FA02204FF4807102F098FA40210220D9
:1087340002F0CEFA022002F037FA204602F0A8F83E
:10874400204600F09BF9044B01221A6038BD00BF9B
:10875400A47F00209C7F0020704E00200D4B10B59C
:108764001C68A4B214F4806F06D04FF6FF321A606E
:10877400094B1B685B68984714F4007F1EBF054BC8
:108784004FF6FF521A6014F4004F01D002F0DAF8E9
:1087940010BD00BF445C00409C7F002008B5002051
:1087A40002F0CBF9003818BF012008BD73B50446A8
:1087B40001A800F04FFF022C88BF4FF0FF3077D89C
:1087C400FEF778FC3B4B00221A60FEF789FC022C72
:1087D40013D0394A394B1A60394B05221A700122D9
:1087E4005A70384A384B1A60384A394B1A60394A39
:1087F400394B1A60394A3A4B5A60304D002000F028
:108804003DF92B68022600221E729A729CB9FFF76A
:10881400C5FF80B10120202102F098F9304602F012
:10882400C3F92B6880225A7201229A72284B1B6862
:108834005B6898472DE01F4A032313604FF480526E
:10884400ADF8042001A9102226488DF807208DF8E0
:10885400063000F0A6FE244B22494FF4805213F157
:10886400FF334A61FBD1134A022111601D4A0A20D9
:1088740010F1FF305361FBD10E4B186004331860C4
:1088840001F02AFA01214FF4000001F0B3FA022C9E
:1088940006D0164B00221A6002F50442043B1A600B
:1088A400134B00241C6014200821FEF72BFC2046E7
:1088B4007CBD00BF405C0040744E0020A47F0020BB
:1088C400A87F00207CD600089C7F002044D60008A6
:1088D400A07F0020F58B000828000020098C0008E8
:1088E4004400002000080140400D0300445C0040A7
:1088F400704E0020F7B5FEF7DDFB234B1B78002BF1
:108904003FD0022002F004FAC0F38F05002D38D0C6
:108914001E4B29B21A8892B2C2F14002914230DA57
:108924001B4E1C4C1C4A36F8081C36F8047C019279
:1089340041EA0747C7F30310103039460093FDF7A7
:1089440043FE019A009B80B9218889B242F82170C4
:108954002188013189B22180218889B23F2988BFC9
:1089640020801988013189B21980013DADB229B244
:1089740008360029D7DC044B00221A70022002F0CA
:1089840013F9FEF7ADFBFEBD98500020904E002079
:10899400086200409C500020984F002010B5FEF75C
:1089A40089FB2C4B1B78002B50D12B4B1A8892B28D
:1089B400002A4BD0294A1278002A47D01A8892B24A
:1089C400102A98BF1C88234B94BFA4B21024A4B2CD
:1089D4000120A100187089B202F06CF91E4B2049E5
:1089E4001A88121B92B21A80013C1E4BA4B2E318DF
:1089F400D8001D4A1D4BB3F800C01FFA8CFC31F897
:108A04002CC042F808CCB3F800C01FFA8CFC51F813
:108A14002CC04FEA1C4C42F804CCB3F800C00CF153
:108A2400010C1FFA8CFCA3F800C0B3F800C01FFAB5
:108A34008CFCBCF13F0F84BF4FF0000CA3F800C0C6
:108A440008328242D7D1012002F09CF8FEF748FB9D
:108A540010BD00BF944F00209E500020A250002063
:108A6400944E0020320C000888610040A050002081
:108A7400002814BF4FF0FF3000207047104A002335
:108A8400138011880F4A89B2118011880E4A89B265
:108A940011800E4A13700E4A138011880D4A89B250
:108AA400118011880C4A89B211800C490C4A10B10A
:108AB4000120087001E00B7001231370002070473F
:108AC400904E00209C500020924E00209850002090
:108AD4009E500020A4500020A0500020A25000204E
:108AE400944F002038B5174D04462B784FF0FF30D3
:108AF4003BB3154B1B889BB23E2B09D9FFF74EFFA6
:108B04002B78002B14BF6FF001004FF0FF3018E0FA
:108B1400FEF7D0FA0D4B0E491A8892B241F8224062
:108B2400013292B21A801A8892B23F2A01D90022E5
:108B34001A80054B1A88013292B21A80FEF7D0FAD5
:108B4400002038BDA25000209E500020A4500020D8
:108B5400944E002070B506460A4C42F20F7504E0AC
:108B64002388AB420CD8013323803046FFF7BAFF89
:108B740010F1020FF4D0002802DB024B00221A800D
:108B840070BD00BF9A500020124B10B51B880446DC
:108B94009BB24FF0FF30DBB1FEF78CFA0E4B0F4A5D
:108BA400198889B252F8212022601A88013292B2BF
:108BB4001A801A8892B23F2A01D900221A80054CE1
:108BC4002388013B9BB22380FEF78AFA208880B277
:108BD40010BD00BF904E0020924E0020984F002000
:108BE40008B5FFF787FEFFF7D9FE002008BD000097
:108BF40008B5034B00221A70FFF7D0FE08BD00BF72
:108C0400944F002008B5034B01221A70FFF772FE3F
:108C140008BD00BF9850002030B50128044685B037
:108C24000D4688BF4FF0FF301AD84FF0000304A957
:108C3400ADF80430ADF80630ADF80830ADF80C30BE
:108C440041F8105D4FF00C0314BF0648064869460E
:108C5400ADF80A3000F006FE044B002043F824501F
:108C640005B030BD0038014000480040BC51002030
:108C740073B504464FF0FF30002C40F0868001AD00
:108C84000121424800F0EEFC284600F0E3FC0223F8
:108C940029468DF806301C264FF400733C48ADF885
:108CA40004308DF8076000F07CFC4FF480632946A3
:108CB4003848ADF804308DF8076000F072FC4823A2
:108CC40029468DF8073032484FF48063ADF80430FC
:108CD40000F067FC4FF4006329462E48ADF80430D9
:108CE40000F05FFC4FF48040012101F075F84FF46F
:108CF400C020012101F07EF847F612212046FFF73B
:108D04008BFF47F612210120FFF786FF042125205F
:108D1400FEF7F8F90122204840F2255100F00BFE3D
:108D240004212720FEF7EEF91C4840F225510122C8
:108D340000F001FE1A481B4904700378DFF868E06C
:108D44000B700B78194A8EF80030147092F800C03A
:108D5400174B83F800C01D78DFF858C08CF800501A
:108D640044704078487049780B488EF8011054706C
:108D7400527801215A705B788CF8013000F0CEFDF6
:108D84000648012100F0CAFD20467CBD10001400F5
:108D94000008014000100140003801400048004034
:108DA400AC500020B4510020B0500020B851002035
:108DB400C4510020A8500020012838B5044688BFBB
:108DC4004FF0FF301DD80F4B6FF001001B5DC3B196
:108DD400FEF770F90C4B0D491A5D02EB84128D5CA1
:108DE4001A5D0132D2B21A551A5D3F2A01D9002206
:108DF4001A55044B1A5D013AD2B21A55FEF770F9AE
:108E0400284638BDAC500020B0500020345100201A
:108E1400012838B504460D4688BF4FF0FF301FD8EF
:108E2400104B1B5D3F2B88BF6FF0010018D8FEF775
:108E340041F90D4B0D491A5D02EB84128D541A5DF4
:108E44000132D2B21A551A5D3F2A01D900221A55AD
:108E5400044B1A5D0132D2B21A55FEF741F90020D3
:108E640038BD00BFAC500020B45100203451002064
:108E7400012838B5044688BF4FF0FF301DD80F4B8A
:108E84006FF001001B5DC3B1FEF714F90C4B0D49E3
:108E94001A5D02EB84128D5C1A5D0132D2B21A554E
:108EA4001A5D3F2A01D900221A55044B1A5D013A72
:108EB400D2B21A55FEF714F9284638BDB85100202D
:108EC400A8500020B4500020F0B50128044687B013
:108ED4000D46174688BF4FF0FF3052D82A4E335DF7
:108EE400D3183F2BC8BF6FF001004ADCFEF7E2F84D
:108EF4000022264B2648274901973CE013F804C07A
:108F040015F8017BDFF890E00CEB841C0EF80C7074
:108F140013F804C00CF1010C5FFA8CFC03F804C0D4
:108F240013F804C0BCF13F0F84BF4FF0000C03F8EA
:108F340004C016F804C00CF1010C5FFA8CFC06F8AE
:108F440004C016F804C0BCF1010F12D1012C15BFE6
:108F5400B1F80CC0B0F80CC01FFA8CFC1FFA8CFCE2
:108F640015BF4CF0800C4CF0800CA1F80CC0A0F89C
:108F74000CC0013292B2019FBA42BFD3FEF7B0F8DF
:108F8400002007B0F0BD00BFB8510020C45100203C
:108F94000048004000380140B450002070B5054638
:108FA4000C461646284621463246FFF78DFF10F13F
:108FB400020FF7D070BD0000144B10B51A8812F0E0
:108FC400200F09D09C882020E4B22146FDF7F2FA54
:108FD40010B92146FFF71CFF0C4C238813F0800FB7
:108FE40013D00B4B1B7853B10020FFF741FF00282F
:108FF400A4BF80B2A08008DAFF23A38005E0A38980
:1090040023F080031B041B0CA38110BD0038014016
:10901400B8510020154B10B51A8812F0200F0AD051
:109024009C882120E4B22146FDF7C4FA18B9013026
:109034002146FFF7EDFE0D4C238813F0800F13D06B
:109044000B4B5B7853B10120FFF712FF0028A4BF3C
:1090540080B2A08008DAFF23A38005E0A38923F06F
:1090640080031B041B0CA38110BD00BF00480040FB
:10907400B85100200E4B10B51A8812F0200F0AD0F8
:109084009C882220E4B22146FDF794FA18B90230F4
:109094002146FFF7BDFE064A138813F0800F05D062
:1090A400938923F080031B041B0C938110BD00BF24
:1090B4000044004070B56A4C206800F096FCB0F59E
:1090C400403F054600F0CA80664B00EA0303002BCC
:1090D40033D0E368002B30D0206800F07BFC628A38
:1090E400238A92B29BB29A4206D2638AE2689BB206
:1090F400D05401339BB26382594B5A6912F0020F68
:109104003ED1598A1A8A89B292B2013A91420CDA52
:109114005A6912F0040F00F0A1805B8A9BB2012B04
:1091240040F09C80002840F099804D4C002120683C
:1091340000F036FC2068012111E04B4B05EA0303E3
:10914400A3B115F4802111D1454C258AADB2012D6E
:1091540040F08480206800F023FC2068294600F059
:1091640012FC636943F00203636177E03F4A05EA56
:109174000202002A3ED03A4B5A6912F0020F07D07D
:109184005A6918686FF300025A614FF4E0612FE0E6
:10919400598A1A8A89B292B291420BD29968186894
:1091A40029B15A8A92B2895C013292B25A8200F091
:1091B4000FFC53E05A6912F0080F04D1186801211A
:1091C40000F0E1FB03E01868012100F0CFFB244B21
:1091D4005A6942F002025A611A8A92B22AB959694A
:1091E400186862F30001596112E018684FF4806155
:1091F40000220FE01E4E1A4C05EA0606A6B163696A
:1092040013F0020F09D06369206862F300036361FD
:109214004FF4E06100F0D1FB20E02179206801F0F7
:10922400010200F0DAFB19E0324620684FF4E061F5
:1092340000F0C3FB0F4B31461D606FF00703A361C1
:109244006369206866F30003636100F0A9FB20688A
:1092540000F0C0FB2068012100F095FB70BD00BF49
:10926400C8510020400000100200001080000010CF
:1092740001000010AC7F002038B51C4D286800F0B8
:10928400B4FB1B4B044600EA030333B128681949B5
:1092940000F0B3FB6FF00503AB61174B04EA030363
:1092A4003BB1124D1549286800F0A7FB6FF0040389
:1092B400AB61134B04EA03035BB10C4C1149206806
:1092C40000F09BFB6FF00603A3612068012100F00E
:1092D4005AFB064C4FF4E0612068002200F06DFB5D
:1092E40063696FF30003636138BD00BFC851002098
:1092F4000001001000010001000200100002000142
:10930400000400100004000108B528B103681970B6
:1093140003680133036003E0C9B20120FDF7B0F92B
:1093240008BD002AF7B58C460446154610DD002218
:1093340000E001321CF802100029FAD1AA42ACBFA5
:109344000D46AD1A13F0020F0CBF2027302700E0A2
:10935400202713F001060DD109E020463946CDF847
:1093640004C0FFF7D1FFDDF804C00136013D002D34
:10937400F3DC00E00026634605E020460193FFF796
:10938400C3FF019B013613F8011B0029F5D105E049
:1093940020463946FFF7B8FF0136013D002DF7DCC2
:1093A4003046FEBDF0B587B004461D460C9E0D9BAD
:1093B400084651B930228DF80C208DF80D10204646
:1093C40003A93246FFF7ADFF43E00A2A14BF002188
:1093D4000121002D0CBF002501F001052DB100284D
:1093E40002DA4042012500E00025DDF838E006A954
:1093F4004FF0000C01F801CDAEF13A0E0DE0B0FBD8
:10940400F2FC02FB1C0CBCF1090FC8BFF4440CF1C4
:10941400300C01F801CDB0FBF2F00F460028EED17C
:109424008DB15EB113F0020F08D020462D210193B7
:10943400013EFFF769FF0125019B04E02D224F1E29
:1094440001F8012C0025204639463246FFF769FF12
:10945400401907B0F0BD0000F0B589B006460D46CE
:10946400059200247AE0252B72D115F8013F002BD8
:1094740077D0252B6CD02D2B02D10135012303E0AD
:10948400002301E043F002032F4615F8012B302A94
:10949400F8D0002202E00A2000FB02C239783D46DF
:1094A400A1F1300C5FFA8CF001370928F3D9732944
:1094B40009D10599081D059009682D48002908BFA0
:1094C4000146304641E064290ED105990193612398
:1094D40000920293081D096805900A223046012370
:1094E400FFF760FF241838E0782906D10599019325
:1094F400081D05900092612307E058290AD10599B7
:109504000193081D05900092412302933046096897
:1095140010220BE075290BD1059901936123009268
:109524000293081D096805900A2230460023D7E7F4
:10953400632912D10599081D096805908DF81C103E
:1095440000218DF81D10304607A9FFF7EAFEC9E790
:1095540029783046FFF7D8FE013401352B78002BEB
:1095640081D116B1336800221A70204609B0F0BDCB
:1095740030D700080EB40FB505AA52F8041B0190A9
:1095840001A80392FFF768FF04B05DF804EB03B091
:10959400704707B5034602A840F8043DFFF75CFF97
:1095A4000EBDCB78F7B513F0100F03F00F020F8840
:1095B4001CBF8B781A4317F0FF0F22D0D0F800C0DD
:1095C40000230197012414FA03F5019E05EA060419
:1095D400AC4211D19E000F2717FA06F512FA06F6CF
:1095E4002CEA050CCD784CEA060C282D08BF446102
:1095F40002D0482D08BF04610133082BE2D1C0F822
:1096040000C00F88FF2F24D9D0F804C00023019292
:10961400012203F1080512FA05F505EA0704AC4234
:1096240012D19E000E3212FA06F5019A2CEA050CAC
:1096340012FA06F6CD784CEA060C282D08BF4461D0
:1096440002D0482D08BF04610133082BE0D1C0F8D3
:1096540004C0FEBD4FF0FF33038002238370DB1888
:10966400C37070470028B4BF1A4B1A4B00F4401C57
:10967400B4BFDB695B68BCF5401F10B582B20AD188
:10968400DFF850C023F07063DCF8044024F0706409
:10969400CCF8044012E010F4801F02BF4FEA505C83
:1096A4004FEA0C1C02FA0CFC04D0C0F3034C032454
:1096B40004FA0CFC23EA0C0343F0706319B1410D66
:1096C40009018A4013430028B5BF024A014AD36105
:1096D400536010BD00000140034B1A6802F03802C9
:1096E40010431860704700BF00200240044B1A6802
:1096F40022F010021A601A6810431860704700BF05
:1097040000200240B1F802C00B8802884CEA03032F
:10971400B1F804C002F4415243EA0C03B1F806C0A4
:1097240043EA0C03B1F808C043EA0C03B1F80AC0D9
:1097340043EA0C03B1F80CC043EA0C03B1F80EC0C1
:1097440043EA0C0342EA03039BB20380838B23F4B2
:1097540000631B041B0C83830B8A03827047838B77
:10976400F0B523F47A6323F01F031B041B0C8383DB
:10977400022303848B68868B022B87B004460D4634
:10978400B6B224D001A88F8800F0C4FAEA88002F6A
:1097940014BF02270127B2F5007F019BAA6803D1F9
:1097A4001B0A0A214B4304E07F01B3FBF7F30A27AA
:1097B4007B43B3FBF2F305330A229BB2B3FBF2F310
:1097C40003F001021202C3F34F0392B200E000223D
:1097D400991E89B2FE2928BF002228BF0223E988E6
:1097E40013430B439BB223842B886A8846EA030302
:1097F40043F400631343AA881343AA8913439BB217
:10980400A38307B0F0BD002302220380438083803A
:10981400C38082608381704721B103889BB243F087
:10982400400304E0038823F040031B041B0C038063
:10983400704721B1838B9BB243F4806304E0838B34
:1098440023F480631B041B0C838370471AB1838841
:109854009BB2194303E083889BB223EA0101818010
:1098640070470000038ACA8823F440531B041B0C6E
:10987400134330B503820D4683890989AA8823F4EA
:10988400B05341EA0202698923F00C030A431B0422
:109894001B0C92B242EA03038381838AAA8923F4CC
:1098A40040731B041B0C134387B00446838201A836
:1098B40000F030FA184BA2899C4212B20CBF049BF0
:1098C400039B002A2A6803DA19215943520002E053
:1098D4001921594392006423B1FBF2F1B1FBF3F275
:1098E4001201100903FB1011A08900B2002806DA46
:1098F400C9003231B1FBF3F303F0070305E00901BA
:109904003231B1FBF3F303F00F0343EA020292B2E4
:10991400228107B030BD00BF0038014021B18389E6
:109924009BB243F4005304E0838923F400531B04E3
:109934001B0C83817047C1F342134FF0010C01F0FB
:109944001F0163450CFA01F101D10C3004E0022B34
:1099540001D1103000E014301AB1036843EA010168
:1099640002E0036823EA01010160704721B1038822
:109974009BB243F4807304E0038823F480731B04D4
:109984001B0C0380704721B103889BB243F400731E
:1099940004E0038823F400731B041B0C038070474A
:1099A40021B103889BB243F4806304E0038823F469
:1099B40080631B041B0C038070471AB183889BB21D
:1099C400194303E083889BB223EA01018180704735
:1099D40001827047008AC0B2704712B141F00101A0
:1099E40001E001F0FE0101827047838A008B9BB283
:1099F40043EA004020F07F407047C94389B2818226
:109A04007047D1F820C08B6802684CEA0303D1F890
:109A140010C022F4FE4243EA0C03D1F814C022F031
:109A2400F00243EA0C03D1F818C043EA0C03D1F85E
:109A34001CC043EA0C03D1F824C043EA0C03D1F858
:109A440028C043EA0C0313430360CB6843600B68EC
:109A540083604B68C3607047002303604360836086
:109A6400C360036143618361C361036243628362D0
:109A7400704719B1036843F0010302E0036823F05F
:109A840001030360704712B10368194302E00368DD
:109A940023EA01010160704710F0805F14BF024B9C
:109AA400024B5860704700BF0004024000000240AF
:109AB4002D4ADFF8B8C00388904214BF0022012267
:109AC400604508BF42F0010210B59BB2CAB9284CE8
:109AD400B0F1804F14BF4FF0000C4FF0010CA042C6
:109AE40014BF64464CF001045CB9224CDFF888C012
:109AF400A04214BF00240124604508BF44F00104BF
:109B04002CB1B1F802C023F0700343EA0C031B4CE0
:109B1400DFF86CC0041B18BF012460450CBF00248F
:109B240004F0010434B123F44073B1F806C09BB2CD
:109B340043EA0C0303808B8883850B8803856AB909
:109B4400104B114A984214BF00230123904208BFCE
:109B540043F0010313B90D4B984201D10B7A0386EC
:109B64000123838210BD00BF002C0140003401405A
:109B74000004004000080040000C004000100040B9
:109B840000140040004001400044014000480140EE
:109B940021B103889BB243F0010304E0038823F05E
:109BA40001031B041B0C038070471AB183899BB209
:109BB400194303E083899BB223EA01018181704741
:109BC400038A828911420CBF0020012019420CBF74
:109BD400002000F001007047C94389B20182704738
:109BE4000D4B1A6842F001021A6059680B4A01EAE7
:109BF40002025A601A6822F0847222F480321A60D7
:109C04001A6822F480221A605A6822F4FE025A600A
:109C14004FF41F029A607047001002400000FFF8E2
:109C24000C4BB0F5803F1A6822F480321A601A682F
:109C340022F480221A6003D0B0F5802F08D103E00B
:109C44001A6842F4803202E01A6842F4A0221A60D0
:109C5400704700BF00100240034B5A6822F47C1284
:109C6400104308435860704700100240014B1860CD
:109C7400704700BF60004242034B5A6822F003025F
:109C840010435860704700BF00100240024B5868F0
:109C940000F00C00704700BF00100240034B5A68EC
:109CA40022F0F00210435860704700BF00100240D9
:109CB400034B5A6822F4E06210435860704700BFB7
:109CC40000100240034B5A6822F4605242EAC0007A
:109CD4005860704700100240014B1860704700BF85
:109CE400D8004242034B5A6822F440421043586061
:109CF400704700BF00100240024B1A6A10431862FA
:109D0400704700BF00100240014B1860704700BF4D
:109D14003C044242224B5A6802F00C02042A02D04C
:109D2400082A15D101E01F4B13E05A685968C2F3A1
:109D34008342023211F4803F08BF1B4B05D05B689D
:109D440013F4003F14BF194B164B5A43026001E051
:109D5400174B0360124B17495A68D0F800C0C2F37E
:109D640003128A5C2CFA02F24260D3F804C0CCF3EA
:109D7400022C11F80CC022FA0CFCC0F808C0D3F86D
:109D840004C0CCF3C22C11F80C10CA40C2605B684A
:109D94000949C3F38133CB5CB2FBF3F20261704730
:109DA40000100240001BB70000093D00808D5B00DD
:109DB40000127A00640000206000002019B1054BF5
:109DC4005A69104303E0034B5A6922EA00005861C0
:109DD400704700BF0010024019B1054B9A69104347
:109DE40003E0034B9A6922EA00009861704700BFC0
:109DF4000010024019B1054BDA69104303E0034B2C
:109E0400DA6922EA0000D861704700BF00100240FE
:109E140019B1054BDA68104303E0034BDA6822EA10
:109E24000000D860704700BF0010024019B1054B14
:109E34001A69104303E0034B1A6922EA000018610F
:109E4400704700BF00100240014B1860704700BF0C
:109E5400400442424309012B04BF084B1B6805D050
:109E6400022B0BBF054B054B1B6A5B6A00F01F00FE
:109E740033FA00F000F00100704700BF0010024008
:109E840007B5002301933120FFF7E4FF019B013361
:109E94000193019BB3F5A06F01D00028F3D03120CA
:109EA400FFF7D8FF003818BF01200EBD21B1064BC3
:109EB4001A8892B2104304E0034B1A8892B222EA41
:109EC40000001880704700BF00280040034B9A88A8
:109ED40092B242F010029A80704700BF00280040FE
:109EE400034A938823F010031B041B0C93807047D0
:109EF4000028004010B50446FFF7E8FF034B220C8E
:109F0400A4B21A839C83FFF7EBFF10BD0028004026
:109F140010B50446FFF7DAFF044BC4F30342A4B2BE
:109F24001A819C81FFF7DCFF10BD00BF00280040B0
:109F3400024B9A8812F0200FFBD070470028004093
:109F4400054A938823F008031B041B0C9380938811
:109F540013F0080FFBD0704700280040012008B51B
:109F6400FFF772FF0020FFF76FFF08BD014B186079
:109F7400704700BF20000E4240F0BE60024B40F428
:109F84002020D860704700BF00ED00E021F0604160
:109F940021F07F01024B41EA00009860704700BF46
:109FA40000ED00E004280BBF054B054B1A681A6846
:109FB4000CBF42F0040222F004021A60704700BF92
:109FC40010E000E010B5064C18B9236801221A828B
:109FD40005E0044B1B681B68984720680A3010BDD5
:109FE400A47F0020A07F002010B5064C18B9236878
:109FF40001221A8205E0044B1B689B68984720687D
:10A004000C3010BDA47F0020A07F002008B5274B92
:10A0140018B91B6802221A8247E0254800221B68EF
:10A0240002801A7812F07F0215D15B7A027813F05D
:10A03400200F14BF42F0020222F0020213F0400F7C
:10A044001B4B027015BF1A781A7842F0010222F0F5
:10A0540001021A7022E0012A27D0022A24D15A7957
:10A0640002F00F0312F0800F4FEA830308D003F1CC
:10A07400804303F5B8431B6803F03003102B08E05A
:10A0840003F1804303F5B8431B6803F44053B3F56D
:10A09400805F02BF037843F001030370054B1B6824
:10A0A4001B699847024800E0002008BDA47F0020F7
:10A0B400B07F0020A07F0020F7B5274B1C68238ABF
:10A0C400267AD3F1010238BF0022042E14BF0026E1
:10A0D40002F00106AEB12149214A0B78012B0CD1C3
:10A0E400204B04271868204B80B2C3185B00002063
:10A0F40018603023138008702AE010231380072788
:10A1040026E0A58AAB428CBF022704279D4228BFC4
:10A114001D462846A369984703463046019300F03C
:10A12400ADFD019B2A460146184600F0C7FC2946AE
:10A13400304600F0BFFD238A30225B1B2382638AF2
:10A14400ED18074B65821A80084B4FF440521A8071
:10A15400014B1B681F72FEBDA47F0020EC51002040
:10A16400B47F0020505C004002300020B27F002009
:10A1740010B50A4B0A491B684978DA7891420AD328
:10A18400997841B99C8834B99A72064B1B685B680C
:10A194009847204600E0022010BD00BFA47F0020A5
:10A1A400A87F0020A07F002038B50E4A0E4C12680C
:10A1B40023685879D9789369984723689A7A7AB149
:10A1C40070B91A7962B99D7855B9084B1B68DB6878
:10A1D4009847236828465A79DA72DA781A7300E0C5
:10A1E400022038BD9C7F0020A47F0020A07F002097
:10A1F40010B53F4B1B68187810F07F0002BF5A7AE5
:10A2040022F020025A7272D002286FD15A88002A92
:10A214006DD11A79002A6AD15A79DFF8D8C022F0B0
:10A22400800012F0800F4FEA800415BF04F18044CF
:10A2340004F1804404F5B84404F5B84414BF21681B
:10A2440021689CF800C014BF01F0300101F44051B2
:10A25400604534BF4FF0000C4FF0010C002914BFCF
:10A2640061464CF00101002940D19B7A002B3DD07E
:10A2740012F0800F4FEA800411D004F1804404F5F9
:10A28400B844236803F03003102B29D1C4B220460C
:10A2940000F0C0FC2046302100F058FC20E004F11E
:10A2A400804404F5B844236803F44053B3F5805F55
:10A2B40016D130B9104B1B6893F82C1000F008FD30
:10A2C40002E0C0B200F092FC22684BF68F7302EAFF
:10A2D400030383F4405343F4004343F080032360B7
:10A2E400064B1B685B699847002000E0022010BD04
:10A2F400A47F0020A87F00209C7F0020A07F002056
:10A3040008B52B4BDFF8ACC018689CF800C0417945
:10A3140021F0800211F0800F4FEA820315BF03F190
:10A32400804303F1804303F5B84303F5B84315BFF5
:10A334001B681B6803F0300303F44053624535D2B5
:10A34400B0F802C0BCF1000C18BF4FF0010C002B98
:10A3540014BF63464CF0010343BB837A33B311F05B
:10A36400800F4FEA82030BD003F1804303F5B84317
:10A37400196848F6BF7201EA020282F010020AE08C
:10A3840003F1804303F5B84319684BF68F7201EA71
:10A39400020282F4805242F4004242F080021A60C7
:10A3A400054B1B689B699847002000E0022008BD0C
:10A3B400A47F0020A87F0020A07F002008B5064BC2
:10A3C4001B685A7A42F020025A72044B1B68DB69FC
:10A3D4009847002008BD00BFA47F0020A07F002074
:10A3E400054B1A68538A18B98988CB1A138201E07D
:10A3F4000868C018704700BFA47F002070B580248F
:10A40400A2B0064608496846224602F035FC3046AA
:10A414000DEB04016D46CDF880D0ADF88440FFF714
:10A42400DFFF22B070BD00BF38D7000808B50C4B61
:10A4340000201B6893F82C1000F04AFC094B1B68A1
:10A44400187A082806D1084B4FF480521A80074B1B
:10A4540010221A80092814BF0020012008BD00BF63
:10A464009C7F0020A47F0020B27F0020B47F0020C6
:10A47400F8B5384B1C68237A022B14BF002601263A
:10A48400042B08BF46F00106002E5BD1032B14BF3A
:10A4940000220122052B08BF42F00102002A4BD002
:10A4A400A369228A191E18BF0121002A0CBF0021AA
:10A4B40001F00101A1B1A58A954228BF154628469D
:10A4C4009847238A07465B1B2382638A3046EB182E
:10A4D400638200F0E1FB2A460146384600F004FBA3
:10A4E400238A53B11C4B4FF4405200201A8001467A
:10A4F40000F0E0FB194B30221A80238AA28A9A4288
:10A5040003D8144B03221B6803E0124A1BB11368DF
:10A5140005221A720CE0126806211172104A1168A1
:10A52400104A89B28A18520013600C4B30221A80E8
:10A53400084B1B681B7A06E0072B03D10A4B1B68E8
:10A54400DB6898470823034A12681372FFF76EFF0B
:10A55400F8BD00BFA47F0020B27F0020B47F00209C
:10A56400505C0040023000209C7F0020BB4BF7B5BC
:10A574001A68BB4EBB4B92B2D31835685B001F6898
:10A584002B7A092B1AD0BFB207F1005707F54057B1
:10A594007F003C4614F8013B2B707B780A376B70C4
:10A5A400B4F8030000F0C4FB6880B4F80700356811
:10A5B40000F0BEFBA88033687F88DF80A84C0122AE
:10A5C40023681A72DA885D78002A61D11A7812F049
:10A5D4007F022ED1092D02D1FFF7CAFD3BE0052DE4
:10A5E4000DD193F90320002A4DDB9A78002A4AD131
:10A5F4009A88002A47D19B7A002B35D043E0032D5B
:10A604000BD1DA78012A27D19A882ABB5B7A13F016
:10A61400200F21D0FFF7D2FE1DE0012D1CD1DA78E6
:10A62400012A19D19A88BAB95B7A13F0200F13D092
:10A634000AE0012A04D10B2D0ED1FFF7B5FD0AE083
:10A64400022A09D1012D02D1FFF7D2FD03E0032D27
:10A6540002D1FFF755FE38B1834B28461B685B696E
:10A66400984703280DD070B97C4B30211A687F4B72
:10A6740092B2D3185B0000221A607D4B1980062326
:10A6840002E0092300E00823754A12681372E1E02E
:10A69400062D18D11A7812F07F0F40F095809B7820
:10A6A400012B03D1704B1B68DB6984E0022B03D1BF
:10A6B4006D4B1B681B6A7EE0032B40F085806A4B60
:10A6C4001B685B6A77E0002D48D1598800297BD14B
:10A6D4005A6822F47F42B2F5003F75D11A7812F01D
:10A6E4007F0203D19B88002B63D06DE0012A09D13E
:10A6F4005D4A5879126893699847002864D12368A1
:10A704009B7A28E0022A5FD15B795A4803F00F0252
:10A7140013F0800F03F070014FEA820315BF03F1B9
:10A72400804303F1804303F5B84303F5B84314BFF2
:10A734001B681B68007814BF03F0300303F4405314
:10A7440082422CBF00220122002914BF002202F001
:10A754000102002A38D0002B2BD135E0082D06D178
:10A764001B7813F07F0F08BF434B25D02CE00A2D34
:10A7740016D11A7802F07F02012A25D19A7A1AB3E7
:10A78400598809BB5A6822F47F42B2F5803F1BD135
:10A79400354A5879126893699847384B60B113E089
:10A7A400552D11D15B887BB9802A08BF344B0BD15E
:10A7B40002E0344B00E03BB12268002151829361F6
:10A7C4000020984700200AE0274B22681B68507835
:10A7D4001B699847032804BF214B1B6806D0204BF4
:10A7E4004FF6FF711B681A8A8A4201D1092203E0DD
:10A7F400022800D012B908221A722BE093F9001033
:10A80400002921DAD98801910198824284BF019AF2
:10A814001A8211D88A420FD21349096891F82C1070
:10A824008A4201D2002105E092FBF1F001FB1022E3
:10A8340012B90121144A11700B4A126892F82C20A3
:10A844009A82FFF739FC05E003221A720F4B4FF48A
:10A8540040521A80FFF7EAFDFEBD00BF505C004085
:10A86400A47F0020043000209C7F002002300020C0
:10A87400B47F0020A87F0020C99F0008ED9F000836
:10A8840001A4000811A00008EC510020B27F0020B0
:10A8940030B50F4B93F800C0002312E0DAB29100F8
:10A8A40001F1804101F5B8410D6842F4004242F0E3
:10A8B400800440F60F7205EA020244EA02020A60CA
:10A8C40001336345EAD3034B40F08000186030BD88
:10A8D400A87F00204C5C004010B5164C23681A7AFF
:10A8E400022A14BF00210121042A08BF41F00101FA
:10A8F40021B1FFF7E1FB23681B7A14E0062A11D18A
:10A904005A78052A0AD11A7812F07F0F06D1D8781E
:10A91400FFF7BEFF084B1B681B6A9847074B1B6871
:10A924009B6898470823034A12681372FFF77EFD59
:10A9340010BD00BFA47F0020A07F00209C7F0020CA
:10A9440070470000F7B50022ADF80620544F554E6D
:10A954009DE013F00F0571D13A6813F0100F92B215
:10A9640032803188504A01F03001118032884C4CD9
:10A9740002F44052328039684BF6BF7201EA020297
:10A9840082F4005282F0200242F4004242F080023B
:10A99400444D3A6008D1226848F60F7302EA030373
:10A9A4002360FFF799FF1EE03B689BB2ADF80630C9
:10A9B400BDF8063013F4006F08D0226840F68F7398
:10A9C40002EA03032360FFF7D1FD0CE0BDF8063073
:10A9D4001BB2002B5BDA226840F68F7302EA030392
:10A9E4002360FFF745FD22684BF6BF7302EA0303B9
:10A9F4002A8802F4805292B20AB183F48053294A1D
:10AA0400128802F4005292B20AB183F40053264A27
:10AA1400128802F0100292B20AB183F01003224AA3
:10AA2400128802F0200292B20AB183F020031F4A76
:10AA340043EA02021A4B92B21A602FE0AC0004F10E
:10AA4400804404F5B84423689BB2ADF80630BDF8E1
:10AA540006301BB2002B0ADA226840F68F7302EA32
:10AA64000303134A23606B1E52F823309847BDF842
:10AA7400063013F0800F0AD0226848F60F7302EAFA
:10AA840003030C4A013D236052F8253098470A4AD3
:10AA940013689BB213F4004F7FF45BAFFEBD00BF9D
:10AAA400005C0040B27F0020B47F00208080FFFF64
:10AAB4004400002028000020445C004001F10051C3
:10AAC400013201F540514900520808E010F801CC68
:10AAD40010F8023C013A43EA0C2321F8043C02300A
:10AAE4000431002AF2D1704701F10051013201F51D
:10AAF40040514900520804E051F8043B013A20F85F
:10AB0400023B002AF8D170474FF6F873024A00EA74
:10AB140003031360704700BF505C0040800000F1E5
:10AB2400804000F5B840036823F4EC4323F070033D
:10AB340043EA010189B201607047800000F180405E
:10AB440000F5B840006800F4C0607047800000F170
:10AB5400804000F5B840026848F6BF7302EA030378
:10AB640001F0100292B20AB183F0100301F0200147
:10AB740089B209B183F0200343F4004343F0800316
:10AB840003607047800000F1804000F5B84002681F
:10AB940048F6BF7302EA030383F0300343F400432F
:10ABA40043F0800303607047800000F1804000F5AB
:10ABB400B84002684BF68F7302EA030383F44053F0
:10ABC40043F4004343F0800303607047800000F1C6
:10ABD400804000F5B840026840F60F6302EA0303C0
:10ABE40043F4004343F0800303607047800000F1A6
:10ABF400804000F5B840036813F4804F09D0026820
:10AC040040F60F7302EA030343F4404343F0800326
:10AC140003607047800000F1804000F5B84003688D
:10AC240013F0400F09D0026840F60F7302EA0303E1
:10AC340043F4004343F0C00303607047064B4908E4
:10AC44001B6849009BB203EBC00000F1005000F503
:10AC54004050400001607047505C0040054B49087B
:10AC64001B6849009BB203EBC000034BC3185B0095
:10AC740019607047505C004004300020054B1B688D
:10AC84009BB203EBC00303F1005303F540535B0095
:10AC940018887047505C0040044B1B689BB203EB60
:10ACA400C000034BC3185B0018887047505C004019
:10ACB40004300020044B1B689BB203EBC000034B21
:10ACC400C3185B0019607047505C004002300020DC
:10ACD4000D4B1A680D4B92B2D31803EBC000400021
:10ACE4003E2909D94B0911F01F0F01D1013B9BB239
:10ACF4009B0243F4004305E04B0811F0010F18BF19
:10AD040001339B0203607047505C00400630002012
:10AD1400054B1B689BB203EBC000044BC3185B00DC
:10AD240018688005800D7047505C00400630002094
:10AD3400C3B2000A40EA03207047000070B51D4BFF
:10AD440001461878012802D8FDF7BAFA30E01A4A09
:10AD5400937852785343023B48BF6FF0010027D4E5
:10AD6400042B02DC0238C0B21FE03E2BA8BF3E23F6
:10AD7400DC1013F0070F18BF01340238C6100D465B
:10AD840059B100F0070001258540EDB205E0B44259
:10AD94000CBF28460020FDF755F9013CF7D20021ED
:10ADA4000220FDF74CF902200121FDF748F90020AB
:10ADB40070BD00BFE44D0020887F0020174BF7B51D
:10ADC4001B78812B14BF0026012686F00107862BF1
:10ADD40014BF40233D2348B10824204601343146A2
:10ADE400E4B2FDF7FFF80C2CF7D114E00C4A082567
:10ADF4001288044692FBF3F3DBB29C4214BF39463B
:10AE040031462846013401930135FDF7EBF8042C53
:10AE1400EDB2019BF1D10020FEBD00BF887F002070
:10AE24009A7F002010B50824204601340521E4B29D
:10AE3400FDF790F80C2CF7D1002010BD38B51F4B4E
:10AE44001878012804D840F6C411FDF75DFA33E000
:10AE54003F282FD80020FDF71BFA0120FDF752FAF6
:10AE64000120FDF721FA0120FFF768FF002821DB0C
:10AE740040F6C4140120FFF761FF002501200135CD
:10AE8400FDF712FA0A2DF9D1FDF734FA0546002030
:10AE9400FFF754FF15B114F1FF34EBD10020FDF797
:10AEA40031FA0020FDF700FA002C14BF00206FF0E7
:10AEB400010001E04FF0FF3038BD00BFE44D002039
:10AEC40070B53B4B05469A785C783A4B5443083C42
:10AED400382CA8BF382400B31A78FF2A65D0FF2283
:10AEE40000201A70FDF716F9042C09DC002504E093
:10AEF400E8B20021FDF7A3F80135A542F8DB54E0E0
:10AF0400E31014F0070F18BF01331C4602E00020C1
:10AF1400FDF798F8013CFAD23FE0274A19781278F5
:10AF2400914242D001269640F6431A70F0B2FDF7E2
:10AF3400F1F8042C0DDC09E005F1080136FA01F101
:10AF4400E8B201F00101FDF77AF80135A542F3DB1F
:10AF54002BE0194BE210197814F0070F174B18BFA8
:10AF64000132083901EA03030826002B91FBF6F6A7
:10AF740003DA013B63F00703013301259D40ED43F0
:10AF8400EDB2541E06E0B4420CBF2846FF20FDF784
:10AF940059F8013CB4F1FF3FF5D100210220FDF73F
:10AFA4004EF802200121FDF74AF8002070BD00BFD1
:10AFB400887F002074000020E44D002007000080FA
:10AFC400F7B53F4B05461C78002C75D13D4B1E78D8
:10AFD4003D4B3246D3E9000101F012FE0122002369
:10AFE40002400B4052EA030166D0384B1A787F3294
:10AFF400D3B2052B3CD8012752B217FA02F212F051
:10B00400230306D112F0180424D112F0040F17D12F
:10B014002EE0012E50D82046FFF7D0FEFFF70EFF9A
:10B024003846FFF7CBFE2846FDF774F82046FDF7B7
:10B034002FF93846FFF782FE2046FFF77FFE3DE0FA
:10B044003846FFF73DFF2046FDF722F92846FDF775
:10B05400C1F833E038460193FFF732FF019B6FF0EC
:10B0640002041846FDF714F92846FDF7B3F825E065
:10B07400FFF7E4FE002811DA124B01201A780021B0
:10B0840001F0CAFD104CD4E9002322EA000023EAAF
:10B094000101C4E900016FF001040FE02846FDF747
:10B0A40039F80020FDF7F4F80120FFF747FE0020EF
:10B0B400FFF744FE002401E04FF0FF342046FEBDBC
:10B0C400ED510020E44D0020F0510020887F002045
:10B0D400F7B5744B04461D78002D40F0DD807248AE
:10B0E400724E90F800C0D6E900016246CDF804C063
:10B0F40001F086FD02460B460120002102400B4070
:10B1040052EA0301DDF804C000F0C680684F3A78C3
:10B114007F32D3B2052B00F29C80012352B213FA82
:10B1240002F212F0230306D112F0180571D112F0C5
:10B13400040F50D18DE0BCF1010F00F2AD805D4BE6
:10B14400BA881988914280F0A7805B4A1188FA88EE
:10B15400914280F0A18028460193FFF72FFEFFF76C
:10B164006DFE0028019B0EDA4F4800210278012071
:10B1740001F052FDD6E9002322EA000023EA01018E
:10B18400C6E9000178E020460193FCF7C3FF0120E3
:10B19400FDF77EF80120FFF7D1FD2846FFF7CEFD2D
:10B1A4003A78019B862A0DD11A88013292B21A800C
:10B1B4003D23B2FBF3F103FB11239BB2002B6ED1B1
:10B1C400002023E01A88013292B212F03F0F1A8055
:10B1D40065D140201AE02846FFF772FE0120FDF7F2
:10B1E40057F82046FCF7F6FF324A28461388013305
:10B1F4009BB21380BA88B3FBF2F402FB1434A4B2FA
:10B20400002C4DD11020FFF7DBFE2046FFF7D8FEBF
:10B2140046E018460193FFF753FE0120FDF738F886
:10B224002046FCF7D7FF2349019B0A8818460132C0
:10B2340092B20A80B988B2FBF1F401FB1424A4B2DF
:10B2440074BB2046FFF7BCFE1020FFF7B9FE204672
:10B2540026E0FFF7F3FD002811DA134B01201A78DA
:10B26400002101F0D9FC114CD4E9002322EA0000AA
:10B2740023EA0101C4E900016FF0010010E0204657
:10B28400FCF748FF0120FDF703F80120FFF756FD06
:10B294000020FFF753FD02E04FF0FF3000E00020F4
:10B2A400FEBD00BFED510020E44D0020F051002010
:10B2B400887F00209A7F0020847F0020F0B5DE4B39
:10B2C40085B01B78002B40F0B281002840F0AF819C
:10B2D400DA4B1C783F2C00F2A78122460120002182
:10B2E40001F09AFCD64DD5E900231943D54B104300
:10B2F400C5E900011D78A5F18103052B00F2FA8050
:10B30400DFE803F00303237A7A10012C00F27E8134
:10B314000120FCF79BFE0028C0F28681FFF782FD26
:10B324003F200EE0012C00F271810120FCF78EFE1B
:10B334000028C0F27981FFF775FDE220FFF740FE97
:10B34400AF20FFF73DFEC0205EE1002C40F05E819F
:10B354002046FCF77BFE0028C0F26681B84EFF222F
:10B364000023D6E9000102430B43C6E90023B54B91
:10B3740001279A785D785543083D042DA8BF04251C
:10B384000FE0E0B20521FCF757FED6E9002304F1F3
:10B39400080117FA01F10A4343EAE173C6E90023FD
:10B3A4000134AC42EDDB4020FFF70AFEA120FFF799
:10B3B40007FEC020FFF704FEA620FFF701FEA2202F
:10B3C400FFF7FEFD2F20FFF7FBFDF820FFF7F8FD48
:10B3D4000020FFF7F5FD2720FFF7F2FD8120FFF79E
:10B3E400EFFD1020FFF7ECFDAC20FFF7E9FD002096
:10B3F400FFF7E6FDAF2007E1002C40F0078120466F
:10B40400FCF724FE0028C0F20F818D4FFF22002399
:10B41400D7E9000102430B43C7E90023894B4FF0EE
:10B42400010C9A785E785643083E042EA8BF042681
:10B4340013E0E0B20521CDF804C0FCF7FDFDD7E927
:10B444000023DDF804C004F108010CFA01F10A43F9
:10B4540043EAE173C7E900230134B442E9DB002481
:10B464004FF47A700134FDF721F8B4F5FA7FF7D17F
:10B47400A820FFF7A5FD3F20FFF7A2FDD320FFF78B
:10B484009FFD0020FFF79CFD4020FFF799FD852DCF
:10B4940004D0A020FFF794FDC02003E0A120FFF713
:10B4A4008FFDC820FFF78CFDDA20FFF789FD1220FD
:10B4B400FFF786FD8120FFF783FD7F20FFF780FDE6
:10B4C400A420FFF77DFDA620FFF77AFDD520FFF726
:10B4D40077FD8020FFF774FD8D20FFF771FD1420A8
:10B4E400FFF76EFDAF20FFF76BFD2020FFF768FD2F
:10B4F400022089E0012D01D1002000E00120FCF7A9
:10B50400A5FD0028C0F290804E4A937852785343A8
:10B51400012B1ADD062B08DC0024E0B205210134DE
:10B52400FCF78AFD042C10D0F7E705210020FCF776
:10B5340083FD05210120FCF77FFD05210220FCF796
:10B544007BFD02200121FCF77AFD3820FCF7E2FDA7
:10B554000020FCF79DFE0020FCF7A6FE0120FFF76B
:10B56400EDFB0020FFF7EAFB41F28830FCF79EFF79
:10B574000120FFF7E3FB0020FFF7E0FB4FF4FA7034
:10B58400FCF794FF0120FFF7D9FB0020FFF7D6FB5F
:10B594004FF4FA70FCF78AFF0820FFF711FD274BE0
:10B5A4001A78274BD3E9000101F02AFB012200237A
:10B5B4001040194050EA010339D00C20FFF700FD78
:10B5C4000620FFF7FDFC0120FFF7FAFC1D4B1B785A
:10B5D400012B15D13920FFF7F3FC1D20FFF7F0FCF8
:10B5E4005020FFF7EDFC6C20FFF7EAFC7C20FFF70E
:10B5F400E7FC154B04A81B6840F8043DFAF78EF9E4
:10B604003820FFF7DDFC0C20FFF7DAFC0B4B1A782F
:10B614000B4BD3E9000101F0F3FA10F0010F0CBF5A
:10B624004FF0FF30002004E06FF0010001E04FF024
:10B63400FF3005B0F0BD00BFED510020E44D002007
:10B64400F0510020887F0020B8D70008F8B5434B9C
:10B654004FF0FF301D78002D7ED1414E33787F337B
:10B66400DAB2052A75D801225BB212FA03F313F099
:10B67400230406D113F0180544D113F0040F20D18C
:10B6840067E03848FAF7AAF92C460FE0A9B200207F
:10B69400FAF716F90027044304E00020FFF718FD29
:10B6A40001370443B3889F42F7DB0135F388B5EBD8
:10B6B400D30FEBDB00200146FAF702F944EA00005D
:10B6C4004AE02848FAF78AF92C4616E02146002079
:10B6D400FAF7F6F805430120FFF7F2FB0120FCF727
:10B6E400D7FD002704E00020FCF774FD0137FFB20A
:10B6F400B388BB42F7D80134E4B2F388B4EBD30F78
:10B70400E4D31FE01748FAF769F9254616E0214605
:10B714000020FAF7D5F805430120FFF7D1FB0120FB
:10B72400FCF7B6FD002704E00020FCF753FD0137C9
:10B73400FFB2B388BB42F7D80134E4B2F388B4EB68
:10B74400D30FE4D300200146FAF7BAF845EA000023
:10B7540002E00120FFF734FCF8BD00BFED510020EA
:10B76400887F0020BCD70008F8B5334B04461B780B
:10B774000D464FF0FF30002B5CD1304B1B78813BE2
:10B78400052B55D8DFE803F003031B3E3E0D04F000
:10B794003F0444F04000FFF713FCC5F3C205044620
:10B7A4000AE03D23B4FBF3F003FB1044E0B2FFF7DF
:10B7B40007FCC5F3C105044645F0B80033E01F4E4D
:10B7C400ED08B388B4FBF3F003FB1040C0F303109F
:10B7D40040F01000FFF7F4FBB3880746B4FBF3F026
:10B7E40003FB104404F00F00FFF7EAFBF38840EA80
:10B7F4000704DB0895FBF3F003FB105565F04F00DD
:10B80400C0B210E004F00F00FFF7DAFBC4F3031436
:10B81400064644F01000FFF7D3FBC5F3C20540EA27
:10B82400060445F0B000FFF7CBFB44EA000001E05A
:10B834006FF00200F8BD00BFED510020887F0020AA
:10B8440008B50E4B1B78B3B90D4B93F90030002BA0
:10B8540006DA0C4B18880C4B1988FFF785FF0CE0AF
:10B86400032908D8094B5B5C181860F07F00C0B24C
:10B87400FFF7A6FB01E04FF0FF3008BDED510020BB
:10B88400887F00209A7F0020847F0020947F0020FE
:10B894006FF0020070476FF002007047F0B587B098
:10B8A40003AB83E80700244B1C78002C3FD1F9F745
:10B8B400F9FF00283BD0214B214A1E889288B242CE
:10B8C40098BF6FF0010034D91E4FBDF812503A886A
:10B8D400ED0801921DE0BDF81420039B02FB043324
:10B8E400029344B13988154B083189B21E803980DE
:10B8F4003046FFF739FF002306E0029AD05C00933C
:10B90400FFF7E6FB009B0133BDF810209342F4DB04
:10B914000134AC42DFDB28465DB1019A094B114684
:10B924001A80064B1888FFF71FFF002001E04FF034
:10B93400FF3007B0F0BD00BFED5100209A7F00201A
:10B94400887F0020847F002010B5044680B9094B0D
:10B954004FF0FF3201201A60FBF794F900280146EA
:10B96400C8BF204605DC0448FAF7FCFB022000E0CF
:10B97400012010BDF8510020C0DA0008003818BFBB
:10B9840001207047F7B51E46C0B90D46044611E0C4
:10B99400A718294638460192FBF7BCF9002805F59B
:10B9A4000075019A05DA06483946FAF7DBFB0120EF
:10B9B40005E00134B442EBDB002000E00420FEBDCE
:10B9C40000DB0008F7B51E46C0B90D46044611E079
:10B9D400A718294638460192FBF7E8F9002805F52F
:10B9E4000075019A05DA06483946FAF7BBFB0120CF
:10B9F40005E00134B442EBDB002000E00420FEBD8E
:10BA04002BDB000800207047002304E011F803C07A
:10BA140000F803C00133013AF8D2704701E000F89E
:10BA2400011B013AFBD27047F7B5C56A04468D4243
:10BA34000E462CD00379F3B100F13003019319467B
:10BA440040782A460123FFF7BDFF10BBA269236A91
:10BA54002071D3189D4238BFE7780AD30BE0A3695D
:10BA64006078ED1801992A460123FFF7ABFF013FE7
:10BA7400FFB2012FF3D8304666B1607804F130018B
:10BA840032460123FFF77EFF18B9E66202E0002088
:10BA940000E00120FEBD000010B504460A464078CF
:10BAA40004F130010123FFF76DFF80BB94F82E32BF
:10BAB40094F82F2243EA0222174B12B29A4228D159
:10BAC40094F8682094F86930120442EA036294F806
:10BAD40066301A4394F8673042EA03220F4B22F08F
:10BAE4007F429A4216D094F8840094F8852000048A
:10BAF40040EA026094F88220104394F8832040EADC
:10BB0400022020F07F40C01A18BF012002E0032069
:10BB140000E0022010BD00BF55AAFFFF46415400BB
:10BB240008B560B1037853B1C3888B4207D140781C
:10BB3400FFF724FF10F0010018BF032000E00920E4
:10BB440008BD0129F7B504460D4657D9C369994282
:10BB540054D20378066A022B28D0032B35D0012B4C
:10BB64004ED101EB510706EB5721FFF75DFF00288B
:10BB740046D1FB0504EBD35393F83030013706EB81
:10BB8400572120460193FFF74FFF019BC0BBFF05E0
:10BB940004EBD75494F8300015F0010F43EA002069
:10BBA40001D000092EE00005000D2BE006EB112169
:10BBB400FFF73AFF20BB2D0604EBD55494F831006F
:10BBC40094F8303043EA00201CE006EBD111FFF773
:10BBD4002BFFA8B96D0604EBD55494F8320094F801
:10BBE4003330000440EA036094F83030184394F88A
:10BBF400313040EA032020F0704003E0012001E0EE
:10BC04004FF0FF30FEBD0129F7B504460D46164638
:10BC14006DD9C36999426AD20378076A022B3ED070
:10BC2400032B4BD0012B5ED101EB510307EB5321C6
:10BC34000193FFF7F9FE019B002855D1D805C00DEB
:10BC440015F001021CBF04EB000C9CF830C0F1B2EB
:10BC54001EBF0CF00F0C4CEA0111C9B220185D1C78
:10BC6400012380F83010237107EB552120460192FF
:10BC7400FFF7DAFE019AB8BBED05ED0D12B1C6F37C
:10BC8400071608E0631993F83030C6F3032623F04F
:10BC94000F0343EA0606651985F8306024E007EBD4
:10BCA4001121FFF7C1FEF8B92D0604EBD55585F82F
:10BCB4003060C6F3072685F8316015E007EBD11133
:10BCC400FFF7B2FE80B96D0604EBD555C6F3072322
:10BCD40085F8306085F83130330C360E85F8323013
:10BCE40085F8336000E002200123237100E0022084
:10BCF400FEBDF7B5C36905460E4661B9C768D7F1FD
:10BD0400010238BF00229F4228BF42F00102002AEC
:10BD140018BF012708E00193FFF713FF0128019BD7
:10BD240035D998423DD337463C4601349C4202D330
:10BD3400012F2ED90224284621460193FFF701FF43
:10BD4400019B60B1B0F1FF3F14BF00220122012822
:10BD540008BF42F0010222BBBC42E6D11BE02846E8
:10BD640021466FF07042FFF74EFFB0B92EB128465E
:10BD740031462246FFF747FF78B92B69EC60B3F1EF
:10BD8400FF3F0DD0013B2B6101236B7108E00120C3
:10BD940007E0002005E0104603E04FF0FF3000E02C
:10BDA4002046FEBD0129F8B504460F4624D9C369CF
:10BDB40099421AD320E020463946FFF7C2FE0546D1
:10BDC400C8B1012818D0B0F1FF3F17D0204639463A
:10BDD4000022FFF718FF90B92369B3F1FF3F02D0A7
:10BDE4000133236166712F4600E00126E3699F4217
:10BDF400E1D3002003E002E0022000E00120F8BDCE
:10BE0400C3690239023B99423DBF8278836A02FBCF
:10BE140001300020704770B504460D46E18081680A
:10BE240001293AD00368DA69914236D279B91A788D
:10BE3400032A01D1596A51B90022E2601A89AA423F
:10BE440082BF5B6A03EB151323611BD825E09E7840
:10BE540036010EE02068FFF774FEB0F1FF3F0146A3
:10BE640019D0012819D92368DB69984215D2AD1B72
:10BE7400ADB2B542EED2E1602068FFF7C1FF00EB3E
:10BE840015102061236805F00F05303303EB4515C9
:10BE94006561002002E0012000E0022070BDF7B5DA
:10BEA400C68804460136B6B20F46002E69D003692F
:10BEB400002B66D016F00F0F59D1C168013303610E
:10BEC400006819B90389B34251D85AE08378013B19
:10BED40013EA16134BD1FFF734FE0128054654D953
:10BEE400B0F1FF3F53D02068C3699D4239D3002F7E
:10BEF40047D0E168FFF7FDFE0546002843D001283E
:10BF040043D0B0F1FF3F42D020680021FFF78CFD01
:10BF1400074600283BD12068394630304FF4007280
:10BF2400FFF77CFD2368294618460193FFF768FF55
:10BF3400019BD86201230DE0137120680021019355
:10BF4400FFF772FD019B10BB22680137D16AFFB273
:10BF54000131D16222689178B942EDD8D36ADF1BEE
:10BF6400D762E56020682946FFF74AFF206123680D
:10BF7400E680303306F00F0603EB461666610020B8
:10BF840006E0042004E0072002E0022000E0012093
:10BF9400FEBD0000F7B504460B780D460131202B99
:10BFA400FAD02F2B14BF002201225C2B14BF13469E
:10BFB40042F001030026002B18BF0D46A6602B7823
:10BFC4001F2B05D820463146FFF725FF6661C8E0E0
:10BFD400A669202130460B22FFF720FD00210191A4
:10BFE40008200A46DDF804C015F80C300CF1010CE9
:10BFF400202B8CBF002701272F2B08BF47F00107F8
:10C00400CDF804C0002F44D15C2B46D02E2B14BF96
:10C01400002701278142A8BF47F001077FB12E3BCB
:10C0240018BF012308280CBF184643F0010000285C
:10C0340040F094809200D2B208210B30D2E713F082
:10C04400800F04D0DFF81CC1803B1CF80330DFF8FC
:10C0540018C137461CF8016F16B19E42FAD17DE033
:10C06400A3F1410C5FFA8CFCBCF1190F3E4698BF5A
:10C0740042F002020AD9A3F1610C5FFA8CFCBCF114
:10C08400190F03D8203B42F00102DBB27354013193
:10C09400A8E7202B94BF0427002700295ED033781B
:10C0A400E52B01D105233370082801D19200D2B2C7
:10C0B40002F00303012B02F00C0208BF47F0100743
:10C0C400042A08BF47F00807F77220460021FFF74B
:10C0D400A2FEE0B920682169FFF7A6FCB8B963693C
:10C0E4001A789AB1DA7A12F0080F0AD1A26903F128
:10C0F4000B018B420BD013F8016B12F801CB664590
:10C10400F7D020460021FFF7CAFEE2E70420A36926
:10C11400DB7A03F00403DBB260B1042814BF00220D
:10C124000122002B14BF002302F00103002B18BFCF
:10C13400052016E0ABB96369DA7A12F0100F0FD05C
:10C14400019A597DAD181A7D42EA0122D97E9B7E5F
:10C1540043EA012343EA0243A36039E7062000E0EF
:10C164000520FEBDD0DB00089CDB000870B5002173
:10C174000446FFF750FE054648BB20682169FFF7D7
:10C1840053FC054618BB63691B78E52B14BF0022DA
:10C194000122002B14BF134642F00103CBB9204601
:10C1A4000121FFF77CFEE6E7666929463046202236
:10C1B400FFF734FC0B223046A169FFF725FCA36985
:10C1C4000122DB7A03F01803337323681A712846BB
:10C1D40070BD20682169FFF727FC05460028F6D1C9
:10C1E400E2E70000F8B5036815461A78303A092AE0
:10C1F40009D893F801C0BCF13A0F04D102330360AB
:10C20400002A40F01C819E4B1C680C60002C00F03E
:10C21400188123786BB16078FFF7B0FB10F0010F41
:10C2240007D1002D00F00F8110F0040018BF0A2080
:10C2340012E1002020706070FFF786FB10F0010F00
:10C2440040F003811DB110F0040F40F00081002183
:10C254002046FFF721FC012817D194F8F231002B76
:10C2640000F0F98094F8F86194F8F931360446EA5C
:10C27400036694F8F63120461E4394F8F73146EAF3
:10C2840003263146FFF708FC00E00026032800F0EF
:10C29400E080002840F0DF8094F83C2094F83B30A4
:10C2A40043EA0223B3F5007F40F0D58094F8472099
:10C2B40094F8463053EA02230DD194F8563094F89A
:10C2C40057201B0443EA026394F85420134394F860
:10C2D400552043EA022394F8402094F842C094F88D
:10C2E4004110A361E270534394F83F0094F83E2058
:10C2F40041EA0C2194F8445094F843C042EA0020E7
:10C3040094F83D7032185CEA052C2262A7702181F2
:10C314000FD194F852C094F853504FEA0C4C4CEAA5
:10C32400056C94F850504CEA050C94F851504CEAC2
:10C33400052CC0EB0C000909C01A401AB0FBF7F732
:10C34400023740F6F6708742E76106D900F570407F
:10C35400874200F28280022500E00125981860627D
:10C364005218D318A3624FF0FF3323610133032D16
:10C3740023715AD1637194F8612094F86030607825
:10C3840043EA0222B218626104F130010123FFF78B
:10C39400F9FA002849D194F82E3294F82F2243EA6E
:10C3A4000222384B12B29A423FD194F8322094F8C8
:10C3B4003330120442EA036294F830301A4394F89A
:10C3C400313042EA0322304B9A422ED194F816229D
:10C3D40094F81732120442EA036294F814321A43AE
:10C3E40094F8153242EA0322284B9A421DD194F85C
:10C3F4001E3294F81F221B0443EA026394F81C22A1
:10C40400134394F81D2243EA0223E36094F81A329A
:10C4140094F81B221B0443EA026394F81822134382
:10C4240094F8192243EA02232361194A25701388D8
:10C43400002001339BB2E0621380E3800CE00B2008
:10C444000AE00C2008E0284606E0032004E00A2065
:10C4540002E0012000E00D20F8BD94F85E0094F89D
:10C464005FC0000440EA0C6094F85CC0032540EA15
:10C474000C0094F85DC040EA0C20606270E700BFD5
:10C484000052002055AAFFFF52526141727241616D
:10C49400FC51002050B9064B1B6803B1187009B158
:10C4A40000230B70024B0020196000E00B20704742
:10C4B40000520020F0B58DB0044600230CA802F011
:10C4C4001F0502AE40F82C1D236005F01E02314604
:10C4D400FFF788FE002840F0998009AB30460199A7
:10C4E4000893FFF757FD15F01C0F56D060B10428D0
:10C4F40040F08C803046FFF739FE002840F08680FB
:10C5040045F00805079E33E015F0040F79D1079E26
:10C51400002E7AD0F37A13F0110376D115F0080FB8
:10C5240026D0327D777DF17E42EA0727B27E3375CD
:10C534007375B376F37633777377B377F3770298BB
:10C5440042EA0122012352EA07470371C36A09D070
:10C5540039460093FFF726FC009B002856D1029A27
:10C56400013FD76002981946FFF75EFA00284DD1C3
:10C5740015F0080F20D00023F372FFF743FAC0F33D
:10C584000723B073F373030C000E33747074029BAF
:10C5940001221A7145F020050EE0002836D1079ECD
:10C5A400002E30D0F37A13F0100F2CD115F0020FB7
:10C5B40002D013F0010F28D1029BDA6AA571E2615F
:10C5C400079A2262327D717DF07E42EA0121B27EB9
:10C5D40042EA002242EA01422261B27FF17F120460
:10C5E40042EA0162317F00200A43717F236042EAFC
:10C5F4000122E260FF22E271DB88A060A061A380D7
:10C6040004E0082002E0042000E007200DB0F0BDA3
:10C61400F0B587B004931746049A002304460E46E7
:10C62400136081880068FFF77BFA0546002840F014
:10C63400A780A37913F0800F40F09F8013F0010FBF
:10C6440000F09D80E268A3680296D31A9F4228BF37
:10C654001F4604F1240301970393059087E0A36820
:10C66400DA0568D12068E179827891420DD30BB95B
:10C67400206902E06169FFF764FA01280BD9B0F17F
:10C68400FF3F4ED000236061E3712768616938463B
:10C69400FFF7B6FB20B9A37963F07F03A3716CE0C5
:10C6A400E379019AC618550A21D0BA78E91891425B
:10C6B40088BFD51AEBB2787802993246FFF762F94F
:10C6C400A37900282ED113F0400F0BD0A069801B52
:10C6D400A84207D2029B039903EB40204FF4007257
:10C6E400FFF792F9E379EB18E3716D0232E0A37975
:10C6F40013F0400F0AD0012378780399A269FFF759
:10C7040061F9A37970B923F04003A371A369B3421B
:10C714000DD023680399587832460123FFF732F984
:10C7240028B1A37963F07F03A371012528E0E3799D
:10C73400A6610133E371A168019AC905C90DC1F568
:10C744000075039BAA4238BF1546591802982A4619
:10C75400FFF75AF9029AA36852190292049A5B19D4
:10C76400A36013685B191360019B5B1B0193019A1F
:10C77400002A7FF474AF059D02E0022500E007253E
:10C78400284607B0F0BDF8B504460E468188006817
:10C79400FFF7C6F90546002840F09E80A27912F002
:10C7A400800F40F09880E3689E4203D912F0020F94
:10C7B40008BF1E460022A368A260FF32E271002E69
:10C7C40059D0206887787F0273B1013B711EB1FB99
:10C7D400F7F1B3FBF7F2914206D37A4202EA03037C
:10C7E400A360F61A61690CE0216949B9FFF781FA7F
:10C7F4000128014635D0B0F1FF3F18BF206159D060
:10C804006161002936D01BE0A37913F0020F05D033
:10C814002068FFF76EFA014620B914E02068FFF79C
:10C8240090F90146B1F1FF3F44D0012919D9236899
:10C83400DB69994215D2A3686161DB19A360F61B19
:10C84400BE42E1D800E03E46A368C6F347279B19E1
:10C85400A360F305E771DE0D6BB12068FFF7D0FA32
:10C8640020B9A37963F07F03A37134E0C6190137BB
:10C87400E77100E00E46A368DB0522D0A269964268
:10C884001FD0A37913F0400F0BD0214651F8243B5D
:10C8940058780123FFF796F8A37960B923F0400391
:10C8A400A371214651F8243B324658780123FFF7FF
:10C8B40069F828B1A37963F07F03A37101250BE024
:10C8C400A661A368E268934206D9E360A37943F0C2
:10C8D4002003A37100E002252846F8BD10B586B0F8
:10C8E400044606A840F8141D00222146FFF77AFCEE
:10C8F40018BB03ABA36120460199FFF74BFBB8B902
:10C90400636973B1DA7A12F0100F15D0597D1A7D6C
:10C9140042EA0122D97E9B7E43EA012343EA024391
:10C92400A36023682046DB880021A380FFF773FA05
:10C93400042808BF052000E0052006B010BD000053
:10C9440000B5124B00201870114B124989B01870B1
:10C95400FFF7A0FD014628B10F48F9F703FC4FF09B
:10C96400FF3010E00D4901A8FFF7B8FF014628B1D8
:10C974000B48F9F7F7FB6FF0010004E0094B0122C3
:10C984001870094B1A7009B000BD00BF4E54002046
:10C994004F5400201052002050DC000883DC0008B3
:10C9A40085DC0008045200204C54002008B5094BD3
:10C9B40000201870084B1870084B1870084B18703A
:10C9C400084B1860084B1860FAF73FF8074B05222C
:10C9D4001A7008BD4E5400204F54002040540020CB
:10C9E4004C54002048540020445400204D5400204E
:10C9F400014B9878704700BF10520020054B821EEF
:10CA0400D96902398A423DBF98789B6A00FB02309B
:10CA1400002070471052002070B51D4B04461B784F
:10CA24000D462BB11B48F9F79DFB6FF005002EE076
:10CA340019480122FFF73EFD184E306068B1FFF738
:10CA44007FFF0028B8BF4FF0FF3020DB1248294693
:10CA54000122FFF72FFD3060B8B90F4B00209A79FF
:10CA64002270DA7962709A686260DA68A2601A6980
:10CA7400E2605A6922619A696261DA691B6AA26199
:10CA8400E361034B01221A7001E06FF0040070BDF2
:10CA94004E54002030DD000850540020BC7F00209C
:10CAA40010B5174B1B782BB11648F9F75BFB6FF0E9
:10CAB400050023E0144B1549DA88D1F818C08A80A0
:10CAC40002780B608A714278CA71426884698A600C
:10CAD4008268CA60C2680A6102694A614269C069BF
:10CAE40094458A61CC61086204D0587824310123CA
:10CAF400FEF748FF024B01221A70002010BD00BF50
:10CB04004E5400208CDD00081052002050540020A8
:10CB14000B4B9A790270DA7942709A684260DA684B
:10CB240082601A69C2605A6902619A694261DA696B
:10CB34001B6A8261C361034B00201870704700BFF9
:10CB4400505400204E54002008B501460448FFF715
:10CB54001AFE044B0028186018BF6FF00F0008BDC0
:10CB640050540020BC7F002013B50D4A03461278B0
:10CB74000C466FF002008AB119460A4801AB2246FE
:10CB8400FFF746FD084B186030B9019BA3420CBF68
:10CB940000206FF0070001E06FF006001CBD00BF2D
:10CBA4004C54002050540020BC7F0020F8B50446AB
:10CBB4000F4600250F4E14E001212046FFF7D4FF55
:10CBC400002815DB237801350A2B14BF002201222B
:10CBD4000D2B14BF134642F0010333B9BD4238BFD5
:10CBE4000134B268F3689A42E6D3002323702846DE
:10CBF400F8BD00BF5054002008B5F8F7A3FD08BDE8
:10CC0400D0400B1CD1409C46203AD340184352429A
:10CC140063469340184370479140031C90409C46E0
:10CC2400203A9340194352426346D3401943704714
:10CC340070B50D4D0D4E0024761BB61003E055F86B
:10CC4400043B98470134B442F9D3094D094EF8F72F
:10CC540027FE761BB610002403E055F8043B9847E2
:10CC64000134B442F9D370BD1CEA00081CEA000880
:10CC74001CEA00081CEA0008002305E011F803C0C0
:10CC8400013A00F803C00133002AF7D17047034684
:10CC940002E003F8011B013A002AFAD1704710B5EB
:10CCA40084469CF8003062460CF1010C002BF8D14C
:10CCB400CC5CD4540133002CFAD110BD10F8013BE4
:10CCC4000A461BB111F801CB6345F7D01078181A46
:10CCD40070470023CA5CC2540133002AFAD170475A
:10CCE40003461A4613F8011B0029FAD1101A70479B
:10CCF40010B5844607E011F8014B634603F8014B75
:10CD0400013A9C462CB1002AF5D104E003F8014B0A
:10CD1400013A002AFAD110BDF7B51F4E0446376810
:10CD2400D7F8E850002D2ED150200191FFF764FF71
:10CD34003368C7F8E800D3F8E820956015605560BB
:10CD4400D3F8E8201561D560D3F8E82095615561E2
:10CD5400D3F8E820D5629562D3F8E82055631563CB
:10CD6400D3F8E820D5639563D3F8E82055641564B7
:10CD7400D3F8E820D5649564D3F8E8201577D3F880
:10CD8400E83001995D62044B20461B68D3F8E82023
:10CD9400012300F003F8FEBD6C010020F0B510B9CA
:10CDA4001068002829D084460D4610F8014B07E08E
:10CDB400B44205D1002BF6D110608CF8003017E096
:10CDC40015F8016B002EF3D1034614B91460204604
:10CDD40013E01F4613F8010B0D461C4615F8016BB2
:10CDE400864207D110B100233B7000E00446146072
:0CCDF400604602E0002EF1D1EBE7F0BD3C
:10CE0000000305070A0C0F11131517191C1E202209
:10CE1000242527292B2D2E3032333537383A3B3D08
:10CE20003E3F414244454647494A4B4C4E4F505184
:10CE300052535455565758595A5B5C5D5D5E5E5F60
:10CE4000606162636465656667676869696A6B6B80
:10CE50006C6D6D6E6E6F6F707071717272737374D2
:10CE600074757576767677777878787979797A7A4D
:10CE70007A7B7B7B7C7C7C7D7D7D7E7E7E7F7F7FE5
:10CE800046696C656E616D652069732025732E009F
:10CE90005B4150505D206661696C656420746F2051
:10CEA0006F70656E2066696C652C20737461747593
:10CEB000733A2025640A005B4150505D2053616D38
:10CEC000706C65206E6F2025642066696C656E61EC
:10CED0006D65202573206F70656E6564206F662018
:10CEE0006C656E6774682025750A004162616E6426
:10CEF0006F6E696E6720444D4120726F7574696E64
:10CF0000652061667465722025642E2564206D732A
:10CF10002C20616674657220256420766F696365D4
:10CF200073206F7574206F66202564004F70656EE6
:10CF3000696E672062616E6B2066696C652025737F
:10CF4000004661696C656420746F206F70656E20A7
:10CF500062616E6B2066696C652E0053616D706C4A
:10CF600065206E6F2025642C2066696C656E616D8E
:10CF7000652069733A2025732C206D696469206EE1
:10CF80006F74652076616C75653D307825782C204E
:10CF900064656361792076616C75652025642C2059
:10CFA000686F6C643D2564004F70656E2073616D21
:10CFB000706C652066696C65206661696C65642EBD
:10CFC00000436C75737465722025643A20256420D3
:10CFD000004F70656E696E67206E65772073616DB6
:10CFE000706C652062616E6B004F70656E696E6774
:10CFF00020636F6E6669672066696C652025730023
:10D00000706C617965722E636667004661696C6554
:10D010006420746F206F70656E20636F6E66696741
:10D020002066696C652E00466F756E6420706172B3
:10D03000616D20257320616E642076616C756520BA
:10D040002573006C65655F6877006D696469636866
:10D05000616E6E656C004D4944492050726F677275
:10D06000616D204368616E676520726563656976EE
:10D070006564202D204368616E67696E6720626178
:10D080006E6B20746F2025640053442063617264CA
:10D0900020706F6C7970686F6E69632073616D705A
:10D0A0006C6520706C6179657200284329203230EC
:10D0B0003131204C204F27446F6E6E656C6C206CB4
:10D0C000656540626173736D616B65722E636F2E6F
:10D0D000756B00496E697469616C6973696E67206C
:10D0E000534420636172642E2E004572726F722069
:10D0F000696E697469616C6973696E672053442055
:10D1000063617264005344204361726420657272EB
:10D110006F723A20636F6E6E656374696F6E20661E
:10D1200061696C6564210052656164696E67204ABB
:10D1300031302073776974636800496E697469617E
:10D140006C6973696E672073796E74682E2E2E0079
:10D1500053796E746820696E697420646F6E652EF1
:10D1600000564F4943455F5343414E0042414E4BA9
:10D170005357495443485F5343414E004D49444936
:10D180005F486F6F6B7300464154414C3A204672C2
:10D19000656552544F5320004D616C6C6F632045A0
:10D1A00072726F722121212000464154414C3A2075
:10D1B0004672656552544F53204D616C6C6F63200D
:10D1C0004572726F722121210A00476F6F64627984
:10D1D000652100476F6F64627965210A003D3D3D1E
:10D1E0003D3D3D3D3D3D3D3D3D3D3D3D3D3D3D0AA2
:10D1F000002121212048415244204641554C5420D1
:10D200002121210A005230203D20253038780A00A3
:10D210005231203D20253038780A005232203D20FE
:10D22000253038780A005233203D20253038780ADE
:10D2300000523132203D20253038780A004C5220EF
:10D240003D20253038780A005043203D20253038D5
:10D25000780A00505352203D20253038780A004289
:10D26000464152203D20253038780A00434653522B
:10D27000203D20253038780A0048465352203D2072
:10D28000253038780A0044465352203D2025303856
:10D29000780A0041465352203D20253038780A0054
:10D2A00021212048415244204641554C54202121FF
:10D2B0000061742050433D3078253038780049446F
:10D2C0004C45000A0A44756D70696E672074686584
:10D2D00020756D6D5F686561702E2E2E0A007C30A2
:10D2E00078253038787C42202535647C4E422025D4
:10D2F00035647C5042202535647C5A202535647C79
:10D300004E46202535647C5046202535647C0A0035
:10D310007C3078253038787C42202535647C4E423C
:10D32000202535647C5042202535647C5A202535E3
:10D33000647C0A00546F74616C20456E7472696578
:10D340007320253564202020205573656420456EA8
:10D35000747269657320253564202020204672652B
:10D360006520456E7472696573202535640A005422
:10D370006F74616C20426C6F636B73202025356481
:10D38000202020205573656420426C6F636B7320EE
:10D3900020253564202020204672656520426C6F70
:10D3A000636B7320202535640A0053697A65206F0A
:10D3B0006620756D6D5F68656170206973202564F6
:10D3C0002062797465732C20757365643A20256436
:10D3D0002062797465732C20667265653A20256435
:10D3E0002062797465730A0043616E277420616C52
:10D3F0006C6F636174652025356420626C6F636BAC
:10D4000073206174202535640A0000000040145424
:10D41000434C434400434C43445F444F4700474C14
:10D4200043445F435553544F4D00474C43445F4B77
:10D43000533031303800474C43445F4B5330313028
:10D44000385F494E56435300474C43445F444F476F
:10D4500000474C43445F5353443133303600474C0C
:10D4600043445F535344313330365F524F54415439
:10D47000454400474C43445F534544313532300006
:10D48000000201001400020001000000010102017D
:10D490000000000000000000000000000000020387
:10D4A0000301020303030303020203014D494F5327
:10D4B0003332004D4248505F434F52455F53544D05
:10D4C00033320053544D333246313078003F005BE5
:10D4D0004D494F5333325F4D4944495F535953458A
:10D4E000585F436D645F44656275675D20636F6D6F
:10D4F0006D616E642068616E646C6572206E6F741D
:10D5000020696D706C656D656E746564206279204C
:10D510006170706C69636174696F6E0A00284552AE
:10D52000524F523A20737472696E67207061737340
:10D53000656420746F204D494F5333325F4D494429
:10D54000495F53656E6444656275674D65737361C9
:10D5500067652829206973206C6F6E676572207477
:10D5600068616E20313030206368617273210A0077
:10D570005B4D494F5333325F4D4944495F526563B8
:10D58000656976655F48616E646C65725D2054699B
:10D590006D656F7574206F6E20706F7274203078B7
:10D5A000253032780A00202530325800253038588E
:10D5B000200000000202020201010200F000007ED1
:10D5C00032000000FEFFFFFFFFFFFFFF0000000032
:10D5D000426F6F746C6F61646572204D6F6465207B
:10D5E0000000000000100140010000000010014098
:10D5F0000200000000100140040000000010014083
:10D60000080000000008014001000000000801407F
:10D610000200000000080140040000000008014072
:10D620000800000000100140100000000010014040
:10D6300020000000000C014001000000000C01402F
:10D640000200000045A90008FD84000845A9000863
:10D6500045A9000845A9000845A9000845A90008F2
:10D6600045A90008D584000812010002000000400E
:10D67000C016FE03000101020301000000000000CB
:10D68000AD860008E1840008E3840008E584000812
:10D69000E9840008ED84000891860008758600087A
:10D6A0001D85000800000000400000006D696469ED
:10D6B000626F782E6F726700C8D6000865000000A0
:10D6C00068D600081200000009026500020100800F
:10D6D00032090400000001010002092401000109CF
:10D6E00000010109040100020103000207240100F6
:10D6F0000141000624020101000624020202000981
:10D7000024030103010201000924030204010101B1
:10D710000009050202400000000005250101010981
:10D720000581024000000000052501010300000002
:10D73000286E756C6C290000D10FED54CFC5FBB875
:10D740009752389138910E7D0FED389301910E91DB
:10D7500000C11F020E91F7041040006E106EE76AC0
:10D7600000000000000000000000000000000000B9
:10D7700000000000000004000000000000000000A5
:10D78000000000002F55461F00D84840376AF76A4E
:10D7900000300000C7062E734A2C137BE97F32004D
:10D7A0002A280D9BFE0B21EF422A2F73B5B8DA769B
:10D7B000E679BF0FEB793E0B00102030060800061B
:10D7C00000808080808000C0C0C0C0C000E0E0E079
:10D7D000E0E000F0F0F0F0F000F8F8F8F8F800FC05
:10D7E000FCFCFCFC00FEFEFEFEFE00FFFFFFFFFF58
:10D7F00000183C7EFF0000FF7E3C18000000000087
:10D800000000000000000000000000000000000018
:10D810000000000000000000000000000000000008
:10D8200000000000000000000000000000000000F8
:10D8300000000000000000000000000000000000E8
:10D8400000000000000000000000000000000000D8
:10D8500000000000000000000000000000000000C8
:10D8600000000000000000000000000000000000B8
:10D8700000000000000000000000000000000000A8
:10D880000000000000000000004F00000000070042
:10D89000070000147F147F1400242A7F2A1200231B
:10D8A0001308646200364955225000000503000049
:10D8B00000001C224100000041221C000014083E10
:10D8C00008140008083E0808000000503000000856
:10D8D000080808080000303000000020100804028A
:10D8E000003E5149453E0000427F400000426151E8
:10D8F0004946002141454B31001814127F10002782
:10D9000045454539003C4A49493000017109050344
:10D9100000364949493600064949291E00000036AB
:10D9200036000000005636000008142241000014A2
:10D9300014141414000041221408000201510906B5
:10D9400000324979413E007E1111117E007F494924
:10D950004936003E41414122007F4141221C007F67
:10D9600049494941007F09090901003E4149497A75
:10D97000007F0808087F0000417F410000204041EF
:10D980003F01007F08142241007F40404040007F5B
:10D99000020C027F007F0408107F003E4141413E9F
:10D9A000007F09090906003E4151215E007F0919E7
:10D9B00029460046494949310001017F0101003FE4
:10D9C0004040403F001F2040201F003F4038403F64
:10D9D00000631408146300070870080700615149C8
:10D9E000454300007F414100000204081020000070
:10D9F00041417F00000402010204004040404040D9
:10DA0000000001020400002054545478007F484470
:10DA1000443800384444442000384444487F0038A7
:10DA20005454541800087E090102000C5252523E10
:10DA3000007F080404780000447D4000002040443A
:10DA40003D00007F102844000000417F4000007C22
:10DA500004180478007C08040478003844444438EE
:10DA6000007C1414140800081414187C007C0804AA
:10DA7000040800485454542000083E484020003C0C
:10DA80004040207C001C2040201C003C4030403C9A
:10DA9000004428102844000C5050503C004464546A
:10DAA0004C440000083641000000007F00000000E8
:10DAB00000413608000201020100000000000000E1
:10DAC0005B6469736B5F696E697469616C697A65BF
:10DAD0005D206572726F72207768696C652063687B
:10DAE00065636B696E6720666F72205344204361E3
:10DAF00072642028737461747573202564290A0088
:10DB00005B6469736B5F726561645D206572726FDF
:10DB100072207768696C652072656164696E672040
:10DB2000736563746F722025640A005B6469736BAC
:10DB30005F77726974655D206572726F72207768B5
:10DB4000696C652077726974696E6720746F2073E1
:10DB50006563746F722025640A005B4745545F5308
:10DB60004543544F525F434F554E545D20436F75AC
:10DB70006E742069732025640A005B4745545F4238
:10DB80004C4F434B5F53495A455D20426C6F636B6A
:10DB90002053697A652069732025640A0020222AAF
:10DBA0002B2C5B3D5D7C7F004E4F204E414D452030
:10DBB0002020204641542020202020004E4F204E7F
:10DBC000414D452020202046415433322020200062
:10DBD000809A90418E418F804545454949498E8FB5
:10DBE0009092924F994F555559999A9B9C9D9E9F03
:10DBF00041494F55A5A5A6A7A8A9AAABAC21AEAF90
:10DC0000B0B1B2B3B4B5B6B7B8B9BABBBCBDBEBF9C
:10DC1000C0C1C2C3C4C5C6C7C8C9CACBCCCDCECF8C
:10DC2000D0D1D2D3D4D5D6D7D8D9DADBDCDDDEDF7C
:10DC3000E0E1E2E3E4E5E6E7E8E9EAEBECEDEEEF6C
:10DC4000F0F1F2F3F4F5F6F7F8F9FAFBFCFDFEFF5C
:10DC50005B46494C455D204661696C656420746F84
:10DC6000206D6F756E742053442043617264202DC3
:10DC7000206572726F72207374617475733A202517
:10DC8000640A002F005B46494C455D204661696C83
:10DC9000656420746F206F70656E20726F6F7420E2
:10DCA0006469726563746F7279202D206572726F7A
:10DCB00072207374617475733A2025640A005B46A0
:10DCC000494C455F5570646174654672656542797B
:10DCD0007465735D20665F6F70656E64697220663F
:10DCE00061696C6564207769746820737461747508
:10DCF00073202564210A005B46494C455F557064DA
:10DD00006174654672656542797465735D20665F0E
:10DD100067657466726565206661696C6564207705
:10DD200069746820737461747573202564210A0016
:10DD30005B46494C455D204641494C5552453A2089
:10DD4000747269656420746F206F70656E206669F7
:10DD50006C65202725732720666F722072656164C9
:10DD6000696E672C206275742070726576696F75B4
:10DD7000732066696C65206861736E277420626524
:10DD8000656E20636C6F736564210A005B46494CC5
:10DD9000455D204641494C5552453A2074726965AB
:10DDA0006420746F2072656F70656E2066696C65A3
:10DDB0002C206275742070726576696F75732066A9
:10DDC000696C65206861736E2774206265656E20DA
:10DDD000636C6F736564210A005B46494C455D20A6
:10DDE0004641494C5552453A207472696564207425
:10DDF0006F206F70656E2066696C6520272573271C
:10DE000020666F722077726974696E672C20627564
:10DE1000742070726576696F75732066696C652011
:10DE20006861736E2774206265656E20636C6F7322
:10DE30006564210A005B46494C455F53656E645337
:10DE4000797844756D705D204552524F5220776845
:10DE5000696C652072656164696E672066696C65CE
:10DE60002C207374617475733A2025640A0045523E
:10DE7000524F523A2052656164696E6720434944AB
:10DE8000206661696C6564207769746820737461C9
:10DE9000747573202564210A002D2D2D2D2D2D2D17
:10DEA0002D2D2D2D2D2D2D2D2D2D2D2D2D0A0043DC
:10DEB00049443A0A002D204D616E756661637475A0
:10DEC00072657249443A0A002D204F454D20417039
:10DED000706C6949443A0A002D2050726F644E619B
:10DEE0006D653A2025730A002D2050726F645265CB
:10DEF000763A2025750A002D2050726F64534E3AF1
:10DF0000203078253038780A002D205265736572EC
:10DF1000766564313A2025750A002D204D616E75B5
:10DF200066616374446174653A2025750A002D208A
:10DF30006D73645F4352433A203078253032780A5B
:10DF4000002D205265736572766564323A2025751E
:10DF50000A004552524F523A2052656164696E6719
:10DF600020435344206661696C6564207769746856
:10DF700020737461747573202564210A002D204379
:10DF800053445374727563743A2025750A002D202A
:10DF90005379735370656356657273696F6E3A2077
:10DFA00025750A002D20544141433A2025750A0069
:10DFB0002D204E5341433A2025750A002D204D61F6
:10DFC00078427573436C6B467265633A2025750A17
:10DFD000002D2043617264436F6D64436C61737301
:10DFE00065733A2025750A002D205264426C6F63D8
:10DFF0006B4C656E3A2025750A002D2050617274B5
:10E00000426C6F636B526561643A2025750A002D7E
:10E01000205772426C6F636B4D6973616C69676EF8
:10E020003A2025750A002D205264426C6F636B4DB7
:10E030006973616C69676E3A2025750A002D20446A
:10E040005352496D706C3A2025750A002D204465A5
:10E050007669636553697A653A2025750A002D2033
:10E060004D6178526443757272656E745644444DC6
:10E07000696E3A2025750A002D204D61785264435F
:10E08000757272656E745644444D61783A202575F8
:10E090000A002D204D6178577243757272656E7457
:10E0A0005644444D696E3A2025750A002D204D6175
:10E0B00078577243757272656E745644444D617838
:10E0C0003A2025750A002D204465766963655369F9
:10E0D0007A654D756C3A2025750A002D20457261D0
:10E0E0007365477253697A653A2025750A002D20B9
:10E0F000457261736547724D756C3A2025750A004B
:10E100002D20577250726F74656374477253697A29
:10E11000653A2025750A002D20577250726F74657C
:10E1200063744772456E61626C653A2025750A001A
:10E130002D204D616E4465666C4543433A2025753C
:10E140000A002D2057725370656564466163743A06
:10E150002025750A002D204D61785772426C6F633F
:10E160006B4C656E3A2025750A002D205772697434
:10E1700065426C6F636B50615061727469616C3A97
:10E180002025750A002D205265736572766564330B
:10E190003A2025750A002D20436F6E74656E745009
:10E1A000726F746563744170706C693A2025750AEA
:10E1B000002D2046696C65466F726D617447726F01
:10E1C000756F703A2025750A002D20436F707946CF
:10E1D0006C61673A2025750A002D205065726D57D5
:10E1E0007250726F746563743A2025750A002D2091
:10E1F00054656D70577250726F746563743A202560
:10E20000750A002D2046696C65466F726D61743A1F
:10E210002025750A002D204543433A2025750A0024
:10E220002D205265736572766564343A2025750A2F
:10E23000005B5344434152445F4552524F523A258A
:10E24000645D206661696C656420746F206163633E
:10E2500065737320534420636172640A005B534406
:10E26000434152445F4552524F523A25645D204427
:10E2700046535F47657450746E53746172742066C0
:10E2800061696C656420746F2066696E64207061DA
:10E2900072746974696F6E0A005B5344434152445F
:10E2A0005F4552524F523A25645D204446535F47C2
:10E2B0006574566F6C496E666F206661696C656443
:10E2C00020746F2066696E6420766F6C756D6520B2
:10E2D000696E666F726D6174696F6E0A005B53449C
:10E2E000434152445F4552524F523A25645D207576
:10E2F0006E6B6E6F776E2066696C6573797374658B
:10E300006D20286F6E6C792046415431322F3136A2
:10E310002F333220737570706F72746564290A0030
:10E320005B5344434152445F4552524F523A256435
:10E330005D204446535F4F70656E46696C65282EBC
:10E340002E4446535F524541442E2E292066616972
:10E350006C65642C20652E672E2066696C65206EC6
:10E360006F7420666F756E640A005B5344434152BC
:10E37000445F4552524F523A25645D2046494C4510
:10E380005F526561644F70656E2829206861732053
:10E390006265656E2063616C6C6564207768696C8A
:10E3A000652070726576696F75732066696C65208B
:10E3B0006861736E2774206265656E20636C6F738D
:10E3C00065640A005B5344434152445F4552524FD7
:10E3D000523A25645D204446535F52656164466944
:10E3E0006C65206661696C65640A005B5344434157
:10E3F00052445F4552524F523A25645D206C65731A
:10E400007320627974657320726561642074686139
:10E410006E2065787065637465640A005B534443DD
:10E420004152445F4552524F523A25645D20444662
:10E43000535F52656164436C6F73652061626F72F4
:10E440007465642064756520746F207072657669E8
:10E450006F7573206572726F720A005B534443419B
:10E4600052445F4552524F523A25645D2046494C12
:10E47000455F57726974654F70656E206661696C9F
:10E48000656420746F20616C6C6F63617465206DCE
:10E49000656D6F727920666F72207772697465207E
:10E4A0006275666665720A005B5344434152445F7D
:10E4B0004552524F523A25645D204446535F4F7097
:10E4C000656E46696C65282E2E4446535F57524947
:10E4D00054452E2E29206661696C65640A005B53E1
:10E4E00044434152445F4552524F523A25645D20A5
:10E4F00046494C455F57726974654F70656E2829AF
:10E5000020686173206265656E2063616C6C656470
:10E51000207768696C652070726576696F75732005
:10E5200066696C65206861736E2774206265656E2C
:10E5300020636C6F7365640A005B5344434152442B
:10E540005F4552524F523A25645D204446535F570F
:10E550007269746546696C65206661696C65640AF8
:10E56000005B5344434152445F4552524F523A2557
:10E57000645D206C657373206279746573207772B3
:10E58000697474656E207468616E20657870656367
:10E590007465640A005B5344434152445F455252E0
:10E5A0004F523A25645D204446535F577269746543
:10E5B000436C6F73652061626F727465642064756B
:10E5C0006520746F2070726576696F75732065724F
:10E5D000726F720A005B5344434152445F4552528A
:10E5E0004F523A25645D2046494C455F5365656B43
:10E5F0002829206661696C65640A005B53444341C5
:10E6000052445F4552524F523A25645D204446536E
:10E610005F4F70656E446972282E2E4446535F52D8
:10E620004541442E2E29206661696C65642C206565
:10E630002E672E206469726563746F7279206E6F25
:10E640007420666F756E640A005B53444341524404
:10E650005F4552524F523A25645D2046494C455F12
:10E66000436F70792829206661696C65640A005BD4
:10E670005344434152445F4552524F523A25645DE0
:10E6800020736F757263652066696C6520646F65C1
:10E69000736E27742065786973740A005B53444372
:10E6A0004152445F4552524F523A25645D204649DB
:10E6B0004C455F476574446972732829206F722046
:10E6C00046494C455F47657446696C657328292047
:10E6D0006661696C65642062656361757365206F4E
:10E6E00066206D697373696E67206469726563740F
:10E6F0006F72790A005B5344434152445F45525262
:10E700004F523A25645D2046494C455F4765744643
:10E71000696C65732829206661696C65642062658F
:10E720006361757365206F66206D697373696E67C9
:10E73000206469726563746F72790A005B534443A5
:10E740004152445F4552524F523A25645D206572F2
:10E75000726F72207768696C652072656164696E9A
:10E7600067202E7379782066696C650A005B5344D4
:10E77000434152445F4552524F523A25645D204610
:10E78000494C455F4D616B6544697228292066617B
:10E79000696C65640A005B5344434152445F4552CF
:10E7A000524F523A25645D2046494C455F4C6F619B
:10E7B0006453657373696F6E4E616D6528290A0035
:10E7C0005B5344434152445F4552524F523A256491
:10E7D0005D2046494C455F557064617465467265BD
:10E7E00065427974657328290A005B53444341529A
:10E7F000445F4552524F523A25645D20736565204F
:10E8000066696C652E6820666F722064657363723A
:10E81000697074696F6E0A002D006D6B6469720017
:10E82000230064656C0072656164005B46494C4579
:10E830005D20446F776E6C6F6164206F6620256485
:10E8400020627974657320696E2070726F677265DB
:10E85000737320282564252529005B46494C455DB6
:10E8600020446F776E6C6F6164206F662025642092
:10E8700062797465732066696E69736865642E00D9
:10E880007772697465007E0030303030303030305F
:10E89000005B46494C455D2055706C6F6164696E44
:10E8A0006720257320776974682025642062797455
:10E8B00065730A00777269746564617461005B4610
:10E8C000494C455D2055706C6F6164206F66202552
:10E8D000642062797465732066696E697368656423
:10E8E0002E0025303858005B46494C455D20557058
:10E8F0006C6F6164206F6620256420627974657393
:10E9000020696E2070726F677265737320282564AA
:10E910002525290000202020202020202020282814
:10E9200028282820202020202020202020202020CF
:10E93000202020202088101010101010101010100F
:10E94000101010101004040404040404040404103F
:10E9500010101010101041414141414101010101CD
:10E960000101010101010101010101010101010197
:10E9700010101010101042424242424202020202A3
:10E980000202020202020202020202020202020267
:10E990001010101020000000000000000000000017
:10E9A0000000000000000000000000000000000067
:10E9B0000000000000000000000000000000000057
:10E9C0000000000000000000000000000000000047
:10E9D0000000000000000000000000000000000037
:10E9E0000000000000000000000000000000000027
:10E9F0000000000000000000000000000000000017
:10EA00000000000000000000000000000000000006
:10EA100000000000000000004300000000000000B3
:10EA200001007F000101000062616E6B2E0000009A
:10EA30000000000000000000FFFFFFFFAAAAAAAA32
:10EA4000FF1010101000000045A9000845A900089B
:10EA500045A9000845A9000845A9000845A90008DE
:10EA600045A9000845A9000845A9000845A90008CE
:10EA700045A9000845A9000845A9000845A90008BE
:10EA8000020406080000000001020304010203045E
:10EA900006070809FE00000014E900080000000055
:10EAA0000000000000000000000000000000000066
:10EAB00000000000000000000000000018EA00084C
:10EAC0000000000000000000000000000000000046
:10EAD0000000000000000000000000000000000036
:10EAE0000000000000000000000000000000000026
:10EAF0000000000000000000000000000000000016
:10EB00000000000000000000000000000000000005
:10EB100000000000000000000000000000000000F5
:10EB200000000000000000000000000000000000E5
:10EB300000000000000000000000000000000000D5
:10EB400000000000000000000000000000000000C5
:10EB500000000000000000000000000000000000B5
:10EB600000000000000000000000000000000000A5
:10EB70000000000000000000000000000000000095
:10EB80000000000000000000000000007C000020E9
:04000005080041E4CA
:00000001FF
